:020000040806ec
:100000000000060862f7150800008a131c000401ae
:100010000200d00700000000005000102100060878
:100020000d490e4a0e4b9b1a03dd043bc858d050b5
:10003000fbdc0b490b4a0020521a02dd043a8850bf
:10004000fcdc0949094a0a4b9b1a03dd043bc858ea
:10005000d050fbdc0748804718821508205100105b
:1000600000c5001018c6011080000608000000023c
:1000700098810f0271000002c809fa79010000009e
:1000800024b10d02d4270d0230280d0294b60d02c2
:1000900068b50d02c4b40d02bcb70d0208b40d0260
:1000a00060b70d021cb80d0268290d0218290d0257
:1000b00074b30d0264b80d0248b70d02c8b20d0248
:1000c000b4b40d025c560d02bc290d024cb60d02f3
:1000d0007cb60d02c8b50d022cb70d0294b10d020d
:1000e000bcb60d020cb80d02d0b20d02ffffffff2f
:1000f00053f04afc1bf074ff25f07ef81bf0faff6a
:1001000081f0004102e000bf83f0004330b54feac8
:1001100041044fea430594ea050f08bf90ea020f35
:100120001fbf54ea000c55ea020c7fea645c7feac8
:10013000655c00f0e2804fea5454d4eb5555b8bfeb
:100140006d420cdd2c4480ea020281ea030382ea5c
:10015000000083ea010180ea020281ea0303362dee
:1001600088bf30bd11f0004f4fea01314ff4801cc1
:100170004cea113102d0404261eb410113f0004fd3
:100180004fea03334cea133302d0524263eb43038a
:1001900094ea050f00f0a780a4f10104d5f1200e28
:1001a0000ddb02fa0efc22fa05f2801841f1000183
:1001b00003fa0ef2801843fa05f359410ee0a5f157
:1001c00020050ef1200e012a03fa0efc28bf4cf088
:1001d000020c43fa05f3c01851ebe37101f000453e
:1001e00007d54ff0000edcf1000c7eeb00006eeb4b
:1001f0000101b1f5801f1bd3b1f5001f0cd34908d5
:100200005fea30004fea3c0c04f101044fea44522b
:1002100012f5800f80f09a80bcf1004f08bf5feab2
:10022000500c50f1000041eb045141ea050130bd92
:100230005fea4c0c404141eb0101013c28bfb1f5a4
:10024000801fe9d291f0000f04bf01460020b1faef
:1002500081f308bf2033a3f10b03b3f120020cdac2
:100260000c3208dd02f1140cc2f10c0201fa0cf0a0
:1002700021fa02f10ce002f11402d8bfc2f1200c05
:1002800001fa02f120fa0cfcdcbf41ea0c019040bb
:10029000e41aa2bf01eb0451294330bd6fea040404
:1002a0001f3c1cda0c340edc04f11404c4f12002ef
:1002b00020fa04f001fa02f340ea030021fa04f301
:1002c00045ea030130bdc4f10c04c4f1200220fa58
:1002d00002f001fa04f340ea0300294630bd21fa96
:1002e00004f0294630bd94f0000f83f4801306bf5c
:1002f00081f480110134013d4ee77fea645c18bf50
:100300007fea655c29d094ea050f08bf90ea020fe6
:1003100005d054ea000c04bf1946104630bd91eade
:10032000030f1ebf0021002030bd5fea545c05d1e1
:100330004000494128bf41f0004130bd14f5800420
:100340003cbf01f5801130bd01f0004545f0fe4194
:1003500041f470014ff0000030bd7fea645c1abfc9
:10036000194610467fea655c1cbf0b46024650ea00
:10037000013406bf52ea033591ea030f41f400212c
:1003800030bd00bf90f0000f04bf0021704730b5b2
:100390004ff4806404f132044ff000054ff0000187
:1003a00050e700bf90f0000f04bf0021704730b548
:1003b0004ff4806404f1320410f0004548bf40421d
:1003c0004ff000013ee700bf42004feae2014fea72
:1003d00031014fea02701fbf12f07f4393f07f4f4d
:1003e00081f06051704732f07f4208bf704793f050
:1003f0007f4f04bf41f40021704730b54ff4607463
:1004000001f0004521f000411ce700bf50ea010265
:1004100008bf704730b54ff000050ae050ea01020e
:1004200008bf704730b511f0004502d5404261eb7e
:1004300041014ff4806404f132045fea915c3ff4bf
:10044000d8ae4ff003025feadc0c18bf03325fea5c
:10045000dc0c18bf033202ebdc02c2f1200300fa0d
:1004600003fc20fa02f001fa03fe40ea0e0021fa32
:1004700002f11444bde600bf70b54ff0ff0c4cf420
:10048000e06c1cea11541dbf1cea135594ea0c0fd2
:1004900095ea0c0f00f0def82c4481ea030621ea0d
:1004a0004c5123ea4c5350ea013518bf52ea033548
:1004b00041f4801143f4801338d0a0fb02ce4ff0fa
:1004c0000005e1fb02e506f00042e0fb03e54ff02a
:1004d0000006e1fb03569cf0000f18bf4ef0010e22
:1004e000a4f1ff04b6f5007f64f5407404d25fea1e
:1004f0004e0e6d4146eb060642eac62141ea5551d1
:100500004feac52040ea5e504feace2eb4f1fd0c12
:1005100088bfbcf5e06f1ed8bef1004f08bf5fea90
:10052000500e50f1000041eb045170bd06f0004642
:1005300046ea010140ea020081ea0301b4eb5c04ef
:10054000c2bfd4eb0c0541ea045170bd41f48011e7
:100550004ff0000e013c00f3ab8014f1360fdebf0c
:10056000002001f0004170bdc4f10004203c35dae8
:100570000c341bdc04f11404c4f1200500fa05f36b
:1005800020fa04f001fa05f240ea020001f000420c
:1005900021f0004110ebd37021fa04f642eb060182
:1005a0005eea430e08bf20ead37070bdc4f10c04ac
:1005b000c4f1200500fa04f320fa05f001fa04f270
:1005c00040ea020001f0004110ebd37041f100015c
:1005d0005eea430e08bf20ead37070bdc4f1200567
:1005e00000fa05f24eea020e20fa04f301fa05f2cf
:1005f00043ea020321fa04f001f0004121fa04f277
:1006000020ea020000ebd3705eea430e08bf20ea46
:10061000d37070bd94f0000f0fd101f00046400080
:1006200041eb010111f4801f08bf013cf7d041ea02
:10063000060195f0000f18bf704703f00046520006
:1006400043eb030313f4801f08bf013df7d043ead7
:100650000603704794ea0c0f0cea135518bf95ea8d
:100660000c0f0cd050ea410618bf52ea4306d1d114
:1006700081ea030101f000414ff0000070bd50ea33
:10068000410606bf1046194652ea430619d094eabd
:100690000c0f02d150ea013613d195ea0c0f05d1a7
:1006a00052ea03361cbf104619460ad181ea0301fb
:1006b00001f0004141f0fe4141f470014ff00000b3
:1006c00070bd41f0fe4141f4780170bd70b54ff04e
:1006d000ff0c4cf4e06c1cea11541dbf1cea1355ce
:1006e00094ea0c0f95ea0c0f00f0a7f8a4eb0504b0
:1006f00081ea030e52ea03354fea013100f08880a7
:100700004fea03334ff0805545ea131343ea12636f
:100710004fea022245ea111545ea10654fea002624
:100720000ef000419d4208bf964244f1fd0404f5dd
:10073000407402d25b084fea3202b61a65eb030539
:100740005b084fea32024ff480104ff4002cb6ebf6
:10075000020e75eb030e22bfb61a754640ea0c0076
:100760005b084fea3202b6eb020e75eb030e22bfb6
:10077000b61a754640ea5c005b084fea3202b6ebf7
:10078000020e75eb030e22bfb61a754640ea9c00b6
:100790005b084fea3202b6eb020e75eb030e22bf86
:1007a000b61a754640eadc0055ea060e18d04fea44
:1007b000051545ea16754fea06164feac30343eae4
:1007c00052734feac2025fea1c1cc0d111f4801fb1
:1007d0000bd141ea00014ff000004ff0004cb6e7aa
:1007e00011f4801f04bf01430020b4f1fd0c88bf49
:1007f000bcf5e06f3ff6afaeb5eb030c04bfb6eb54
:10080000020c5fea500c50f1000041eb045170bd46
:100810000ef0004e4eea113114eb5c04c2bfd4eb73
:100820000c0541ea045170bd41f480114ff0000ef7
:10083000013c90e645ea060e8de60cea135594ea73
:100840000c0f08bf95ea0c0f3ff43baf94ea0c0f76
:100850000ad150ea01347ff434af95ea0c0f7ff4eb
:1008600025af104619462ce795ea0c0f06d152ea3f
:1008700003353ff4fdae1046194622e750ea410623
:1008800018bf52ea43067ff4c5ae50ea41047ff434
:100890000daf52ea43057ff4ebae12e74ff0ff3c99
:1008a00006e000bf4ff0010c02e000bf4ff0010c6a
:1008b0004df804cd4fea410c7fea6c5c4fea430ce3
:1008c00018bf7fea6c5c1bd001b050ea410c0cbf32
:1008d00052ea430c91ea030f02bf90ea020f002094
:1008e000704710f1000f91ea030f58bf994208bffb
:1008f00090422cbfd8176feae37040f001007047b8
:100900004fea410c7fea6c5c02d150ea013c07d10e
:100910004fea430c7fea6c5cd6d152ea033cd3d059
:100920005df8040b704700bf8446104662468c4653
:100930001946634600e000bf01b5fff7b7ff002886
:1009400048bf10f1000f01bd4df808edfff7f4ffaf
:100950000cbf012000205df808fb00bf4df808ed3a
:10096000fff7eaff34bf012000205df808fb00bf5d
:100970004df808edfff7e0ff94bf012000205df87f
:1009800008fb00bf4df808edfff7ceff94bf012034
:1009900000205df808fb00bf4df808edfff7c4ff2d
:1009a00034bf012000205df808fb00bf4fea410c76
:1009b0007fea6c5c02d150ea013c0ad14fea430c59
:1009c0007fea6c5c02d152ea033c02d14ff0000096
:1009d00070474ff0010070474fea410212f50012d4
:1009e00015d211d56ff47873b3eb625212d94fea76
:1009f000c12343f0004343ea505311f0004f23fa60
:100a000002f018bf404270474ff00000704750eab4
:100a1000013005d111f0004008bf6ff00040704771
:100a20004ff00000704700bf4a0011d212f50012cb
:100a300011d20dd56ff47873b3eb62520ed44fea36
:100a4000c12343f0004343ea505323fa02f07047b6
:100a50004ff00000704750ea013002d14ff0ff30f4
:100a600070474ff00000704753b94ab9002908bfda
:100a700000281cbf4ff0ff314ff0ff3000f096b957
:100a8000adf1080c6de904ce00f01af8ddf804e0d1
:100a9000dde9022304b07047430803f05533c01a60
:100aa000830800f0333003f03333184400eb1010a8
:100ab00000f00f3000eb002000eb0040000e70470c
:100ac0002de9f04f099d04460f46002b48d18a427c
:100ad000944661d9b2fa82f343b1c3f120019f4039
:100ae00002fa03fc9c4020fa01f10f434fea1c413b
:100af0001ffa8cfe220cb7fbf1f601fb167706fb02
:100b00000ef042ea0742904208d91ceb020206f1bd
:100b1000ff3702d2904200f237813e46121aa4b249
:100b2000b2fbf1f001fb102200fb0efe44ea02448e
:100b3000a64508d91ceb040400f1ff3202d2a645f9
:100b400000f21c81104640ea0640a4eb0e04002689
:100b50001db1dc400023c5e900433146bde8f08ffc
:100b60008b4209d9002d00f0fd800026c5e9000167
:100b700030463146bde8f08fb3fa83f6002e4bd1f4
:100b80008b42c0f0f280824240f2ef803046002d6e
:100b9000e3d0c5e90047e0e702b9ffdeb2fa82f32d
:100ba000002b40f09d80891a4fea124e97b2012621
:100bb000200cb1fbfef20efb121140ea014107fbd3
:100bc00002f088420fd91ceb010102f1ff382cbf63
:100bd0004ff001094ff00009884203d9b9f1000f25
:100be00000f0cf804246091aa4b2b1fbfef00efb22
:100bf000101100fb07f744ea0144a74208d91ceb97
:100c0000040400f1ff3102d2a74200f2b48008468a
:100c1000e41b40ea02409be7c6f12007b34001fa1b
:100c200006f422fa07fcf940b2404cea030c20fa21
:100c300007f34fea1c491c431ffa8cfe00fa06f327
:100c4000200cb1fbf9f809fb181140ea014108fb3f
:100c50000ef088420fd91ceb010108f1ff3a2cbfbe
:100c60004ff0010b4ff0000b884203d9bbf1000f8e
:100c700000f08d80d046091aa4b2b1fbf9f009fb4f
:100c8000101100fb0efe44ea01418e4507d91ceb12
:100c9000010100f1ff3401d28e457fd8204640eaa1
:100ca0000840a1eb0e01a0fb029841454c46c64608
:100cb00002d306d14b4504d20138b9eb020468ebec
:100cc0000c0e002d70d01a1b61eb0e0122fa06f3f8
:100cd00001fa07f7f14000261f43c5e900713ce720
:100ce00002fa03fcc3f1200001fa03f221fa00f634
:100cf0004fea1c4e24fa00f11ffa8cf79c40114376
:100d0000b6fbfef00a0c0efb106642ea064200fb40
:100d100007f696420ed91ceb020200f1ff382cbff9
:100d20004ff001094ff00009964202d9b9f1000fc6
:100d300031d04046921b89b2b2fbfef60efb162262
:100d400041ea024106fb07f28a4207d91ceb010186
:100d500006f1ff3801d28a4223d84646891a46ea6c
:100d6000004625e72e462846f7e6841a61eb030382
:100d700001201f460be76444023849e76444023807
:100d8000e1e6023a61442ee7023e6244c6e6a8f17b
:100d9000020861446fe702386244cbe702386144dd
:100da0007de7023e6144d9e72e46d6e6704700bf94
:100db00010f8012b11f8013b012a28bf9a42f7d005
:100dc000d01a7047034613f8012b002afbd1181ada
:100dd000013870477bb972b90029bebf00204ff0bf
:100de000004106e008bf00281cbf6ff000414ff033
:100df000ff30fff7dbbfadf1080c6de904ce002931
:100e000009db002b1adbfff75bfeddf804e0dde910
:100e1000022304b07047404261eb4101002b1bdb11
:100e2000fff74efeddf804e0dde9022304b04042a6
:100e300061eb4101524263eb43037047524263eb63
:100e40004303fff73dfeddf804e0dde9022304b0d3
:100e5000404261eb41017047524263eb4303fff7ad
:100e60002ffeddf804e0dde9022304b0524263eb1b
:100e70004303704709b504480068044b03441b68ea
:100e80001b68029309bd000034cb00100400000071
:100e900009b504480068044b03441b685b6802936f
:100ea00009bd000034cb00100400000009b504485f
:100eb0000068044b03441b689b68029309bd000053
:100ec00034cb00100400000000b1807b704708b1f3
:100ed000c07b7047ff20704708b1408970474ff6cc
:100ee000ff70704708b1808970474ff6ff707047f8
:100ef00042680068101a704709b504480068044b3e
:100f000003441b681b68029309bd000034cb00102a
:100f1000000000007047000010b5002101201af009
:100f20009dfe04461af01cff24b9bde810400420c1
:100f30000bf080be0028f8d102482df08ffb00286e
:100f4000f3d110bd0ccb001008b50bf091fe0438a6
:100f500018bf012008bd000010b5fff7f5ff20b154
:100f6000bde81040014bdb69184710bd0ccb0010e9
:100f700010b5fff7e9ff20b1bde81040014b5b6af7
:100f8000184710bd0ccb001010b5fff7ddff20b1e6
:100f9000bde81040014b1b6a184710bd0ccb001078
:100fa000f8b504460e4617461d4624b92846bde846
:100fb000f84025f010bde72000f042f9304625f05a
:100fc0000afde72000f060f9384625f004fd013cf9
:100fd000ebe70000014b1860704700bf38cb0010f2
:100fe0002de9ff410446002003911bf0e7f8234b55
:100ff0001b6813b12046039998474ff47f0000f017
:101000007ff8602000f09ef800f090f80023009335
:1010100001231b4a18461b4901f026f8e72000f07f
:1010200033f94ff47f0000f06bf80226164ddff81d
:101030006880164f2b4641460320134afff7b0ff46
:101040002b4639460320104afff7aaff2a4641469d
:1010500003200f4bfff7a4ff3a4620460d4b0b49e8
:10106000fff79eff012e07d100222146822004b007
:10107000bde8f0411af046be0126dbe738cb001090
:10108000a5a80d02b4290d02a0860100e09304007a
:10109000a0bb0d0000350c00f049020037b500255b
:1010a0000195069d079c009500f074fa04b120603c
:1010b0007f28a8bf7f2040b203b030bd10b5054bdc
:1010c0001b7800fb03f4044b0020db689847604367
:1010d000000c10bd3a5100102051001038b50546e3
:1010e000c0f307400c46fff7e9ff2080c5f3072057
:1010f000fff7e4ff6080e8b2fff7e0ffa08038bdb3
:10110000014b1860704700bf40cb0010014b1860c6
:10111000704700bf44cb001010b9024b18687047ed
:10112000014bfbe740cb001044cb0010044b1a7876
:1011300022b100210120197001f0b2b8704700bf40
:101140003ccb0010014b1870704700bf3a510010a3
:10115000014b1878704700bf3a510010024b1860dd
:10116000024b1960704700bf48cb00104ccb0010f9
:1011700010b5054b0446db68002098472402b4fbf9
:10118000f0f0c0b210bd00bf205100102de9f341b6
:10119000dff83480044600216846d8f808309847c4
:1011a0006e46671e02340020d8f80c3036f8025b19
:1011b00098472d02b5fbf0f507f8015fa742f2d181
:1011c00002b0bde8f08100bf2051001010b4054b03
:1011d00082885c684188a446002300885df8044b3f
:1011e000604700bf2051001030b50e4d85b0044659
:1011f000fff7ecff2b689bb12088fff7b9ff039046
:101200006088fff7b5ff0290a088fff7b1ffdde926
:10121000022103460020009003482c680068a04784
:1012200005b030bd48cb00104ccb001007b5694667
:10123000fff754ff6846fff7d7ff03b05df804fbe4
:1012400008b510b1e72805d008bd0120bde8084069
:1012500024f0f3bd074b1b7853b1074b1868fff719
:10126000e5ff6322054b1a70ff22054b1a70ebe76e
:10127000044bf3e73ccb001044cb00103951001075
:101280003851001040cb001008b510b1e72804d049
:1012900008bdbde8084024f0d0bd0020fff7c6ff20
:1012a0000022034b1a700122024b1a70f0e700bfb4
:1012b000395100103851001013b518b1e72807d084
:1012c00002b010bd104b5b6902b0bde8104018477a
:1012d0000e4b1b78a3b10e4b1c680b4b00219b6877
:1012e00068469847bdf80220bdf800301343bdf8aa
:1012f000042013439bb22bb10020fff797ffdfe7d9
:10130000044be9e72046f8e7205100103ccb0010e1
:1013100044cb001040cb001038b5094b1a7802f0ce
:10132000ff0462b90125214620461d7000f0b8ff78
:101330002046fff77bff034b1c70034b1d7038bd2d
:101340003ccb0010395100103851001013b5044641
:1013500008466946fff7c2fe6322bdf800306343ca
:10136000b3fbf2f3adf80030bdf802306343b3fbda
:10137000f2f3adf80230bdf8043004fb03f0b0fb2b
:10138000f2f0adf804006846fff72eff02b010bd82
:1013900010b40f4c024623780e4983b9012008701f
:1013a0000878e72a0344d8b220700ed10a4b1b7884
:1013b0004bb10a4b19685df8044bfff7c7bf632bad
:1013c000eed1ff20ebe7064bf4e75df8044b7047e6
:1013d00039510010385100103ccb001044cb0010a4
:1013e00040cb0010024b1878003818bf012070471e
:1013f0003ccb001084b030b503ac84e80f00064c41
:1014000003ad0fcd0fc495e8030084e80300bde8e9
:10141000304004b0704700bf2051001070b5054641
:1014200000200e46144631f07dfe40b12346324680
:101430006968403058f07cf8231a5842584170bd12
:1014400070b5054600200e46144631f06bfe40b1e3
:10145000234632466968403058f025fa231a58422c
:10146000584170bd01211020baf014be08b510b16a
:10147000bbf006f8012008bd01210c20baf00abe1d
:1014800008b510b1baf0fcff012008bd30b5044624
:1014900085b078b1684639f04ffa6a46234604ad04
:1014a000144603ccac4218605960224603f108038d
:1014b000f6d1012005b030bd1fb5044648b101a8e2
:1014c00039f0e6fd01ab03cb206018686160a060d5
:1014d000012004b010bd000038b50d46044608b91f
:1014e000002038bd0029fbd0002031f01bfe002871
:1014f000f6d00023e360044b0120c4e900354ff02f
:10150000ff33a360ede700bf9d130002f8b50e4660
:10151000054608b90020f8bd0029fbd0002031f0b5
:1015200001fe04460028f5d040343146204657f0ed
:1015300004fe07463146204657f001fe002fe9db46
:101540000028e7db034bc01ba860c5e9003601207b
:10155000e1e700bfc1130002002908bf3221024b9e
:101560001970024b186070473b51001054cb0010ab
:1015700070470cb402b07047034b1860034b1960fe
:10158000034b1a60704700bf58cb00105ccb0010b3
:1015900050cb00102de9f04f4ff0010c00244ff01c
:1015a000ff36d0f804e0964504d211f80e80b8f169
:1015b000000f09d18268511e03eb0213002980f24b
:1015c000a8812046bde8f08fb8f13a0f7dd033d81e
:1015d000b8f1220f00f0a58010d8a8f109085ffa31
:1015e00088f8b8f1170f0dd8ac4d0cfa08f818eac6
:1015f000050f07d0456801354560d2e7b8f12c0fdb
:1016000000f02981d0f8048042450ed911f8085025
:101610005db13a2d00f25e811f2d00f246810a2d48
:1016200000f25581082d40f24b81002b40f057818c
:1016300008f1ff354560a4e0b8f17b0f1dd00ad852
:10164000b8f15b0f19d0b8f15d0fdbd1002bd1d011
:101650004ff0020906e0b8f17d0fd3d1002bc9d0bd
:101660004ff001098568013d03eb0518002d2fdac5
:101670000135bfd16ff00104a3e70134002bb9d0cd
:101680008568099faf4265d905f1010ec0f808e0f1
:101690004fea051a03eb051e0025cee90166cef8d8
:1016a0000c50c5686f1c1fbf03eb0519d9f80c500f
:1016b0000135c9f80c50b8f17b0f0cbf012502258c
:1016c00003f80a504568cef804508568013d1ce0d7
:1016d000d8f8047001371ad0d8f808a0baf1ff3f43
:1016e00015d198f800b0cb45c4d10ef1010ec0f869
:1016f0000ca0c8f808e003eb051edef80470013703
:1017000009d0def80870013705d1c56072e7013de8
:10171000a8f11008aae7013d6f1caef1100eecd144
:1017200068e70ef10109c0f80490d0f80480424542
:1017300002d911f8085025b9c0f804e06ff002048e
:101740003fe7222d2dd1e3b18568099faf4204d830
:10175000c0f804e04ff0ff3433e700274ff0030aee
:1017600005f1010e4fea051803eb0515c0f808e076
:10177000c5e90166ef60d0f804e003f808a0c5e908
:10178000019ec56801346f1c3ff434af002b3ff459
:1017900031af03eb051edef80c500135cef80c50ce
:1017a00028e75c2d11d108f1010595420dd2456065
:1017b0004d5d752d2cd86d2d0bd8662d28d85b2d41
:1017c0001ed8222d01d02f2d22d14568013545602c
:1017d000abe76e3d072d1bd801a757f825f000bfda
:1017e0004b17000291170002911700029117000297
:1017f0004b170002911700024b17000297170002c7
:1018000040f241475c3dedb20cfa05f53d42dcd1ba
:10181000c0f804e02ee74ff0040a08f10205456025
:10182000d0f80480424512d911f808507db1a5f1d5
:10183000300bbbf1090f04d925f02005413d052de2
:10184000e6d808f10105baf1010a4560e8d145681a
:10185000013d4560b9e7002b3ff4ccaec5682d01d2
:101860005d5d013d012d7ff6c5ae856805f1ff3850
:1018700003eb051eb8f1000ffff6bcae1ef8105cbe
:10188000013d012d0cd85ef80c5c013508d05ef8e6
:10189000085c013504d1c0f80c80abe61300800071
:1018a00008f1ff38aef1100ee4e7a5f120091f4f53
:1018b0005ffa89f90cfa09f919ea070f7ff4b5ae56
:1018c000203d5e2da4d808f1010545609ae60d2d56
:1018d000f6d1aae605f0df09b9f15d0ff8e78568f2
:1018e000099faf427ff634af002705f101084feaa8
:1018f000051903eb0515c0f80880c5e90166ef601e
:10190000d0f8048003f80970c5e901e84568013d95
:1019100090e653f80c2c013204d053f8082c013215
:101920003ff40caf0139103b48e600bf0110000442
:101930000023c0e901334ff0ff33c36070476ff0fd
:10194000770070476ff0770070476ff0770070474f
:101950006ff0770070476ff0770070470020704796
:10196000002070472de9f34180460c46002627f001
:10197000e0ff37460546d8f8003040469b69984757
:10198000002834db18d0d8f80030012240461b690b
:101990008df807700df107019847002827dbd8f86c
:1019a0000030012140465b69984700281fdb013663
:1019b000e1e700241d46dee7c4b1d8f80030224636
:1019c00053f8140c012158f8003040449b689847a4
:1019d00010f1a00f0ad0002809db27f0aaff431b53
:1019e0009c42e6d92c440346241ae3e7304602b071
:1019f000bde8f0812de9f0418046c2b000200d46df
:101a0000174631f08ffb044618b34ff4847200215f
:101a100068464034baf081fd6a462946204657f0b0
:101a200097fb50b32f212846bcf003fcb8b1854288
:101a300015d0411b2846bcf0cdfb0646c8b1014677
:101a4000204658f0e3fb38b1113005d03046baf0eb
:101a500017fd6ff0e0000de03046baf011fd47f4dd
:101a600080773b462a464146204658f0cdfc08b1d7
:101a7000efe7044842b0bde8f0819df80030112b3b
:101a8000efd0e6e7fcfefffff8b5074600200d4665
:101a90001646fff7f1fc0446a0b100223946fff7d5
:101aa00035fd28b132462946204639f021fe38b9a5
:101ab0006ff0e00500212046fff7e2fc2846f8bd64
:101ac0000025f7e7004df9e7fcfefffff8b50746f4
:101ad00000200d461646fff7c5fc0446a0b10022c3
:101ae0003946fff7f9fc28b132462946204639f03d
:101af00003f938b96ff0e00500212046fff7b6fc86
:101b00002846f8bd0025f7e7004df9e7fcfeffff8a
:101b10000fb413b50a4b586a2df029fe58b1094c81
:101b200005ab80212046049a0193bcf02fff0028ca
:101b3000bcbf0023237002b0bde8104004b0704762
:101b40009ccd001060cb001008b5044b586a2df0f6
:101b50000efe10b10022024b1a7008bd9ccd001081
:101b600060cb0010021e80f2348112f5967f00f0e7
:101b7000328100f3b580a64b9a4200f02e810133ea
:101b80009a4271da12f5c86f51dca3f580739a425c
:101b90003edaa0487047c9320b2afad801a353f89d
:101ba00022f000bf2b1d0002271d0002131b0002a4
:101bb000131b0002131b0002131b0002131b000265
:101bc000131b0002131b0002131b0002231d000243
:101bd0005f1d0002e6320b2adbd801a353f822f086
:101be0003b1d0002131b0002131b0002131b00020b
:101bf000131b0002371d0002131b0002131b0002ff
:101c0000131b0002331d00022f1d0002631d000282
:101c100002f24562052a00f2da80dfe812f0d6000f
:101c2000d400d200d000e40006007b4870477b4b14
:101c30009a4200f0da8001339a420ada12f5af6f65
:101c400000f0d5807649734b76488a4218bf184613
:101c50007047754b9a4200f0cc806e48734b12f57a
:101c6000aa6f08bf18467047714b9a4200f0c380b4
:101c700001339a421bda1f3b9a4200f0be806ff498
:101c8000a6639a420bda0b3b9a4200f0b880093304
:101c90009a4200f0b68067495e4b6748d5e712f577
:101ca000a56f00f0b08065495a4b6548cde7654b9c
:101cb0009a4200f0aa8001339a4208da4f3b9a42d6
:101cc00000f00a815348604b12f5966fc9e75f4bed
:101cd0009a4200f003814f485d4b12f57a7fc0e7ce
:101ce00012f1bd0f2eda12f1c90fbff654af12f187
:101cf000da0f20da12f1e60fbff66caf12f5827f31
:101d000000f0ee800cdc12f58c7f00f0eb8012f519
:101d1000877f00f0e9803f484e4b12f5917fa0e7a6
:101d200012f1fa0f00f0e2803a4b4b4812f1f00f3b
:101d300018bf18467047374b484812f1d20f18bfea
:101d40001846704712f18c0f00f0d28012f18b0f01
:101d500018da12f1a00f00f0cd8012f19f0f0ada0d
:101d600012f1b40f00f0c8802a4b3d4812f1aa0fbf
:101d700018bf18467047274b3a4812f1960f18bf04
:101d80001846704712f1780f00f0b88012f16e0f0c
:101d900000f0b6801f4b344812f1820f18bf18466e
:101da000704732487047324870473248704732486f
:101db000704732487047324870473248704732485f
:101dc000704732487047324870473248704732484f
:101dd000704732487047324870473248704732483f
:101de000704732487047324870473248704732482f
:101df000704732487047324870473248704732481f
:101e0000704732487047324870473248704700bfc9
:101e1000b9faffffb02a0d02642b0d029cfafffff6
:101e200092faffff6d2b0d02a6faffff382c0d0270
:101e3000ecfaffffbafaffff082c0d02e2faffffef
:101e4000762c0d0294fbffff892c0d02b4fbffffe3
:101e5000e32c0d02ee2c0d023e2d0d02c42d0d02c1
:101e6000ba2d0d02902a0d02f42d0d026a2d0d02dd
:101e70005b2d0d024d2d0d02352d0d02232d0d0272
:101e8000182d0d020a2d0d020b2b0d02f92a0d0241
:101e9000e72a0d02d52a0d02be2a0d02af2c0e0232
:101ea000992b0d02e02d0d027a2d0d022f2d0d0222
:101eb000262b0d02392b0d02572b0d02832b0d0201
:101ec000f72b0d02ba2b0d02d82b0d02a42b0d02fd
:101ed0001f2c0d02502c0d020a4870470a4870470b
:101ee0000a4870470a4870470a4870470a487047ce
:101ef0000a4870470a4870470a4870470a487047be
:101f00000a4870475a2c0d029c2c0d02b72c0d026a
:101f1000cf2c0d02a62c0d02fb2c0d02a62d0d02be
:101f2000892d0d02972d0d02a22a0d02d22d0d0230
:101f300010b5084b0446586a2df019fc10b106483c
:101f400003782bb92046bde810400021fff70abef8
:101f500010bd00bf9ccd001060cb0010a0f130037d
:101f6000dab2092a01d818467047a0f16103052b9f
:101f700001d857387047a0f14103052b94bf37387b
:101f80004ff0ff307047102af8b506460c461bd9b3
:101f900000252078fff7e2ff071e15db6078fff7ca
:101fa000ddff031e10db43ea0713052d735505d132
:101fb00002340135062decd1012006e0a278e31ca5
:101fc0003a2a01d11c46f4e70020f8bd034b186003
:101fd000034b1960034b1a60704700bfe0cb001041
:101fe000e4cb0010e8cb0010f0b5164b05461e6898
:101ff0000f461446abb036b9134b1b6803b3134bf3
:102000001b7883421cdc23791b0706d427f091fc44
:102010002379606143f0080323718eb1dde9302339
:10202000a02102a8bcf0b2fc9f28c4bf7e238df87b
:10203000a63000233a4600932946234602a8b0471b
:102040002bb0f0bde0cb001054cb00103b51001082
:1020500030b585b008ac54f8045bcde90054039466
:10206000fff7c2ff05b030bd70b404460d46104600
:1020700019464bb1054b1e6836b100232246039327
:10208000b4462b4670bc604770bc7047e4cb001070
:1020900070b51a46134b04461d680e46aab035b9f2
:1020a000114b1b68bbb1114b1b78834213dc2e9b79
:1020b000a02102a8bcf06afc9f28c8bf7e2301466d
:1020c000c4bf8df8a6309f213db100232246009366
:1020d00002a83346a8472ab070bd034b02a81b686c
:1020e0009847f8e7e4cb001054cb00103b510010a8
:1020f00008b410b585b007ac54f8043b00940394c1
:10210000fff7c6ff05b0bde8104001b07047000002
:102110002de9f04f8846294907460d68adb0002be0
:102120003ad035b926490968b1b3264909788142c0
:1021300032dc00211446dff89090dff884b08df88f
:10214000ac10d61814f8013b2ca84fea131c19f850
:102150000cc0084403f00f034a1c00f8a4cc19f883
:10216000033002312ca80244a02902f8a43c09d172
:10217000adb14ff0000a43463a46cdf800a003a89f
:10218000a8475146a642ddd131b175b100233a4688
:10219000009303a84346a8472db0bde8f08fdbf8b5
:1021a000003003a898472946ece72cab1944044bb0
:1021b00001f8a45c1b6803a89847ede7e4cb001086
:1021c00054cb00103b510010342e0d02074b024639
:1021d0001b680bb100221847054b186828b1054b46
:1021e0001b789a42b4bf002001207047e8cb001052
:1021f00054cb00103b5100104528dabf0a2390fb56
:10220000f3f00620034bd8bf20eae07053f820001b
:10221000704700bf182e0d0270b50d46044620b958
:102220000a201c4a1c49fef7dbfe19f013fca37bb5
:10223000db070bd563680bb1a2689a60d4e9013261
:1022400082b15360a37b03f0fe03a37313490b68b1
:102250006db1002283b11e7b257bae420bd91a469d
:102260005b68f7e70d4a1360ece70c6007e063b9c1
:1022700001238b7409e09c60002af6d05460c4e905
:102280000132a37b43f00103a373bde8704019f052
:10229000e5bb00bf57690202452e0d02eccb0010d2
:1022a00010b5044619f0d6fb094b1a8a5cb1013a05
:1022b00092b21a821a8a92b20ab901229a74bde8bd
:1022c000104019f0cbbb013292b21a82f7e700bf7f
:1022d000eccb001010b519f0bdfb044b1c8a19f0b3
:1022e000bdfba4b2b4fa84f0400910bdeccb0010e1
:1022f0002de9f04f85b04ff00009054619f0aafb13
:10230000ca4683464b46012049464f464e464a46fa
:10231000614cd4f8008010b3b8f1000f1fd098f8ca
:102320000d300f2b5ffa83fa15d1d8e90531284615
:1023300098470022d8f8106098f80e10238a94f875
:1023400012909bb2b3fa83f30020c9b25b095ffa23
:1023500089f9a274dde7b8f81470bfb2eae758460d
:10236000cde9021319f07afbdde90213a27a524596
:1023700002d1a289ba4261d0002284f80aa0a781c2
:10238000e281002b57d011f0020067d1434bc6f316
:1023900007481f78424bffb2db6898477843f5b295
:1023a000c6f3072700fb08f847434543b4f80cc0c1
:1023b0004fea18413a0c280c884617460546bcf1ee
:1023c000000f05d0a67ae389022e44d0032e49d00f
:1023d000b9f1000f08d1a388434505d1e388bb427a
:1023e00002d12389ab4226d0dff8b4900023d9f87c
:1023f00004602a4639464046b0472a4e3368b3b196
:10240000d9f80c30002098474fea08212b023a02f5
:10241000b3fbf0f3b2fbf0f2b1fbf0f0002100915e
:10242000c1b2214836680068dbb2d2b2b047a4f826
:102430000480e780258105b0bde8f08f002fa0d093
:10244000e0890544adb2bd4224bfb5fbf7f207fbfe
:102450001255e58195e7b3eb5c0fb9d300252f4604
:10246000a846b5e74fea5c06b3eb5c0f34bff31a3e
:102470009b1b9bb203fb01f803fb02f703fb00f578
:10248000b8fbf6f8b7fbf6f7b5fbf6f51ffa88f8d8
:10249000bfb2adb29ce700bfeccb00103a510010c8
:1024a0002051001048cb00104ccb0010064b0022ee
:1024b000194641f8042b5a601a828a805a81da60e0
:1024c00001229a74704700bfeccb001070b5d0e9c0
:1024d0000043204643f31d03002b0ddd5a1050f836
:1024e000226000eb8205b6888e4203d29b1a281d1b
:1024f000013bf1e71346efe7001b801070bd0000c1
:1025000070b51048d0e88f5f15f001050e4e16d15a
:1025100025f03efc98b1102023f026fb044650b174
:10252000c0e90055856005738020b9f0a1ff10b1a6
:1025300020232060a3600348346025f063fc3068ea
:1025400070bd00bf00cc001004cc0010f8b50746e9
:10255000fff7d6ff037b044673bbb988fff7b6ffce
:102560000546d4e90006b54204da50f825309b88c8
:102570008b4224d0a3689e420ddb0136002e05dd80
:10258000b100baf04bff20b90e4814e0b9f078ff63
:1025900000202060a6602668626806eb8501920034
:1025a000a2eb8502081db9f09eff002046f82570b9
:1025b000636801336360f8bd6ff0d100fbe76ff033
:1025c000b300f8e7fcfeffff2de9f84307460e468f
:1025d0009046fff795ff037b0546a3b177b1d0e99d
:1025e000004304eb83094c45234607d04146186855
:1025f0000434b8470028f6d0bde8f88336b16b68dc
:1026000000203360f8e76ff0d100f5e73046f3e7dc
:1026100070b506460c46fff773ff037b05467bb19a
:102620003146fff753ff6b6898420cda2b6853f87a
:1026300020309a88b24206d144b10020236070bd98
:102640006ff0d100fbe76ff0a900f8e72046f6e74e
:1026500010b50446fff754ff022c05bf0123037396
:102660006ff07700002010bd38b538220d460021ec
:102670000446b9f052ff4ff0ff3200232046c4e970
:102680000f23a56338bd000030b505468db000208e
:1026900030f048fd044618b330f07afc2b6c9907f3
:1026a00006d40025204630f097fc28460db030bdfa
:1026b000294604f1400057f0bbfb0028f1da202244
:1026c00000230290cde90423aa6b32200192064a2e
:1026d0000649009204aafff7bbfc6ff0e005e1e7b2
:1026e0006ff0e005e1e700bf652e0d025d2e0d02e3
:1026f000002370b501f14006044601461a463046f3
:102700008eb057f034f900284ff0000511da20237d
:10271000cde90635a36b029001930f4b3220009355
:102720000e492b4606aafff793fc6ff0e0000eb0af
:1027300070bd04232146304605aa059557f0b3f82d
:10274000042807d02023cde90635a36b029001931e
:10275000034be3e70598eae7842e0d025d2e0d0298
:10276000a32e0d0210b50446236c08468cb0abb105
:102770002146403057f0a4fb00280dda2022002328
:10278000cde90423a26b02900192054a3220009207
:10279000044904aafff75cfc002323640cb010bdbd
:1027a000c22e0d025d2e0d0238b50546002030f018
:1027b000b9fc044650b130f0ebfb28462146fff748
:1027c000d1ff2046bde8384030f006bc38bd0000df
:1027d00030b505468db0002030f0a4fc044610b39f
:1027e00030f0d6fb21462846fff7bcffa96b04f169
:1027f000400057f011fe00280fda811c0dd0202276
:102800000023cde90423aa6b02900192074a3220eb
:102810000092074904aafff71bfc20460db0bde853
:10282000304030f0d9bb0db030bd00bfe22e0d02fc
:102830005d2e0d02002a70b540f6031518bf012564
:10284000036c044635ea03030e468cb01fd0fff735
:1028500089ff2b462146a26b06f1400057f0d4fdbc
:10286000002813da811c14d020220023cde9042390
:10287000a26b02900192084a32200092074904aaf2
:10288000fff7e6fb6ff0e0000cb070bd25640020a0
:10289000fae76ff0a900f7e7fe2e0d025d2e0d029c
:1028a0002de9f04705468cb000208946904630f06f
:1028b00039fc0746002863d030f06afb0122394614
:1028c0002846fff7b7ff041e1bdb07f1400a294625
:1028d000504656f034fc061e10da20200023aa6b66
:1028e000cde904030192284a02960092322027493a
:1028f00004aafff7adfb6ff0e00402e0032e07dc53
:10290000234c384630f068fb20460cb0bde8f08719
:10291000eb6b002b09da39462846fff7e9fe041e67
:10292000efdb17d1042eebd1ec63ea6b002390456b
:10293000a8bf904629465046b21a57f018f800280a
:102940000cda20210023aa6bcde904130192029036
:10295000104acae7f31ea342e6dcd1e743464a46e3
:102960002946504656f09fff80450446c9d0202294
:102970000023cde90423aa6b02900192064ab4e732
:102980006ff0e004c0e700bf1d2f0d025d2e0d02a9
:10299000e8feffff842e0d02a32e0d022de9f04765
:1029a00005468eb000208946164630f0bbfb8046b7
:1029b00000287fd030f0ecfa002241462846fff78d
:1029c00039ff041e18db08f1400a2946504656f02c
:1029d000b6fb071e17da4ff0200c0023aa6bcde9d7
:1029e00006c30192354a029700923220344906aa62
:1029f000fff72efb6ff0e004404630f0edfa204682
:102a00000eb0bde8f087032f0fdc002229465046a8
:102a100056f0c6ff002828da20260023aa6bcde94d
:102a2000066301920290274adee7eb6b002b06da81
:102a300041462846fff75cfe041edddbec63eb6bd2
:102a4000b342e2d13744b7f5805fdedc33464a4615
:102a50002946504656f06cfd86420446ccd02022d2
:102a600000230290cde906231ee0002329461a46e2
:102a7000504656f07cff002808da20240023aa6b79
:102a8000cde90643019202900f4aade7042329469f
:102a9000504605aa059656f04bfd042808d0202183
:102aa0000023cde906130290aa6b0192074a9be727
:102ab000ee63cbe76ff0e004a1e700bf1d2f0d022e
:102ac0005d2e0d023c2f0d02842e0d025f2f0d0294
:102ad00010b401291346c06808d102685968146807
:102ae00003f1080223465df8044b18476ff07700a6
:102af0005df8044b704738b5144619b904220846ee
:102b0000226038bd1368032b07d903685b689847b8
:102b10000028f6d104232360f3e76ff0bd00f0e74f
:102b2000836900200b607047836900200b60704749
:102b300013b5114b0c461b7e062b1ad0cbb10121cd
:102b4000684611f021f8684610f0e1ff684611f080
:102b50009bf9dfed0a7a20ee270abceec00a10eee0
:102b6000103a9bb26846236011f01ef8002002b0b4
:102b700010bd6ff0d100fae720cc001000008043b8
:102b80000a4b10b5036014234360012304464381bc
:102b9000074bc0e903200181436100210430fff7a6
:102ba000d5fc044b2046236010bd00bf08360d0243
:102bb000512a000214360d0210b50446fff7e0ff5b
:102bc000014b2046236010bd44360d0208b506f0c7
:102bd000c3fbbde8084006f0d5bb07b5019006f081
:102be000bbfb019903b05df804eb06f0f5bd08b539
:102bf00006f0b2fbbde8084006f0febb07b5019049
:102c000006f0aafb019903b05df804eb06f09ebc48
:102c100007b5019006f0a0fb019903b05df804eb45
:102c200006f0aabc38b500250b4c03210b4a0c4812
:102c3000fff7c2ff072120460a4afff7a1ff0a4b10
:102c4000a5612360094c18212046094afff798ff27
:102c5000084ba561236038bd20cc0010e2350d0281
:102c600008cc0010eb350d0224360d023ccc0010d0
:102c7000f6350d0234360d02074b1a7812b10021d9
:102c8000064a11705a7812b10121054a11709b78d9
:102c90000bb109f09fbf704758cc001012d1001043
:102ca00010d10010fff7e8bf10b5c36804460bb998
:102cb000b8f08cfe0369043098470021a061606978
:102cc000bde810402cf08cbe10b509f0abff124be4
:102cd000124c1b780246b3fa83f35b09a070237091
:102ce00080b10120002205216070104604f0fafa3c
:102cf00009f092ffbde8104000231a461946184615
:102d000004f08cbb014604f0c7f902460028e8d164
:102d1000014604f010fae5e712d1001058cc00107b
:102d2000012af8b5064603d10b6803600020f8bd00
:102d3000022a08d0032af9d100680028f6d01c2105
:102d400022f01afff2e71c200c6822f00dff074664
:102d500030b105460fcc0fc594e8070085e80700a1
:102d60003760e3e7012a70b5054603d10b680360bd
:102d7000002070bd022a08d0032af9d1006800287b
:102d8000f6d0102122f0f8fef2e710200e6822f0b3
:102d9000ebfe044618b196e80f0084e80f002c60a3
:102da000e6e721b18b88834201d08968f9e70846bc
:102db00070470000f8b5037d05460f46164653b12f
:102dc0000368d9680120fff7ecff044630b183891e
:102dd000bb4201d18673f8bd8168f3e7014610203c
:102de0000cf0bafb08b92c75f5e7054b036001231d
:102df00083802b698781836086732861ebe700bf3e
:102e00001000030008b5c1680120fff7caff28b110
:102e100083891b2b01d08168f6e7012008bd0000e3
:102e200038b5037d04460d463bb103680420d968dc
:102e3000fff7b7ff014608b1c56038bd10200cf0a0
:102e40008bfb08b92075f8e7044b036004238380eb
:102e50002369c0e902352061efe700bf10000300dd
:102e600010b58368044613b10322014698472046f3
:102e700010bd000010b50446034b40f8043bfff7bb
:102e8000efff204610bd00bf54360d0210b50446ba
:102e9000fff7f0ff2046142122f06efe204610bd01
:102ea00010b5074b04460360406918b12cf073fd60
:102eb000002363612046fff7ddff204610bd00bf01
:102ec00068360d0210b50446fff7eaff20461821c8
:102ed00022f052fe204610bd10b50446024b03609e
:102ee000fff7deff204610bd7c360d0210b504460c
:102ef000fff7f2ff20461c2122f03efe204610bdc7
:102f000038b50446006928b1856800210cf036fb0d
:102f10002846f8e7204638bd002330b587b0cde914
:102f20000233049301238df814301023adf80430dc
:102f3000032301ac00280d460094adf806308df84f
:102f4000083005dd4ff47a7141436846fff768ffaa
:102f5000ab0704d401220a216846fff72bff204665
:102f6000fff750ff80f00100c0b2fff736fe0022ed
:102f70002046114622f058fa04466846fff7c0ff83
:102f8000204607b030bd00002de9f0470e469846b8
:102f90001021002388b0cde904330693adf80c105e
:102fa000012303211746109a0df10c09002a05464a
:102fb000cdf808908df81c30adf80e108df810305b
:102fc00005dd4ff47a7102a85143fff729ffb5b12f
:102fd000beb1002f41d0b8f1000f3ed0002407eb66
:102fe000080ab4420dd0444535f8141034bf3a5d98
:102ff0001af8012c02a8fff7ddfe0134f1e72c4698
:10300000ede74846fff7fefe002780f00100c0b262
:10301000fff7e3fd3a46484601a9019722f004fa7a
:10302000041e11dbfff7e3fd0198c0b183883c4625
:10303000012b07d1b4420ed035f814308289013407
:103040009a42f7d1b9f01cfa02a8fff759ff2046bf
:1030500008b0bde8f0870024f4e7024cf4e704462a
:10306000f2e700bff2feffff73b506461c200d46d7
:1030700022f07afd044628b3144b03600023c3609a
:10308000ab683bb10222294604309847eb682361c4
:10309000ab68e360002220460d4b0121236040f81d
:1030a000142f2cf06dfc0b4b3046236033680194d9
:1030b0005b6801a99847054620b9236820469b68ac
:1030c00098472c46204602b070bd00bf54360d0212
:1030d00068360d027c360d02f0b51f463c4b164695
:1030e00093f82c2005460c4689b0f2b1586a2cf0b2
:1030f0003efbd0b90690102022f036fd18b1c0e991
:1031000001460570c760334b04900793324b30483b
:1031100004a90693fff7a8ff0546b8b9044604a81a
:10312000fff79efe204609b0f0bd02f091fbc8b942
:10313000f34313f0010300d195bbfff7c5fd012d4b
:103140003ed0022d3cd0bdb10024ebe700224ff071
:10315000ff3140692cf024fc2b6828469b68ac6941
:103160009847dce716f00403e2d11a460621012055
:1031700000940bf07dffdbe7002cd3d0e317cde903
:10318000044301212b46154a009504a8cde90655b4
:1031900026f01efd04460028c4d0fff76dfdc1e7f0
:1031a000012d0dd0022dcfd11a46184605210393cb
:1031b00004f098f8039b1a461946184604f02ef9b5
:1031c0003146204609b0bde8f040fff7a5be00bf7c
:1031d0009ccd001061310002e52c0002252c00027c
:1031e00000684168d0e902230078fff775bf2de938
:1031f000f0411f46002304460d46164601211a469b
:10320000184603f0b6ff3b46324629462046bde845
:10321000f041fff761bf00002de9f04f9846554b94
:10322000174693f82c2087b00546dde910940e462a
:1032300022b3586a2cf09bfa00bb04901c2022f0a9
:1032400093fc38b1129bc0e90056c0e90278c0e98e
:1032500004948361484b02900593484b454802a96a
:103260000493fff701ff0446002855d1054602a844
:10327000fff7f6fd284607b0bde8f08f02f0e8fa48
:103280008246002854d1e44314f001046dd0fff7c6
:103290001bfd4ff0000a00210846fff701f8e72068
:1032a000fdf7f2ff43463a4631462846cdf80090f6
:1032b000fff76afe002105460120fef7f1ffe72037
:1032c000fdf7beff002c4dd120461bf000f809f0a1
:1032d000cffc0446002009f0d7fc0646b8bb013cf1
:1032e000e4b2012c33d809f09dfc80b3304626f0bf
:1032f00013fb4ef660260446002026f00dfb001b53
:1033000061f10001b04271f100031ed202f0a0fa97
:10331000d8b902f0adfaefe700224ff0ff31406973
:103320002cf03efb236820469b68a56998479ee7e2
:1033300014f0040ba7d15b465a4606210120cdf8b4
:1033400000900bf095feda469de702f081fabaf1a3
:10335000000f8fd007f09afb002304211a4612f0c9
:10336000e2f887e7fff788fcb1e720461af0acffe8
:1033700091e700bf9ccd001001330002a12c000298
:103380001fb5006883690293436901930369009341
:10339000d0e90223d0e90001fff73eff05b05df858
:1033a00004fb2de9f0471f46dde9088900230446a8
:1033b0000d461646ddf828a01a460121184603f0ee
:1033c000d8fe3b46324629462046cde9099acdf83b
:1033d0002080bde8f047fff71fbf70b51d460023f2
:1033e00088b00e461446adf816001a46012118465c
:1033f00003f0bffe0c9b0094cde9015301230df1b6
:103400001f0219460df116008df81f60fff7c9ff66
:1034100008b070bd38b51546d0e902239342044682
:1034200007d2d21a4068aa4228bf2a461844b9f0e7
:103430004df8e26801202a44e26038bd012a02d139
:10344000016000207047022a04bf0b680360f8e7a0
:1034500013b5044608460191fdf7b4fc0246204628
:10346000236801991b6802b0bde8104018470000ae
:1034700004281fb5034614460cd14ff6ff7345f6da
:103480001b210920002a08bf194604b0bde81040de
:1034900018f0c2be01280ed100233c220093112354
:1034a00012481349002c18bf01461248006802f068
:1034b00091fd04b010bd09280ad100230b480c4926
:1034c0000093002c18bf014611233c220a48ede767
:1034d0000028eed1002aecd00246cde90100009090
:1034e00000214ff4007003f0adf9e2e788360d02d9
:1034f0008ea90d023c5100104051001009280a46c7
:1035000008b50dd8084b195c914203d1042801d0ad
:10351000082803d1195c1a54fff7aaff002001e024
:103520004ff0ff3008bd00bf4d510010092838b5dd
:103530000c4613d8a9b104280b4d0cd1092018f062
:1035400075fe45f61b2380b2c31a584258412070bd
:103550002871002038bd2b5c0b70fae74ff0ff306c
:10356000f8e70846f6e700bf4d51001037b50022d6
:103570000df107010546fff7d9ff044628b99df86c
:10358000072028461146fff773ff204603b030bde1
:10359000014b1860704700bf68cc001038b50b4b6a
:1035a00045681c6864b100f1080100222846a04764
:1035b000044618b10649284610f036fe204638bdac
:1035c0000449284610f030fe0349f4e768cc0010a7
:1035d0008d360d02bb360d02f1360d020c4a0d4b35
:1035e00000b51a601c2389b00021adf80430142303
:1035f000029001a8cde90311cde90511adf806103f
:103600000791adf80c30fff7c9ff09b05df804fb76
:103610002950000268cc001010b50f4b04461b68ff
:10362000834208d1002301211a46184603f0a1fd68
:10363000002011f06bf800221146104603f0e9fd5e
:10364000024640b9054b1b68a34204d1bde81040b7
:10365000014603f093bf10bd4451001048510010c3
:1036600030b50d4b05469b7885b003f0ff0483b958
:10367000224601210220fff741ff084b22461d7020
:103680004ff4806023460021cde90144009403f00b
:10369000d9f805b030bd00bf4d5100104c5100109d
:1036a00013b50024022022460df107018df80740d2
:1036b000fff73cff9df8070060b1224603200df1a3
:1036c00007018df80740fff731ff9df80700001b49
:1036d00018bf012002b010bd07b5fff7e1ffa0b190
:1036e0000b4b1a7802f0ff0342b1002302201a4666
:1036f000194603b05df804ebfff779bd0549009367
:103700001a460120097809f0c5fa03b05df804fbf8
:103710000dd500104c510010f0b585b0fff7c0ff7b
:1037200048b3164d2b7833bb01222a70144a4ff44c
:1037300000600021cde9013300921a4603f082f8bf
:1037400026f0f7f847f22f5704460e4efff7a8ff72
:1037500030b90020287005b0bde8f040fff7bcbfcd
:1037600026f0e7f8001bb842f3d802f081f83046a3
:1037700004f078f8eae705b0f0bd00bf6ccc0010ab
:10378000593600029ccd001037b5837a04460d46a9
:10379000ebb926f0abfe636818442389206113b9a6
:1037a00026f0b0fe2081e36813b926f0a5fee060a4
:1037b00015f0010f0cbf0025042504f06dfd00235a
:1037c000e1681a46009505f081f803b030bd014864
:1037d000fbe700bfe2faffff2de9f0411646ca07fa
:1037e00088b038d511f0020f0cbf0024042404f077
:1037f00053fd214604f0e2fe14f00805074626d1e9
:1038000006b34ff0ff08294642463046b8f085fe21
:10381000124b134904a8cde90436cde90685fff71c
:1038200017fe3b460c210f4a01a8cde9015503952f
:10383000b9f0aafe01a904a8fff70afe0a4904a8e4
:10384000fff706fe630702d44620fff709ff38465c
:1038500008b0bde8f0810824c9e700bf40370d0279
:103860002e370d0282440d0234370d0230b5044666
:10387000002585b0039104f00ffd62682369039968
:10388000d31a0095228904f0d9fe05b030bd00009e
:1038900070b5324e044696f82c3086b0002b49d0d5
:1038a000706a2bf064ff0546002843d12c4b1c2086
:1038b00005932c4b0294049322f056f904460028f9
:1038c00031d0294bc5600360049b3bb1022202a9a1
:1038d00004309847059b2361049be3600025204644
:1038e000224b2a462360012140f8145f2cf048f84f
:1038f0001f4b01a92360f2692b46306b01942bf01a
:1039000094ff014650b9706a08b12bf05dff0022a8
:103910004ff0ff3160692cf043f8a5692368204619
:103920009b68984700e0054602a8fff799fa2846e9
:1039300006b070bd04f0b0fc037d63b90d4b1b787d
:1039400003f0ff05002bf2d00b4b1b78002b0cbfb4
:1039500001250225ebe70325e9e700bf9ccd001018
:10396000fd380002bd33000254360d0268360d02e8
:103970007c360d0260cc00104d5100100068fff73e
:1039800087bfc1684a69506803681b681847000010
:1039900038b50c461546c8683ab11146b9f03efd37
:1039a00038b1e0600020256138bdb8f069fde56000
:1039b000f8e70148f8e700bffcfeffff10b591f8fb
:1039c00043300c46db0748680cd500210bf0d6fdd0
:1039d00094f8433023f0010384f843300023c4e912
:1039e000013310bdb8f04cfdf8e708b508b109f097
:1039f00013f9002301211a46184603f0bafbbde86b
:103a0000084001f0fdb810b5c468a068b8f030fdfa
:103a1000606018f01ff894f842202ab963687bb1ff
:103a2000022384f84230144618f018f86cb160682c
:103a3000b8f026fd2046bde8104000210bf09ebde9
:103a4000012284f842201c46eee710bd136810b531
:103a5000032b17d90b685c1c0c6018700b685c1c7e
:103a60000c60040a1c700b685c1c0c60040c1c705d
:103a70000b68000e5c1c0c60187001201368043b7e
:103a8000136010bd0020fce773b58b6804460d463b
:103a900000931bb90026304602b070bdcb88006889
:103aa000694601aa0193fff7d1ff06460028f1d02d
:103ab000019b012beed9009aa389511c0091137030
:103ac000009a1b0a511c00911370019b2268023b53
:103ad000910701930ed5012bdcd9009ae389511c83
:103ae00000911370009a1b0a511c00911370019be6
:103af000023b019323685a070ed423681b0706d59f
:103b00006946606801aafff7a1ff0028c2d0aa6831
:103b1000009b9b1aeb80bee76946a06801aafff7ed
:103b200095ff0028e9d1b5e738b50c4b416003603b
:103b30000023c0e902330361044617f08bff0546fa
:103b4000214607482af052fc214606482af05afc32
:103b5000284617f083ff204638bd00bf94370d027a
:103b60004f3f0002713f00022de9ff41cb8806461e
:103b70003f2b0f4640f29380886860b1338a032b55
:103b80000cd9002301220293cde9002303230393e0
:103b90006846fff779ff04b0bde8f08100214420ba
:103ba0000bf0dafc044638b90123cde900300423d8
:103bb000029003933946ebe718230380bb884ff04c
:103bc000000843807b88c0e9038883606ff063034b
:103bd000c0e90c8846614062c0f83880c363738acc
:103be00001339bb273828568a0f8403080f843802f
:103bf000002d35d12b4b00f11801c3612a4803f089
:103c00005dfe032384f8423063886560462b0ed046
:103c100010d8322b07d004d8283b012b03d900251c
:103c200008e03c2bfbd10120fff7dffef7e7284639
:103c3000fff7dbfe0023a362b368e36203b19c627b
:103c4000338ab460013333820023cde90133b4f801
:103c50004030adf80c50adf80e3003230093a9e7c7
:103c6000402d0fd8414628460bf076fc606048b1e5
:103c700094f8433043f0010384f84330022384f87e
:103c80004230cce7094b0848e36104f1180103f026
:103c900015fe00230225636084f84230cae7002045
:103ca00079e700bf033900023cd9001087390002d0
:103cb00070b58b8884685cb1b4f840209a4209d012
:103cc000e46af8e7d8b9636833448b60012070bdbb
:103cd0000020fce794f84230022bf9d1cd88a66b86
:103ce000a36872199a42f3d8402d8868ead8002850
:103cf000edd0636801462a469819b8f0e7fba26b3d
:103d0000a36815449d42a563e0d1064b0648e361d4
:103d100004f1180103f0d2fd0023a363032384f808
:103d20004230d3e7033900023cd90010f8b506460b
:103d30008b8884684cb1b4f840209a4207d0e46a7a
:103d4000f8e7e3683b448b6016e0002019e094f844
:103d50004230042bf9d1cd88002df6d0a76b236912
:103d60007a199a42f1d8402debd8886848b1e168b9
:103d70002a463944b8f0aafba06b2844a06301206e
:103d8000f460f8bdf0b54b780c46502b85b00cd1e3
:103d900091f90030002b41dacb8833b1886888b3c1
:103da0008a88142a03d01e2a2ed000202ae010214f
:103db000684621f081fb1028f7d8e3884500b3eb73
:103dc000400ff2d36b46a2685619b24218d01f4674
:103dd00019780232090901f13000392888bf01f150
:103de000370002f8020c3978013301f00f0101f1bc
:103df0003000392888bf01f1370002f8010ce4e7f0
:103e0000e580012005b0f0bd042bced90b4b1a681c
:103e10001b79026003710523cb80f2e78b88282b86
:103e200006d0b3f5977fc0d10120fff7defde8e7ac
:103e300000228c20114617f065ffe2e783370d0260
:103e400010b5cb6a0c460bb18a6a9a62d4e90a2390
:103e500062b1d362038a013b038294f842300bb112
:103e6000032b05d1042384f8423010bd8360f1e7b1
:103e7000606840b194f84330db070dd500210bf0aa
:103e80007dfb00236360e36833b9216b21b92046d1
:103e9000bde810400bf072bb044b04f11801e36164
:103ea0000348bde8104003f009bd00bf31400002e7
:103eb0003cd900101fb5cb880c463f2b38d98b68f6
:103ec000002b37d08b88816829b1b1f840209a4205
:103ed00001d0c96af8e700230122cde90233cde918
:103ee000002319b391f84230042b0dd8dfe803f01a
:103ef00003070c0312000223adf80c3004e0042386
:103f0000adf80c30fff79cff21466846fff7bcfd7b
:103f100004b010bdcb6b0193092300930b691bb157
:103f200002930d230093efe7c160ede70523e3e77c
:103f30000020ede71846ebe77fb5cb8804463f2b22
:103f40000d4615d98868a0b18b884bb96ff08b06e8
:103f5000a368e3b1de632046a168fff771fff7e7ce
:103f6000a16841b1b1f840209a420ad0c96af8e785
:103f7000002004b070bd01230291cde9003105237a
:103f80000ae06ff08b032046cb63fff759ff002355
:103f90000122cde900230293294668460393fff7e7
:103fa00073fde6e74b78013b042b0ed8dfe803f006
:103fb000030507090b00fff7d7bdfff77bbffff72e
:103fc00077befff7b3befff7b7bf0020704708b555
:103fd00003465a780846013a0e2a194605d8fff7d3
:103fe000e1ff80f00100c0b208bdfff7cbfef8e7ab
:103ff000012838b50c460bd0022815d16ff0950575
:10400000a3689bb1dd632046a168fff719fff7e7be
:10401000c96849b18a6b0b699a4205d100252046cf
:10402000cd63fff70dffe560002038bde360fbe7df
:1040300038b54b6805460c4613b103685b68984772
:10404000e3682bb12b680022214628461b6898475d
:10405000236b13b1616be06b98472046bde8384095
:1040600000210bf08bba2de9f0411f464b68054645
:104070000c461646ddf8188013b103685b68984754
:10408000c4e90c7817f0e6fc94f84230032b01bf2a
:104090000423e66384f84230002417f0dffc2cb1df
:1040a00021462846bde8f041fff7c2bfbde8f081d8
:1040b000c1684869fff7bcbf03681b681847000068
:1040c00007b50022044bcde900021146104605f069
:1040d00001f803b05df804fb3940000208b54ff465
:1040e0007a7022f076fcbde80840002010f00ebb8c
:1040f00008b54ff47a7022f06cfcbde8084010f06f
:104100001dbb10b5c36804460bb9b7f05ffc03696b
:104110000430984723682046bde810409b68184744
:1041200008b54ff47a7022f054fcbde80840002036
:1041300010f007bb08b54ff47a7022f04afcbde8d6
:104140000840002010f0ccba37b5446925680093c8
:10415000ad6813460a4601462046a84703b030bd65
:10416000012a38b5044602d10b68236003e0022a15
:1041700003d0032a0dd0002038bd0c200d6821f09b
:10418000f3fc03460028f0d095e8070083e8070019
:10419000ebe700680028eed00c2121f0edfceae707
:1041a000012a034602d1016000207047022a04bfa1
:1041b000d1e90001c3e90001f6e7000010b50446ab
:1041c000034b40f8043bfef74bfe204610bd00bffa
:1041d000c8370d0210b50446fff7f0ff2046142142
:1041e00021f0cafc204610bd10b50446024b036006
:1041f000fff7e4ff204610bddc370d0210b5044682
:10420000fff7f2ff2046142121f0b6fc204610bd36
:1042100010b50446074b214640f8043bfff784fce9
:10422000214604f118000cf089f800232046c4f858
:10423000f43010bdf0370d0210b5044608f018fd3b
:10424000042805d104f11800bde810400cf058ba5c
:10425000092017f099fe0028f4d0002010bd183076
:104260000df05cba0048704770cc0010024bc3f8e8
:10427000f4000020704700bf70cc001010b44369f8
:104280000a4619680c680146184623465df8044b37
:1042900018470146406903685b681847fff754bf39
:1042a000f0b5354e074696f82c300d46144687b0cb
:1042b000002b51d0706a2bf05afa00284cd1049090
:1042c0000c2021f051fc10b1c0e9015407702b4bb8
:1042d000029005932a4b1c20049321f045fc0446d0
:1042e000002832d0274b03600023c360049b3bb1fe
:1042f000022202a904309847059b2361049be360d6
:1043000000252046204b2a462360012140f8145ff7
:104310002bf036fb1d4b01a92360f2692b46306b55
:1043200001942bf082fa014650b9706a08b12bf063
:104330004bfa00224ff0ff3160692bf031fba56989
:10434000236820469b68984700e0054602a8fef7d0
:1043500087fd284607b0f0bd0d4c84f8fc70d4f8fa
:10436000f80028b18368c4f8f830b8f089f8f6e7a7
:10437000c4f8f8500546ece79ccd00101543000248
:10438000e140000254360d0268360d027c360d0203
:1043900070cc001003681878d3e90112fff780bfd2
:1043a00073b5064614200d4621f0defb0446d0b15d
:1043b0000e4b03600023c360ab683bb10222294669
:1043c00004309847eb682361ab68e360084b3046e4
:1043d0002360336801945b6801a9984718b9236882
:1043e00020469b68984702b070bd00bfc8370d02d9
:1043f000dc370d027fb5144e044696f82c300d467e
:1044000093b1706a2bf0b3f970b9104b69460393fe
:104410000f4b30460293cde90054fff7c1ff6846c9
:10442000fef71efd04b070bdd4f8f43023b90a20a5
:10443000084a0949fcf7d4fd2846d4f8f43004b002
:10444000bde87040184700bf8cd400108d480002b2
:104450002141000257690202a0370d02f0b50c4657
:10446000d0f8f83085b0002b00f04c829988628833
:10447000914200f02f829b68f5e76388e72b00f2fa
:10448000d980db2b26d85a2b00f2ad80452b3fd8a4
:10449000292b00f29f80132b6ad8012b00f070812a
:1044a000d0f8f430002b00f07581214605b0bde84e
:1044b000f040fff79fbf6ff4fa7213442046052bbc
:1044c00000f2df81dfe813f0e001e301e601e9013a
:1044d000ec01ef01dc3b0b2be2d801a252f823f0f8
:1044e0008f470002974700029f470002a74700023c
:1044f0002144000221440002214400022144000220
:104500002144000221440002af470002b7470002e5
:10451000463b142bc4d801a252f823f0c546000232
:10452000d1460002e1460002e9460002f1460002df
:10453000f946000221440002214400022144000205
:1045400021440002214400022144000221440002cf
:1045500021440002214400022144000221440002bf
:1045600021440002214400022144000209470002c4
:10457000143b152b94d801a252f823f07346000285
:10458000814600022144000221440002214400022d
:10459000214400022144000221440002214400027f
:1045a0002144000289460002914600029946000219
:1045b000a1460002a9460002214400022144000253
:1045c000214400022144000221440002b1460002bd
:1045d000b9460002322b00f0b2803c2b7ff460af72
:1045e0000023c34aa6e0642b00f0d280c83b9ab2f5
:1045f0000b2a3ff655af0b2b3ff652af01a252f8f4
:1046000023f000bf6f4700027747000221440002f9
:1046100021440002214400022144000221440002fe
:104620002144000221440002214400027f4700028d
:1046300087470002b3f5fd7f4bd8b3f5fa7fbff48f
:104640003aafb3f5967f00f0108127d8f03b9ab2cd
:104650000d2a3ff625af0d2b3ff622af01a252f8ef
:1046600023f000bfbf4700022144000221440002a2
:10467000214400022144000221440002214400029e
:10468000214400022144000221440002c7470002e5
:10469000cf470002db470002e3470002b3f5c87fc3
:1046a00000f0eb800cd840f22d12934200f0e18034
:1046b000b3f5977f7ff4f4ae20460df0cafc1be003
:1046c00040f2911293427ff4ebae20460df060fa77
:1046d00012e0a3f226239ab2042a3ff6e1ae042b9d
:1046e0003ff6deaedfe813f0e200e600ea00ee009f
:1046f000f20020460df014fd002301461a46f1e0b9
:1047000020460df047fdf7e720460df05bfdf3e78f
:1047100020460df06dfdefe720460df0bffdebe705
:1047200020460df04ffee7e720460df069fee3e777
:104730000023704a1946d5e000236f4afae70023a8
:104740006e4af7e700221146104602f0b9fed3e7a1
:1047500000220121104602f011ff00231a46e9e76a
:1047600020460df0e1fdc7e720460df0effdc3e761
:1047700020460df0fffdbfe720460df009febbe728
:1047800020460df063feb7e720460ef019fdb3e7b3
:10479000a36823b100236ff077011a46a2e08026b8
:1047a000574f60693246036821461b6898470546a3
:1047b00040b1002211462046fff760fd0023294644
:1047c0001a468fe0e368014603906846cde900731e
:1047d0000296fff775fc002205460028ead1039bec
:1047e0009e4202d203eb1316dbe72361e6e7204685
:1047f0000df062fd80e720460df074fd7ce7204659
:104800000df033fe78e720460df032fe74e72046c7
:104810000df031fe70e720460df030fe6ce72046cb
:104820000df02ffe68e720460df02efe64e72046cf
:104830000df06afd60e720460df06efd5ce7204656
:104840000df025fe58e720460ef0d2fb54e7204637
:1048500005b0bde8f0400ef045bc20460ef072fcfd
:104860004ae720460ef074fc46e720460df0bcfbfc
:1048700042e720460df0e8fb3ee720460df068f9e0
:104880003ae70ef023f837e70df0e6fe34e70df0d7
:104890004dff31e70df080ff2ee70df0a1ff2be774
:1048a0000df0aaff28e70ef07bf925e720460df072
:1048b00043fa21e720460df0b9fa1de720460df036
:1048c00011fb19e720460df029fb15e720460df0f6
:1048d00043fb11e79b79022b7ff4cfad00236ff0f0
:1048e00081011a46204605b0bde8f040fff72cbc18
:1048f000a140000271400002b54000025d4000028c
:1049000040370d0290f8fc30e5e700bfd0e9001019
:10491000fff770bd0148fff77bbc00bf70cc0010f3
:104920000023202200b58bb0cde90223054a0120e7
:104930000092054902aafdf78bfb4ff0ff300bb048
:104940005df804fbfb370d02f4370d02f0b50024cf
:1049500020274ff4837605460e4bc5b0009302aa7c
:1049600023461e200c49cde90274fdf771fb324647
:10497000214602a8b7f0d1fd3a4621462846b7f0b5
:10498000ccfd23462246314602a805f0f3fa45b095
:10499000f0bd00bf57380d02f4370d022de9f0418c
:1049a000ceb04ff4837204460e460ca80021b7f037
:1049b000b4fd00234ff483711a460ca805f0fcfaed
:1049c000b0f5837f2dd1bdf83030b3f5837f28d18a
:1049d00080213046149d17f033fa854234d00025eb
:1049e000202780213046ddf85080cde9047517f08e
:1049f00027fa214bcde90180009304aa2b463220ef
:104a00001e49fdf725fb9df83530322001931c4be4
:104a10001a49009304aa2b46cde90475fdf718fb4b
:104a20000ae020210023174acde904130092282030
:104a3000124904aafdf70cfb2046fff787ff4ff051
:104a4000ff304eb0bde8f0819df83530002bc6d068
:104a50000dad0fcd0fc495e80700002384e80700d3
:104a60002022cde90423084a1e200092034904aa0b
:104a7000fdf7eefae3e700bfa3380d02f4370d02ad
:104a8000c8380d026f380d02db380d0210b5044630
:104a90000846802117f0d4f9e061002010bd000025
:104aa00030b50020b1b003f05ffb032017f06cfac3
:104ab0000446002837d0444b1d888022002110a8ce
:104ac000b7f02bfd10a825f04bfe9df84030012bd0
:104ad00016d920220023cde908233c4a2820009241
:104ae0003b4908aafdf7b4fa2cb13a4b3a491a6887
:104af00010a8b7f0ebfc394a136843f004031360c5
:104b00009df8402020218ab1012a4ff000034cd0ab
:104b10000192334acde90813009228202c4908aab3
:104b2000fdf796fa1fe041f23365c6e7ddf8423043
:104b3000cde90812bdf882101e200791d9b2069166
:104b4000c3f307210591c3f307411b0e03930df136
:104b50004203cde90123234b049100931c491346e2
:104b600008aafdf775fa4ff6fd71bdf88220531eb5
:104b70009bb28b4202d81cb1aa4201d0adf8825040
:104b800010a91948fff70aff002c14bf11200620b6
:104b9000154a10a903f06af8044618b9124810a97a
:104ba000fff774ff204631b030bdcde908130df199
:104bb0004201cde901210d4a1e200092044908aab4
:104bc000fdf746facfe700bf6051001012390d0221
:104bd000f4370d02982f0d027f2f0d0258d30010cd
:104be000a8390d023e390d0274cd001080390d0236
:104bf00003f0baba08b5002003f0f8fac0b208bd55
:104c00000122014b1a70704770cd001013b50f4b85
:104c100004461b7823b102b0bde81040fff780be08
:104c20000b4b01911b78002bf5d1fff7e3ff002818
:104c3000f1d1084b1b7803f0ff02002bebd120468b
:104c4000019902b0bde8104003f02aba11d100105a
:104c500012d1001070cd0010fff7d8bf13b50f4b65
:104c600004461b7823b102b0bde81040fff758bee0
:104c70000b4b01911b78002bf5d1fff7bbff0028f0
:104c8000f1d1084b1b7803f0ff02002bebd120463b
:104c9000019902b0bde8104003f02eba11d1001006
:104ca00012d1001070cd0010fff7d8bf08b500205a
:104cb00003f086fa10f1780f08bf002008bd00202d
:104cc00003f090baf0b5022806460d4614468db0a2
:104cd00005d00a2834d01f4c20460db0f0bd20204e
:104ce00000231d4fcde904033a68cde901211b4a99
:104cf000009201201a4904aafdf7aaf93d6000f0cc
:104d0000a7fd10b914f00104e6d0164b00245b781f
:104d1000b342e1d12023cde90434134b04aa00931c
:104d2000012023460e49fdf793f908220223294664
:104d3000cde904232046234604aa00f07ffecbe7fa
:104d400020210023094fcde904133a68cde901255c
:104d5000074acde7f2feffff58510010e4390d027b
:104d6000f4370d0274cd0010473a0d025c5100106b
:104d7000153a0d0219b1022803d00a2806d00448ba
:104d80007047044b1b6800200b607047024bf9e72b
:104d9000f2feffff585100105c51001003689b6841
:104da00018470eb403b503ab53f8042b002101934d
:104db0000ff039fb02b05df804eb03b070472de94a
:104dc000f04106460d46904624f0b3fd074624f018
:104dd000b0fdc01b40450ed83468236820461b69cf
:104de00098470028f3d0236820465b6998472870cd
:104df0000020bde8f0814ff0ff30fae72de9f04fd9
:104e000016461a46002385b00f4633600df10f0198
:104e100001928246fff7d3ff019a044628b14ff072
:104e2000ff34204605b0bde8f08f9df80f50182dd7
:104e300013d008d8022d20d0042df2d0012deed1b0
:104e40004ff080081be005f0df03412b35d0202d0b
:104e500014bf4ff0ff340224e3e750460df10f0179
:104e6000fff7adff04460028d9d19df80f30182b6d
:104e7000d5d14ff0ff333360d3e74ff48068b946a4
:104e800009f8015b012508f1040b5d450cd8494682
:104e900050460192fff793ff09f101090028bed1a6
:104ea0000135019aadb2f0e7bb787a78db43dbb22b
:104eb0009a42b4d1c6f80080b3e70124b1e738b50f
:104ec0000d46002102f58070033313f8014b2cb11d
:104ed000b1f5807f02d054540131f6e700245454d8
:104ee000ff32195d202905d0102c03d0013402f8bf
:104ef000011ff6e700210a220155b9f0c1fa4ff46b
:104f00008063e8602b8138bdf8b51d46531c04460c
:104f10000cd08ab1d0f818644f78f3b29f4213d006
:104f200000681521fff73aff012004e00068062120
:104f3000fff734ff0020f8bd00680621fff72effc1
:104f40000120c4f81404f6e786bbcb7803b30b4604
:104f5000069a2946fff7b3ff324631462846fef748
:104f600013fc50b118212068fff718ff20681821a2
:104f7000fff714ff4ff0ff30dde72b6906216b6070
:104f80002068fff70bff43212068fff707ff04e0cd
:104f90000123c0f81434c0f810340120d4f81834b8
:104fa000c4f820040133c4f81834c4e72a81284621
:104fb00000220331fef75afc50b118212068fff798
:104fc000edfe20681821fff7e9fe6ff00100b2e75f
:104fd0006b682a89062113446b60d5e72de9ff41f0
:104fe0001746044600250e464ff4887200213846c5
:104ff000b7f093fa04f10808c4f81054c4f81c542c
:10500000c4f82054c4f81854c4f814544146204637
:10501000636803aafff7f2fe012810d0022819d016
:1050200030bbc4f81c04334641462046039a00971f
:10503000fff76aff002811dc04b0bde8f0811821f9
:105040002068fff7abfe20681821fff7a7fe6ff07e
:105050000200f1e706212068fff7a0fed4f814341f
:10506000002bd3d0d4f81034002bcbd0f068e3e77a
:10507000d4f82034002b08dbd4f81c34432101334e
:105080002068c4f81c34fff789fed4f81c34052bc3
:10509000e4dd18212068fff781fe20681821fff762
:1050a0007dfe0020c8e70000f0b50446c7b040f21e
:1050b00024400f4620f058fd054618b141f28833d0
:1050c000046043603946284602aafff787ff061ea0
:1050d00048dd002201213846fef77efb021e31db4f
:1050e00006212868fff75afe20462a490ff09cf84f
:1050f000204629490ff085f8204602a90ff081f8d3
:10510000204626490ff090f8204625490ff079f8ff
:105110000a22314620460ff091f8224920460ff02e
:1051200083f823682046db6998474ff47a7021f0b2
:1051300050fc0124284640f2244120f01dfd204669
:1051400047b0f0bd182128680192fff727fe18210b
:105150002868fff723fe2046019a1349fff721fe36
:105160000024e7e718212868fff718fe18212868af
:10517000fff714fe721c04d10c4920460ff054f8be
:10518000eee7b31c01d10a49f7e703360cbf094922
:105190000949f2e76b3a0d028b3a0d02af2c0e0271
:1051a000923a0d022e630d02993a0d02b13a0d02a8
:1051b000e83a0d02fe3a0d020f3b0d0201200af003
:1051c0002bb908b50023c269006b2af02efbb0fa98
:1051d00080f0400908bd70b505460e468069002183
:1051e0002af0eefa002304461a463146286b2af0cc
:1051f0003dfb18b1201e18bf012070bd0120fce747
:1052000008b500238269006b2af030fbb0fa80f009
:10521000400908bd38b50546fff7d3ff044620b165
:10522000686a10b100212af0cffa204638bd012a61
:1052300002d1016000207047022a04bf0b6803609e
:10524000f8e7036818470000014b18682af04dbbc7
:10525000e4cd001010b5044c236813b920462af0a1
:1052600060fb206810bd00bfd0cd001010b50a4c07
:10527000d4e88f3fdb070cd4204622f089fd40b1f3
:1052800006482af028fb204622f0bcfd0448b6f070
:10529000f6fe024810bd00bf98cd0010e4cd00100e
:1052a000c9510002014b1860704700bf94cd001037
:1052b00038b5002383608b6804460d462bb102226b
:1052c0009847eb68e360ab68a360204638bd0000f8
:1052d00030b5214b8db00093204b69460393204b92
:1052e00004a80293fff7e4ff4ff4a0526423cde932
:1052f00008236ff000430a9332231a4cadf82c3088
:105300000223204600258df82e30174b04a940f8c3
:10531000043bfff7cdff089b04f128006361099b64
:105320006562a3610a9be361bdf82c3023849df87c
:105330002e3084f822302af0cefa0c4b04a82360d9
:1053400084f82c502563fdf78bfd6846fdf788fd3a
:10535000074b9d600db030bd3d510002c3510002ae
:10536000af5100029ccd0010343b0d02443b0d02b6
:10537000d4cd001010b5c36804460bb9b6f026fbb7
:105380000369043098470021a0616069bde81040be
:105390002af026bb10b5c36804460bb9b6f016fb5d
:1053a000036904309847002120766069bde8104009
:1053b0002af016bb08b505f0fdfa002008bd000074
:1053c00007b51346002200920a46014605480068c8
:1053d00010f07ff8002818bf6ff0ef0003b05df801
:1053e00004fb00bf60d30010012a70b5054603d14d
:1053f0000b680360002070bd022a08d0032af9d18f
:1054000000680028f6d0102120f0b6fbf2e710204b
:105410000e6820f0a9fb044618b196e80f0084e856
:105420000f002c60e6e7012a70b5054603d10b6832
:105430000360002070bd022a08d0032af9d1006859
:105440000028f6d0102120f097fbf2e710200e681c
:1054500020f08afb044618b196e80f0084e80f009c
:105460002c60e6e7012a08bf016000207047012a8e
:1054700038b5044602d10b68236003e0022a03d04a
:10548000032a0dd0002038bd0c200d6820f06cfbe5
:1054900003460028f0d095e8070083e80700ebe713
:1054a00000680028eed00c2120f066fbeae7012a14
:1054b00070b5054603d10b680360002070bd022a59
:1054c00008d0032af9d100680028f6d0102120f076
:1054d00053fbf2e710200e6820f046fb044618b19b
:1054e00096e80f0084e80f002c60e6e7012af8b583
:1054f000064603d10b6803600020f8bd022a08d0dd
:10550000032af9d100680028f6d0142120f034fbda
:10551000f2e714200c6820f027fb074620b105466f
:105520000fcc0fc523682b603760e5e7012af8b57b
:10553000064603d10b6803600020f8bd022a08d09c
:10554000032af9d100680028f6d0142120f014fbba
:10555000f2e714200c6820f007fb074620b105464f
:105560000fcc0fc523682b603760e5e7012a03469f
:1055700002d1016000207047022a04bfd1e9000176
:10558000c3e90001f6e7012a02d10160002070475b
:10559000022a04bf0b680360f8e7012a08bf016014
:1055a00000207047012a02d1016000207047022ac2
:1055b00004bf0b680360f8e7012af8b5064603d17b
:1055c0000b6803600020f8bd022a08d0032af9d135
:1055d00000680028f6d0182120f0cefaf2e7182053
:1055e0000c6820f0c1fa074630b105460fcc0fc554
:1055f00094e8030085e803003760e3e7012a0346e7
:1056000002d1016000207047022a04bfd1e90001e5
:10561000c3e90001f6e700224ff0ff312af0c0b9dc
:1056200000224ff0ff312af0bbb9000010b504464c
:10563000034b40f8043bfdf713fc204610bd00bfb0
:10564000543b0d0210b50446fff7f0ff204614212d
:1056500020f092fa204610bd10b5074b04460360b7
:10566000406918b12af097f9002363612046fff7db
:10567000ddff204610bd00bf683b0d0210b504469b
:10568000fff7eaff2046182120f076fa204610bde9
:1056900010b50446024b0360fff7deff204610bd45
:1056a0007c3b0d0210b50446fff7f2ff20461c219b
:1056b00020f062fa204610bd10b50446034b40f8b6
:1056c000043bfdf7cdfb204610bd00bf903b0d0213
:1056d00010b50446fff7f0ff2046142120f04cfae5
:1056e000204610bd10b5074b04460360406918b151
:1056f0002af051f9002363612046fff7ddff2046c1
:1057000010bd00bfa43b0d0210b50446fff7eaff31
:105710002046182120f030fa204610bd10b504466e
:10572000024b0360fff7deff204610bdb83b0d02c1
:1057300010b50446fff7f2ff20461c2120f01cfaaa
:10574000204610bd406a2af012b8000010b404468a
:105750000748134600682ab1214600235df8044b30
:105760000ff09cbd0a4621465df8044b0ff09dbd2d
:1057700060d30010f0b52e4e044696f82c300d463e
:1057800087b0002b4ad03046fff7dcff07460028e1
:1057900044d1284b1c200593274bcde902450493a7
:1057a00020f0e2f90446002831d0244bc7600360a2
:1057b000049b3bb1022202a904309847059b236158
:1057c000049be360002520461d4b2a4623600121ef
:1057d00040f8145f2af0d4f81a4b01a92360f2694b
:1057e0002b46306b01942af020f8014650b9706abc
:1057f00008b129f0e9ff00224ff0ff3160692af07b
:10580000cff8a569236820469b68984700e00546c5
:1058100002a8fdf725fb284607b0f0bd05f036f9d4
:105820002a46214607b0bde8f0400ff086be00bf13
:105830009ccd0010c9570002ed540002903b0d02b0
:10584000a43b0d02b83b0d02d0e90001fff792bf67
:10585000054b1b7803f0ff0023b1044b1878003888
:1058600018bf0120704700bf5ecc00105bcc001059
:1058700008b50948fff766ff68b1002007f004fa91
:1058800020b1bde80840044801f0ecbf0120bde8ac
:10589000084009f0c1bd08bd8cd40010002190b5ae
:1058a00083b0044600af08461ff006fec31d23f078
:1058b0000703adeb030d0146786068461ff0fcfd61
:1058c00020467a68694605f05ffe20460c37bd46e3
:1058d00090bd0000014b1860002070475cd30010a1
:1058e0007fb51d4d044695f82c300e46b3b12846c1
:1058f000fff728ff90b9194b69460393184b2846c8
:10590000cde900460293fdf7affb044688b9054692
:105910006846fdf7a5fa284604b070bd94b1631c33
:1059200013d021460f4802f05bf90e4802f045f90a
:105930000be04069fff774fe236820469b68a56969
:105940009847e5e7074802f033f9064804b0bde898
:10595000704002f089b900bf9ccd0010e9580002e8
:105960007d550002e8cd0010d0e90001fff7b8bf77
:105970002de9ff41014640b368460ef0b3f8009ea2
:105980009df80940ddf804809df80850fff760ff9e
:1059900000b305f025fe4ff00103d0e8cf7fc0e84b
:1059a000423f002af9d1ffb2002ff6d1c660c0f8fd
:1059b0001080057544750023c0e88f3f07f02cf96f
:1059c0000024204604b0bde8f08105468046044628
:1059d0000646dbe707f020f916f0040625d0002c78
:1059e000efd0134c94f82c3013b904f0e3ffe7e741
:1059f0002046fff7a7fe0028f7d10e4b6946039318
:105a00000d4b20460293fdf72ffb054658b1406928
:105a1000fff706fe2b6828469b68ac6998476846e6
:105a2000fdf71efacde70446f9e73446c9e700bfa3
:105a30009ccd001035530002e5530002f0b504463a
:105a40002c481f4690f82c300e46154687b0dbb127
:105a5000fff778fec0b90490102020f085f818b147
:105a6000c0e90046c0e90257234b02900593234b3f
:105a7000204802a90493fdf7f7fa044660b90546e9
:105a800002a8fdf7edf904e0012c25d9022c0cd079
:105a90001b4d284607b0f0bd4069fff7c1fd2368e4
:105aa00020469b68a5699847eae7294602a80ef0b8
:105ab00019f805f095fd029b0025d90744bf9df814
:105ac000102002729a0744bf039a42605b0744bfea
:105ad0009df811304372dce70a4800972b463246a6
:105ae000214600680ff0bffc07b0bde8f0400ff0a2
:105af000f1ba00bf9ccd0010895a0002a7530002e2
:105b0000f2feffff60d300100068d0e90223d0e965
:105b10000001fff793bf000030b5044628481d463a
:105b200090f82c3087b00bb3cde90012fff70afed6
:105b3000dde90012d0b90490102020f015f828b14a
:105b4000019a0099c0e90225046041601d4b029052
:105b500005931d4b1a4802a90493fdf785fa0446e4
:105b600070b9054602a8fdf77bf906e0042c19d0b0
:105b7000052c1cd0032c0cd0144d284607b030bd8a
:105b80004069fff74dfd236820469b68a56998474b
:105b9000e8e70f4b1b787bb1082007b0bde8304029
:105ba000fff70ebc0a4b1b7833b10920f5e7084b11
:105bb0001b780bb10a20f0e76ff0d105dde700bfdd
:105bc0009ccd0010555b000269530002f2fefffffe
:105bd0005bcc00100068d0e90223d0e90001fff798
:105be0009bbf000073b506461c200d461ff0bcff8e
:105bf000044628b3144b03600023c360ab683bb179
:105c00000222294604309847eb682361ab68e360c1
:105c1000002220460d4b0121236040f8142f29f06b
:105c2000affe0b4b30462360336801945b6801a9db
:105c30009847054620b9236820469b6898472c461c
:105c4000204602b070bd00bf543b0d02683b0d0200
:105c50007c3b0d022de9f04305462e48994690f80d
:105c60002c3087b00e4690460e9f2bb3fff76afd8f
:105c700010bb049018201ff077ff40b10f9bc0e9c4
:105c80000056c0f8088080f80c9007614361224bf1
:105c900002900593214b1f4802a90493fff7a2ff2e
:105ca000054670bb044602a804f00104fdf7d8f8cd
:105cb000204607b0bde8f083b9f1000918bf4ff0e6
:105cc0000109cde9007816484b463246294600685e
:105cd0000ff0f2fa04460028ead0fff7b9fd0646b5
:105ce0000028e5d006f0c4ff012803d10d4b1b7836
:105cf000002bddd03a4649462846fff727fd3446bb
:105d0000d6e74069fff787fc2b6828469b682c7e06
:105d10009847c8e79ccd0010a95c000239550002e5
:105d200060d300100cd5001007b500684269037bf2
:105d3000019202690092d0e901120068fff78aff20
:105d400003b05df804fb000030b5174c054694f82d
:105d50002c3085b003b32046fff7f4fce0b9134bb9
:105d600020460393124b694600950293fff73affd2
:105d7000044678b14069fff74efc236820469b68d3
:105d8000257e9847684605f00105fdf769f8284625
:105d900005b030bd0546f5e704f078fe002105b0fa
:105da000bde830400ff0c6bb9ccd0010355d000251
:105db000075500020068fff7c7bf0000f0b50446b2
:105dc00022481f4690f82c300d46164685b0fbb190
:105dd000fff7b8fce0b9029010201ff0c5fe18b123
:105de000c0e900450672c760194b00900393194b38
:105df000694616480293fff7f5fe054658b9044672
:105e0000684604f00104fdf72bf8204605b0f0bd0c
:105e100055b9002415e04069fff7fdfb2b682846c3
:105e20009b682c7e9847ebe75cb12046faf7caffe7
:105e30004028eed820463b463246294604f04cfe28
:105e40000446003c18bf0124dfe700bf9ccd0010d2
:105e5000d95d00022f5400020068c368027ad0e9bd
:105e60000001fff7abbf00007fb5054622480c4696
:105e700090f82c301646f3b1fff764fcd8b90290c5
:105e80000c201ff071fe10b1c0e9005486601b4b5e
:105e9000009003931a4b694617480293fff7a2fe3e
:105ea000044680b90546684605f00105fcf7d8ffb1
:105eb000284604b070bd7db93146204604b0bde827
:105ec000704004f0c2bf4069fff7a5fb236820467d
:105ed0009b68257e9847e6e710230021adf8003047
:105ee000084b68460195cde90234adf8021004f084
:105ef000acff0546dce700bf9ccd0010895e0002c8
:105f0000ef53000289ac000203681868d3e901125c
:105f1000fff7aabf30b5114c054694f82c3085b078
:105f20008bb12046fff70efc68b90d4b6946039311
:105f30000c4b204602930095fef732fa6846fcf7b8
:105f40008fff05b030bd0022074b114618680ff0d7
:105f500078fa05b0bde8304004f09ebb9ccd00103f
:105f6000ed5e00022555000260d300100068fff7c7
:105f7000d1bf00001fb50e4c94f82c3083b12046e1
:105f8000fff7e0fb60b90b4b694603930a4b2046d1
:105f90000293fef705fa6846fcf762ff04b010bdf5
:105fa0000021064b186804b0bde810400ff01eba7f
:105fb0009ccd00104f5f00021b55000260d3001003
:105fc00008b5fff7d7ffbde80840fff741bcfff772
:105fd000d1bf00002de9f04705463d4886b013f0db
:105fe000100f1c460e461746ddf8389090f82c30fe
:105ff0000df1080822d003f0ff0a002b46d0fff76e
:10600000a1fb002842d1049014201ff0adfd28b15f
:10601000c0e90056c0e90274c0f810902d4b029000
:1060200005932d4b41462a480493fef7b9f94046a3
:10603000fcf716ff504606b0bde8f08733b3fff714
:1060400081fb18bb049014201ff08efd28b1c0e91d
:106050000056c0e90274c0f81090204b02900593de
:106060001f4b41461a480493fff7bcfd044658b144
:106070004069fff7d0fa236820469b6894f818a07f
:1060800098470af0010ad2e78246fae70023cde9f1
:1060900003330c230293b9f1000f05d0d9f8043073
:1060a0000393d9f80830049314f0010f14bf45226c
:1060b000652224f0010313430a480093cdf80480bd
:1060c0003b463246294600680ff08af88246b1e71f
:1060d0009ccd001069600002ad5400028360000294
:1060e0006d54000260d3001007b500680369009387
:1060f000d0e90223d0e90001fff76cff03b05df89f
:1061000004fb07b5006803690093d0e90223d0e9d6
:106110000001fff75fff03b05df804fb00210148b9
:1061200001f0e8bce8cd001030b5cc1c2a3114f8e1
:10613000035c033405f00f0205f0f00342ea02129b
:1061400043ea1515130243ea0543436014f8052c8e
:1061500002f0f00545ea12152b4302f00f024360ee
:10616000827214f8043ca14203eb830303eb830324
:106170004fea430320f8083fd9d130bd002138b59c
:1061800004460846fcf78cf81c2500232046094ce1
:1061900005fb0342416801331161817a0d2b517374
:1061a00030f8081f9182f3d10021bde8384001206a
:1061b000fcf776b8f8cd00100c2808b50ad81c22d8
:1061c000054b02fb0030002201730121fcf724f88b
:1061d000002008bd0120fce7f8cd001011f00402fa
:1061e00038b50cd000240b4d00222846114601344e
:1061f000fcf712f80d2c05f11c05f5d138bd0c2863
:10620000fcd81c24034b114604fb0030bde8384089
:10621000fcf702b8f8cd00100c289fbf1c22044bdd
:1062200002fb0030807b94bf00f00100002070472b
:10623000f8cd0010f0b58a0705460c469db01cd578
:1062400001256822002102a8b6f067f9214901a8ba
:106250000195fff769ff01a8fff790ffe30709d554
:10626000ff232a4640f6af618df803300df103009d
:1062700020f0d3fc00201db0f0bd0368012b27d116
:10628000fff77cff14f00100f5d001a90846322683
:106290002b4668355a68c2f30357c2f3033444ea05
:1062a00007144c709c7a02f0f00204f00f042243b1
:1062b0008a7033f8082fb2fbf6f29d4201f8032fe3
:1062c000e8d10123402240f6af618df80430cfe7da
:1062d0000120d0e7c43b0d0270b50268012a18d135
:1062e00011f0020105d00c49fff71eff00210846fe
:1062f00070bd0b461c26094d06fb03521469013381
:106300004460547b0d2b8472928a20f8082ff3d1bd
:10631000ede70121ebe700bfc43b0d02f8cd001013
:106320000c289dbf1c22024b02fb0030002070474e
:10633000f8cd0010022803d0032807d000207047b2
:10634000142909d00adc4ff4fa707047142907d0d9
:1063500009dc4ff4fa507047c8207047642070473a
:106360004ff47a6070474ff47a7070470021224ae8
:1063700030b50b4615461c24adb004fb015001316d
:106380000d29c2e900439360037302f11c024373b9
:10639000837303618382f0d16822002112a8b6f0d2
:1063a000bcf80123402240f6af6001a9119320f010
:1063b000fffb18b99df80430012b1ad00f4b01aa2e
:1063c00003f12005144618685968083303c4ab422a
:1063d0002246f7d1998818689b79a1802060a37123
:1063e00001a911a8fff7a0fe11a8fff7c7fe2db065
:1063f00030bd0df10501f4e7f8cd001004240d02c5
:106400002de9f04f4ff0180a91469b460e4615496c
:1064100085b0d1e9004103900afb014adde90e781d
:106420000c34a4f10c018a4511d054e90301039bfb
:106430003140184050ea010307d000945b464a46b9
:106440003146039854f8045ca8471834e9e72fb1a3
:1064500040463b4605b0bde8f04f184705b0bde8e3
:10646000f08f00bf64cf001030b5d1e90054d0e9ff
:1064700000232a40234013430cd0836813b18a6859
:10648000934207d1c3683bb158680b69c31a58429d
:10649000584130bd0020fce70120fae7704710b5f5
:1064a000044628211ff068fb204610bd012af8b5dc
:1064b000064603d10b6803600020f8bd022a08d00d
:1064c000032af9d100680028f6d018211ff054fbe8
:1064d000f2e718200c681ff047fb074630b105466d
:1064e0000fcc0fc594e8030085e803003760e3e7ad
:1064f0002de9f043dff8d88093b08146d8f800004a
:106500000e4615461c4629f01bfa15f0a3fa002387
:106510000746cde90096cde90333029505933cb1da
:10652000628821460c2a28bf0c2203a8b5f0ceffb2
:106530006d4606ac0fcd0fc495e803000cae0df10f
:10654000180c84e80300bce80f001f4d0fc694e848
:106550000300d5f80490ab6886e8030099451adb80
:1065600009f10104002c286810dd18216143b6f000
:1065700055ff70b9154c384615f070fad8f8000080
:1065800029f0edf9204613b0bde8f083b5f078ffaf
:1065900000202860ac6018236a6803fb09f95a439d
:1065a0002c68a2eb09024c442146e0180caeb5f071
:1065b0009aff0fce0fc496e803006b6884e80300cf
:1065c000013300246b60d6e764cf0010fcfeffffb0
:1065d00070cf00102de9f04f8fb00193574b8346d9
:1065e00018688946164629f0abf915f033fa1822d7
:1065f000534fcde902b9d7e90045019b55430496b5
:106600000deb020c05930df108090aae824699e8dc
:106610000f008ce80f0086e80f004a4b04eb0508da
:10662000ed105d43ad10002d1ddd21463046fff716
:106630001bff30bba346183421463046fff714ff3a
:10664000f8b90bf1300421463046fff70dffc0b911
:106650000bf1480421463046fff706ff88b90bf1dd
:106660006004013ddfe7a8eb0403302b27d0482b63
:106670001ed0182b4cd121463046fff7f5fe0028de
:1066800046d0a04545d004f11806b04541d031466a
:106690004846fff7e9fe48b92546b446bce80f0076
:1066a0000fc59ce8030085e8030018341836ece7b2
:1066b00021463046fff7d8fe0028e2d118342146a3
:1066c0003046fff7d1fe0028dbd11834d3e71d4850
:1066d000e31adb10151b00fb03f304d4ed10454354
:1066e0005819814200dacd1a182101fb05412046d4
:1066f000521ab5f0f8fe7b685b1b7b60504615f0c4
:10670000adf90e4b18680fb0bde8f04f29f027b96e
:10671000444618267a683b6806fb02339c42edd05b
:106720002546d7e9003106fb01329542cfd02869d2
:1067300010b16b6903b198471835f2e770cf0010bc
:1067400064cf0010abaaaaaa2de9f0471f461e4b42
:10675000164693f82c2086b00546dde90e890c46d6
:10676000eab1586a29f003f8c8b9049018201ff05c
:10677000fbf928b1c0e90054c0e90267c0e9048907
:10678000124b02900593124b02a90f480493fdf798
:1067900007fe02a8fcf764fb06b0bde8f087dff84f
:1067a00034a0daf8000029f0cbf828463b46324600
:1067b0002146cde90089fff723fedaf8000006b094
:1067c000bde8f04729f0cbb88cd400101d6800025a
:1067d0002d64000270cf00102de9f047dff860c093
:1067e0000746dde90898dcf804c00e46ccf3080c37
:1067f00015461c46bcf1000f16d00021282008f0d9
:10680000abfe0146a0b1002383600a4bc0e90476c9
:106810000360c0e90654c0e90898074b4360bde82f
:10682000f047064801f04ab8bde8f047fff78cbfd3
:10683000bde8f087f43b0d02f76700023cd9001079
:1068400000ed00e010b4039ce40703d55df8044bb1
:10685000fff7d6bd5df8044bfff7bebf002307b5b9
:10686000024600214ff48040cde90033fff7b4ff2a
:1068700003b05df804fb13b50446436a0193036a51
:106880000093d0e90623d0e90401fff75dff002162
:10689000204602b0bde8104008f070be07b50168a0
:1068a0004b6901930b690093d1e90223d1e90001ff
:1068b000fff74aff03b05df804fb00000023044a21
:1068c0000448c2e900339360036029f02ab800bf8e
:1068d00064cf001070cf0010002210b5114604469e
:1068e00000f0dafb024638b1002320461a4619466a
:1068f00000f094fd012010bd0146204600f01bfc75
:106900000028f8d0f0e7002373b506220093032196
:10691000012008f0adfb0320fff7deff0646042050
:10692000fff7daff05460520fff7d6ff00230446f0
:1069300026b11a461946032000f0aafe2db1002305
:1069400004201a46194600f0a3fe44b10023052096
:106950001a46194602b0bde8704000f099be02b078
:1069600070bd836900200b60704738b5144619b9b3
:1069700004220846226038bd1368032b07d9036838
:106980005b6898470028f6d104232360f3e76ff093
:10699000bd00f0e7836900200b6070471830036882
:1069a00000200b6070471830036800200b607047b0
:1069b00038b505460c4615f04df8ab69236015f067
:1069c0004df8002038bd000070b5044622f0b1ff3c
:1069d000124e0346726b06f120001ab19b1ab3f5f2
:1069e0007a7f18d310230021336217f05ffb051e56
:1069f0000fdb22f09eff7063094e234606f1100460
:106a0000324603caa24218605960164603f10803d1
:106a1000f6d1284670bd0025eee700bfd8d00010a3
:106a2000f8d000101fb568460c46fff7cdff0028d0
:106a3000a4bf039b236004b010bd1fb568460c467d
:106a4000fff7c2ff0028a4bfbdf80a30236004b0de
:106a500010bd1fb568460c46fff7b6ff002807dbe0
:106a60009df80520bdf80830d20748bf5b4223607f
:106a700004b010bd1fb568460c46fff7a5ff0028ff
:106a8000a4bfbdf80630236004b010bd70b50e4e33
:106a900088b022f04eff336b1bb1c01ab0f57a7f7d
:106aa0000ed30a4c68460a4902ad0cf07bfe0fcdae
:106ab0000fc495e8030084e8030022f03aff306336
:106ac000014808b070bd00bfd8d00010e0d0001061
:106ad00094d9001038b50d46fff7d8ff044688b1a9
:106ae00003685b699847b5eec00af1ee10fa0cd462
:106af000236820469b699847beeec80a002085edb2
:106b0000000a38bd6ff07700fbe76ff06300f8e72d
:106b100038b50d46fff7baff044688b10368db6855
:106b20009847b5eec00af1ee10fa0cd4236820465f
:106b30001b699847beeec80a002085ed000a38bde3
:106b40006ff07700fbe76ff06300f8e738b50d46ac
:106b5000fff79cff0446b8b103685b699847b5ee40
:106b6000c00af1ee10fa12d4236820465b699847f8
:106b7000dfed087a20ee270abceec00a10ee103acc
:106b800000209bb22b6038bd6ff07700fbe76ff001
:106b90006300f8e70000804338b50d46fff776ff45
:106ba0000446b8b10368db689847b5eec00af1ee59
:106bb00010fa12d423682046db689847dfed087a84
:106bc00020ee270abceec00a10ee103a00209bb25d
:106bd0002b6038bd6ff07700fbe76ff06300f8e7dc
:106be0000000804310b50c46fff750ff28b1036842
:106bf0009b6898472060002010bd6ff07700fbe78e
:106c00000048704774cf00102de9f041504c082126
:106c10002046504a0025fbf7b3ff1c2114274e4b9a
:106c20004e4a23606018a561fbf7aaff4c4bdff8c2
:106c3000cc81e3614b4b4c4ec4e90f734b4b29465f
:106c4000636404f13803a3646563c4f83880e664c0
:106c500004f13c00fbf77afc454b2946a363454b06
:106c6000c4e91458e365444ba765236604f1540353
:106c7000c4e9193604f15800fbf768fc3f4b0921c1
:106c800063653f4ae56604f17000fbf779ff3d4b11
:106c9000c4f8885023673c4c3c4b182223603033a7
:106ca0006360294604f10800b5f037fc102229463c
:106cb00004f12000b5f031fcc4e90c55344c21211d
:106cc0002046344afbf75cff334b25212360334ccd
:106cd000334a2046fbf754ff324b22212360324ccb
:106ce000324a2046fbf74cff314b23212360314cc5
:106cf000314a2046fbf744ff304b24212360304cbf
:106d0000304a2046fbf73cff2f4b282123602f4cb5
:106d10002f4a2046fbf734ff2e4b292123602e4caf
:106d20002e4a2046fbf72cff2d4b2a2123602d4ca9
:106d30002d4a2046fbf724ff2c4b2b2123602c4ca3
:106d40002c4a2046fbf71cff2b4b2360bde8f0814b
:106d500074cf0010fc3b0d02b43c0d02053c0d024b
:106d6000c43c0d020c000200512a0002123c0d022c
:106d7000d43c0d021b0002001c3c0d02e43c0d0241
:106d8000283c0d02f43c0d02d8d00010a4540d0292
:106d900018d00010303c0d02143d0d0248d00010f8
:106da0003b3c0d02343d0d0200d00010473c0d026b
:106db000043d0d0230d00010533c0d02243d0d0265
:106dc00060d00010603c0d02443d0d02a8d00010c0
:106dd000673c0d02743d0d02c0d00010783c0d02de
:106de000843d0d0290d00010893c0d02643d0d02df
:106df00078d000109a3c0d02543d0d0208360d0269
:106e000030b5134b8db01d78e5b100240420224627
:106e10000df10f011c708df80f40fcf787fb9df8fa
:106e20000f3093b12023cde904340a4b1e200a49c8
:106e3000009304aa2346fbf70bf9224621460420bf
:106e4000fcf75cfb28460db030bd1d46fae700bfdd
:106e5000625100108c3d0d02f4370d02012a38b545
:106e6000044602d10b68236003e0022a03d0032a00
:106e70000dd0002038bd0c200d681ef075fe0346b5
:106e80000028f0d095e8070083e80700ebe70068ea
:106e90000028eed00c211ef06ffeeae7012a02d195
:106ea000016000207047022a04bf0b680360f8e706
:106eb000012a034602d1016000207047022a04bf64
:106ec000d1e90001c3e90001f6e7012a02d101601e
:106ed00000207047022a04bf0b680360f8e7012a0c
:106ee000034602d1016000207047022a04bfd1e9a5
:106ef0000001c3e90001f6e7012a02d10160002088
:106f00007047022a04bf0b680360f8e707b5016801
:106f100011f00101019107d106f0aaf9019903b01e
:106f20005df804eb06f05aba06f0a2f903b05df87a
:106f300004eb06f0afba000007b5006850b101a934
:106f4000c0b22ef041fb28b904f0c8fe012201991d
:106f500005f0a0fc04f0c2fe05f09efa0122044bed
:106f60001a700022034b1a7003b05df804fb00bfd7
:106f700013d1001012d1001030b50d46044685b073
:106f800010bb03460a4600900321012008f070f868
:106f9000194b1c700122194bc3e88f2f04f09efe81
:106fa0000722214605f0aefd04f098fe294605f0c3
:106fb000eafaf0b904f092fe05f038f9022818d088
:106fc00001201ff006fdf5e703a9c0b22ef0fcfa80
:106fd00048b904f083fe2a46039905f093fd04f0b6
:106fe0007dfe05f0d4f804f079fe05f07ef8002867
:106ff000dad005b030bd00bf13d1001014d100109d
:1070000001790068fff7b8bf08b504f067fe05f026
:1070100029fa04f063febde808400722002105f0cc
:1070200071bd0000042810b51bd005282dd1184cc7
:107030007e2200212046b5f070fa4ff0ff33c4f8ed
:107040007e30a4f88230c4f85730a4f85b306ff07b
:107050007b0323700023204663701cf003ff20464f
:1070600010bd0c4c572200212046b5f056fa4ff0c7
:10707000ff330021c4f85730a4f85b305d2320466d
:107080002370617016f09afee9e70020e8e700bf80
:1070900015d1001099d1001073b50d46d8b911f073
:1070a000ff0506d104f01afe02b0bde8704005f0fd
:1070b00066b8012d06d104f011fe02b0bde87040a3
:1070c00004f03ebe022d34d104f008fe02b0bde84b
:1070d000704004f03cbe01a9c0b22ef075fa30bb7e
:1070e00004f0fcfd019904f0c5ff0446f8b104f07a
:1070f000f5fd019905f00af8064604f0effd019947
:1071000005f00cf815f0ff0506d1022e01d002287b
:107110000dd1204602b070bd012d04d1022e14bf46
:1071200000240124f5e7022d01d10228f7e700240d
:10713000efe70446ede713b530b904f0cffd02b038
:10714000bde8104005f011b86946c0b22ef03cfa17
:1071500068b9019001a900982ef0fbfa002806db1f
:10716000019800f04100012801d102b010bd0020bb
:10717000fbe70020704713b5044638b904f0aefdb4
:10718000214602b0bde8104004f057bf01a9c0b2cb
:107190002ef01afa30b904f0a1fd019904f04dff68
:1071a00002b010bd0020fbe713b5044638b904f067
:1071b00095fd214602b0bde8104004f04cbf01a986
:1071c000c0b22ef001fa30b904f088fd019904f044
:1071d00042ff02b010bd0120fbe713b5044638b9e9
:1071e00004f07cfd214602b0bde8104004f018be5a
:1071f00001a9c0b22ef0e8f930b904f06ffd019991
:1072000004f00efe02b010bd0020fbe77047002026
:10721000704708b506f02cf8bde8084006f02cb819
:1072200007b50c4b5b68cde90012c3f3080343b903
:1072300006f01ef8dde9001203b05df804eb06f07d
:1072400061b906f015f8dde9001203b05df804eb52
:1072500006f03cb800ed00e010b5052886b011d16d
:10726000104605921cf064fd059b044638b9cde933
:1072700001000090012210200021fff7e3fa2046d0
:1072800006b010bd004cfae7f2feffff13b504464e
:1072900048b904f023fd214604f0eefdb0fa80f079
:1072a000400902b010bd01a9c0b22ef08df940b95d
:1072b00004f014fd019904f0dffd003818bf01202f
:1072c000efe70020ede74ff0ff3070474ff0ff3061
:1072d000704708b505f0ccffbde8084005f0d0bf09
:1072e000704700007fb5104e044696f82c300d46ce
:1072f00093b1706a28f03bfa70b90c4b694603935e
:107300000b4b30460293cde90045fdf749f868463e
:10731000fbf7a6fd04b070bd2046e9b204b0bde89d
:107320007040fff729be00bf9ccd0010816f0002a6
:107330005f6e000237b504460068a8b9002201213b
:10734000174b10461a70174b19700321fff7caff2d
:1073500004f0c4fc05f0aef86368db071dd503b08c
:10736000bde8304005f058bc00220321fff7baff0a
:10737000207801a92ef028f9054628b904f0aefcc2
:107380002a46019905f086fa2368002bd6d004f02e
:10739000a5fc04f0aafe0028d0d003b030bd00bf89
:1073a00013d1001012d1001030b5174d044695f8d6
:1073b0002c3085b08bb1686a28f0d9f968b9134bc5
:1073c00028460393124b694600940293fcf7e8ffaa
:1073d0006846fbf745fd05b030bd54b16946e0b2e3
:1073e0002ef0f2f828b904f079fc0122009905f09a
:1073f00051fa04f073fc05f04ff80122054b1a70a6
:107400000022054b1a70e6e79ccd0010b96e000211
:107410004b6e000213d1001012d100107fb5234e25
:10742000044696f82c300d4693b1706a28f09ff907
:1074300070b91f4b304603931e4b6946cde900459a
:107440000293fcf7adff6846fbf70afd04b070bd80
:10745000a4b900220121184b10461a70174b19705d
:107460000321fff73fff04f039fc05f023f8eb0799
:10747000ecd504b0bde8704005f0cebb204600223c
:107480000321fff72fffe0b269462ef09df8044676
:1074900028b904f023fc2246009905f0fbf904f01a
:1074a0001dfc04f022fe0028d3d0cfe79ccd0010b5
:1074b000b5720002316e000213d1001012d100101b
:1074c00070b52a4b0c465b6886b0c3f30803002beb
:1074d00039d1274e96f82c30b3b1706a28f047f9ad
:1074e000054688b9234b30460593234b02a90294e5
:1074f0000493fbf7b9fd0446c8b9054602a8fbf79b
:10750000affc284606b070bd14f00101019107d10f
:1075100005f0aefe019906b0bde8704005f05ebf13
:1075200005f0a6fe06b0bde8704005f0b3bf2a46e0
:107530004ff0ff31406928f033fa236820469b68fa
:10754000a5699847dae711f00102019208d105f028
:107550008ffe0121019a06b0bde8704005f0b6be6d
:1075600005f086fe00220221f5e700bf00ed00e0f5
:107570009ccd00108d6e00021d6e00027fb5174b72
:1075800004465b680d46c3f308031646ebb9144b7b
:1075900093f82c20cab1586a28f0e9f8a8b90290eb
:1075a0000c201ef0e1fa10b1c0e9004586600d4bd9
:1075b000694603930c4b009009480293fcf7f0fed8
:1075c0006846fbf74dfc04b070bd324629462046a4
:1075d00004b0bde87040fff773bf00bf00ed00e0ee
:1075e0009ccd001095770002dd6d000237b50122b9
:1075f000244b05681a700022234b1a70234bc3e8f2
:107600008f2ffff7fdfb044638b1002211461046cc
:1076100003b0bde83040fff7b1bf04f05ffb214687
:1076200004f0fefb0028f0d01db301a9e8b22df054
:10763000cbff40b904f052fb019905f053fa04f076
:107640004dfb04f0a4fd04f049fb04f086fd18b9dd
:1076500004f044fb04f020ff04f040fb002104f0a0
:10766000dffb60b104f03afb03b0bde8304004f04a
:1076700033bf04f033fb294605f034fae3e703b0e7
:1076800030bd00bf13d1001012d1001014d1001072
:1076900030b5304d044695f82c3085b08bb1686a12
:1076a00028f065f868b92c4b284603932b4b6946a4
:1076b00000940293fcf774fe6846fbf7d1fb05b01b
:1076c00030bd0122264b1a700022264b1a70264b21
:1076d000c3e88f2ffff794fb054638b1002211460f
:1076e000104605b0bde83040fff748bf04f0f6fa99
:1076f000294604f095fb0028f0d024b36946e0b297
:107700002df062ff40b904f0e9fa009905f0eaf9ba
:1077100004f0e4fa04f03bfd04f0e0fa04f01dfd8f
:1077200018b904f0dbfa04f0b7fe04f0d7fa002130
:1077300004f076fb0028c2d004f0d0fa05b0bde812
:10774000304004f0c9be04f0c9fa214605f0caf978
:10775000e2e700bf9ccd00106d750002796e00025b
:1077600013d1001012d1001014d1001070b505f023
:107770007ffd05f081fd00283cd1224e3378ebb926
:10778000214c2378d3b905f04dfa98b31f4bd3e8b9
:107790008f3fdbb20bb1237863bb04f09ffa04f098
:1077a000eefc38bb04f09afa04f0dffc034608bb99
:1077b000bde8704002460146fff76abf04f08efa4a
:1077c00004f0ddfcb8b100220f4c10462578237878
:1077d000edb2002b14bf07210621fff783fd002324
:1077e0001a4619461846fff719fe0023084a337057
:1077f0001360257070bd04f071fa04f0b6fc002827
:10780000e1d1f7e711d1001012d1001014d100100e
:1078100070d9001003681868d3e90112fff7aebef3
:1078200013b543690446cde900030a4990f82220c4
:10783000094b243027f084ff20b10a20074a084969
:10784000f9f7cefb94f82c3013b927f098fff9e73d
:1078500002b010bd993d0d02357800025769020251
:10786000a73d0d02002313b50193036801a91b680e
:107870009847044620b1019828b103681b689847cf
:10788000204602b010bd0446fae708b5012380f88f
:107890002c3004461ef0f0fbb5f030fd251d2046cf
:1078a000fff7e0ffe3680bb9b4f090f828462369ce
:1078b0009847f4e708b5fff7e8ff000070b5054604
:1078c0000c4614f0c7f86b686bb19c600026a6608c
:1078d0006c6014f0c3f8054b586a30b13146bde80e
:1078e000704027f071bf2c60f0e770bd9ccd001098
:1078f00038b50446006868b114f0acf82568ab6888
:107900002360236803b9636014f0a8f828466b6805
:107910009847012038bd704710b504460c211ef071
:107920002bf9204610bd436913b183690c30184709
:10793000704713b500210446084628f017f80023c5
:10794000204601a9019328f081f8019c0cb1012384
:1079500023710021012028f009f82cb1236820466a
:107960009b6898470023237102b010bd08b5fdf74e
:107970006fff48b10df0b0ff002204210df02dfc87
:10798000bde808400df0a6bb6ff0d10008bd0000b7
:1079900009490c2008b5b4f015f8014650b1074b61
:1079a000036000238360064b4360bde80840054840
:1079b000fff784bf08bd00bf0d700f02f03d0d0240
:1079c000a97900023cd9001010b403685a6899687c
:1079d000541001eb6200d20748bf0a591b685df8da
:1079e000044b48bfd3581847012a38b5044602d182
:1079f0000b68236003e0022a03d0032a0dd0002085
:107a000038bd0c200d681ef0aff803460028f0d0fa
:107a100095e8070083e80700ebe700680028eed050
:107a20000c211ef0a9f8eae708b510b103685b68fd
:107a30009847bde80840fff799bf07b5806830b1a7
:107a40000023cde900131a46022128f00bf803b0f9
:107a50005df804fb38b5836804469bb16ff00041c4
:107a6000fff7ebff0021a06827f0f7ff237903f071
:107a7000ff0513b127f083fef8e72946a06828f038
:107a80003bf8a56038bd000038b505460446054bf7
:107a900045f80c3bfff7deff2846fbf7e1f92046ef
:107aa00038bd00bf003e0d0210b50446fff7ecffe5
:107ab00020461c211ef060f8204610bd10b504467b
:107ac000064b03608068fff7c5ff237b23b1a068e6
:107ad00010b103685b689847204610bd143e0d0244
:107ae00010b50446fff7eaff204610211ef044f8c7
:107af000204610bd284b2de9f04103604ff0ff33c5
:107b000006460d4688b04360002943d11c201ef074
:107b10002bf80446002834d00c20d6f804800695b3
:107b20001ef022f818b11d4b8660c0e900351c4bd1
:107b30000490236000230df1080c04af97e80300c4
:107b40008ce803002371a36004f10c0292e80300a7
:107b500087e803009ce8030082e80300114a0693cb
:107b60006261a269414607920f4a04f10800a261ce
:107b7000cde900330d4a234627f056ff3846fbf780
:107b80006ff9b5fa85f530466d09b460357308b004
:107b9000bde8f0810c46f4e7143e0d0211790002b5
:107ba000003e0d026979000249790002b3780002b3
:107bb0006ff000418068fff740bf13b58468002173
:107bc0002046fff73affa06840b100236ff0004263
:107bd0001946cde900231a4627f044ff02b010bd34
:107be000f0b58368054698680e468bb0f0b1002169
:107bf00027f091ff041e18bf0124ab689868b8b144
:107c000000226ff000474ff47a7303217343cde9ec
:107c1000007227f027ff034650b9a8686e60a4b928
:107c200039460bb0bde8f040fff707bf0446e4e774
:107c300020220023cde90223094a3220009209497b
:107c400002aafaf705fa0bb0f0bd80680028fad056
:107c50001a460121cde9007327f004fff3e700bfc6
:107c6000bf3d0d02f4370d02fff780be2de9f04f46
:107c70000025b5b081460c4692460995002a78d079
:107c80005378002b75d029462a221da81c95b4f0e4
:107c900044fc08230c20cde90130cde90c550cad96
:107ca00000959af800102e2350461caa2cf07ef95d
:107cb000014600285dd1102218a8b4f02efc4c23f8
:107cc00014939af80130b9f1110f15930cbf0223e8
:107cd00001232946169314aa09ab1ca8cdf85c9081
:107ce0002cf02af9002844d10125099b4bb9202208
:107cf000cde91c23a44a32200092a4491caafaf719
:107d0000a7f9202100236ff0e508a14acde91c1353
:107d1000009201209d4901951caafaf799f9dff814
:107d20006cb2099c002c00f0aa81d4e902126068b0
:107d30002df02afa00262023071ecde91c3680f2fa
:107d40009880d4e90173e26807930692b4f0b8f919
:107d5000079b0168069acde901738e4b049103924b
:107d600000935946334632201caafaf771f9e469a8
:107d7000d8e7894b5a6822b19b6813b10225099351
:107d8000b3e7002c73d025781db1012d35d0002527
:107d9000abe71022294620a8b4f0bffb02264c23f3
:107da000b9f1110fcde91c360cbf33460123d4f8cd
:107db00002001e93cde91455cde91655cde90c55b9
:107dc000cdf87c900a952ef070fb10230a9014aa2f
:107dd00030460aa92ef065fb002886d00821b4f8a9
:107de00042306e4a0ca8b5f0cffb09ab1caa0ca917
:107df00014a82cf0a1f8032577e71c2200210da878
:107e0000b4f08bfb4823b9f1110f4ff000060c932f
:107e10000cbf022301235c2231461da80aaf0e933a
:107e2000cdf83c901c96b4f078fb60225c4b1ca90a
:107e3000a01ccde90a6608f06af90821b4f84230be
:107e4000564a3846b5f0a0fb2023cde914361cabca
:107e50000193544b28464d49009314aa3346029788
:107e6000faf7f6f8394609ab0caa1ca8c1e7254673
:107e70003be7e36859460493a368012003936368d2
:107e80001caacde90173484b00933346faf7e0f89a
:107e90002a2231461da81c96b4f03ffb60680228d8
:107ea00046d00a2850d020220023cde914231caa52
:107eb000cde901723d4a594600921e20039614aa4c
:107ec000faf7c6f8b9f1110f76d1626800230a2ad1
:107ed00072d11c2219460ca8b4f01ffb1c228df88d
:107ee00030206368022b8df8313032d00a2b30d02d
:107ef000012304220a9340f6ff71384600920aab30
:107f00002df00df960b320230026cde91436b4f02e
:107f1000d7f803685946cde90173254b3220009309
:107f200014aa3346faf794f838462df01ff91ee7e5
:107f30002e2361691caa04312ef0b3fa63695888b4
:107f40002ef0b9fa0646aee761692e231caa083165
:107f5000f2e741f234602ef0acfaadf83200c7e738
:107f600006901c2238460ca92df09af8069b18b3ef
:107f70002022cde914230f4a59460092322014aa38
:107f8000faf766f8d0e700bf2c3e0d02f4370d0279
:107f90004f3e0d02603e0d026451001074650d02eb
:107fa000a1af00021c3e0d029f3e0d02d03e0d020d
:107fb000f53e0d022b3f0d023846d4e904212df089
:107fc000d7f820238046149390b100231593b4f082
:107fd00077f802681cabcde903622c4acde9017346
:107fe000009200235946322014aafaf731f89be791
:107ff0001cabcde90173264b159000932549034630
:108000000396012014aafaf723f8b9f1110f224bb5
:108010000ad1023d012d07d85968e26931b19a6051
:108020004ab90991c3f80480012505e0002afbd074
:108030000999c3e9011245461f60baf1000f04d047
:10804000d4e904215046b4f041fa00260c960ca95c
:108050006068fcf78ffe01220c996068fcf732fe25
:10806000304604f011fe012808d1304627f07dfb90
:108070000a49149014aa38462df0c1f815b1099890
:108080002bf058ff404635b0bde8f08f553f0d024c
:108090008b3f0d02f4370d02645100100873048009
:1080a00030b50a4601461148002300688db02df016
:1080b00067f8041e15dab4f003f8036800250c2bea
:1080c00012d02023cde90435b3f0faff0368084944
:1080d000cde90143074b3220009304aa2b46f9f760
:1080e000b7ff20460db030bd2c46fae764510010b2
:1080f000f4370d02af3f0d0230b50a46014617486e
:10810000082300688db02df037f8041e07dab3f0ad
:10811000d7ff03680b2b05d1b3f0d2ff0024204614
:108120000db030bdb3f0ccff03680b2bf4d0b3f02f
:10813000c7ff03680c2befd020230025cde90435c1
:10814000b3f0beff03680649cde90143054b322079
:10815000009304aa2b46f9f77bffe0e76451001077
:10816000f4370d02c83f0d0230b5144c89b02368b6
:10817000002b1fdbc20715d5012118462cf092fffa
:1081800080b921f0d6fb0546002220216846fff782
:10819000b3ff002806db21f0ccfb41f28732431b02
:1081a0009342f1d920682cf0e1ff4ff0ff332360b8
:1081b00009b030bd6ff0d100fae700bf6451001084
:1081c00013b501a831f0c0fd002242f21073114630
:1081d00001a831f04dfe044601a831f0c6fd20464d
:1081e00002b010bd6ff0770070470000014b1868b7
:1081f000c017704764510010014b1868704700bfea
:108200006451001010b50446503060f0dcf804f101
:10821000440060f0d8f82046faf7c6fa2046bde8d8
:108220001040b0211df0a8bc38b50446062060f00f
:10823000b9f8054668b1204660f0c0f8002229462a
:10824000204660f013f9034628b1bde8384032f00b
:1082500071ba6ff07703184638bd08b560f046f97b
:1082600018b1bde8084032f065ba08bd08b560f045
:1082700059f918b1bde8084032f05cba08bd0022d7
:108280001421c0e90022c0e90222026101800275c6
:10829000427582617047000010b50a4cd4e88f3fe8
:1082a000db070cd420461ff073fd40b10648fff7f2
:1082b000e6ff20461ff0a6fd0448b3f0e0fe0248aa
:1082c00010bd00bffcd1001000d20010a18300023d
:1082d0002de9f0478469a0b0289f002c00f094801d
:1082e000d4f8a0509d4211d39e18ae420ed9eb1a7d
:1082f000761b3246194404f14400fff7b7ff00280b
:1083000069dbd4f8a0303344c4f8a030d4f8a030ee
:10831000bb4229d200217c2201a80091b4f0fdf8d3
:1083200022f0e4f8d4f8a030c61900eb030904f1f8
:108330004408b14516d2a6eb090abaf1800f28bf4e
:108340004ff0800a69465246484622f001f900285b
:1083500041db524669464046fff788ff00283adb7a
:10836000d144e6e7c4f8a070d4f8a030ab4229d9d4
:1083700004f15006304604f1440160f051f830bb7e
:10838000304604f17c0160f0e7f818b132f0d2f920
:10839000002820db4822204604f15c01faf7fefaaf
:1083a000002818dbd4f8ac30ab4203d121f0c1fa7d
:1083b000c4f8a400d4f8a830d4f8a02013445d1b5e
:1083c000c4f8a850d4f8a83043b9002003e032f034
:1083d000b1f90028d4da20b0bde8f08721f0a9fa7d
:1083e000d4f8a430c01a47f22f539842edd9204652
:1083f000faf74af90028eedb21f09bfac4f8a40052
:108400000020c4f8a800e6e76ff0d100e3e710b55c
:108410000446006808b1fff7f5fe204610bd0000d5
:1084200008b50248fff7f3ff08bd00bf18d20010df
:108430000368016013b11846fff7e4be70470000ff
:1084400070b5856906468ab03db3d5e927329a42b0
:1084500026d1202205f15c0105f17c00b4f026f85c
:10846000044688b1002320220e4ccde9022332209d
:108470000d49009402aaf9f7ebfd2046f9f748fbf5
:108480000a4c20460ab070bd2846faf78df92146fd
:1084900006f11800fff7ccfff3e76ff0d104f0e727
:1084a000034ceee7ec3f0d02e13f0d02cdfaffff7a
:1084b000b9faffff10b50446806992b040b1faf7ef
:1084c00087f9002104f11800fff7b2ff12b010bdc8
:1084d000054901a8faf7c8f801a8faf779f901a83f
:1084e000faf762f9f2e700bf1b400d0270b5037d99
:1084f00005468ab0c3b18469b4b1d4f8a8309bb141
:1085000021f017fad4f8a430c01a47f22f5398423a
:108510000ad92046faf7b8f800284ff0000605db24
:1085200021f007fac4e929060ab070bd2023cde97d
:108530000236074b0190009332203346054902aac8
:10854000f9f786fd28460ab0bde87040fff7b2bfd4
:108550002c400d02e13f0d027fb5037d05460e461e
:108560003bb318300021fff763ff687d08b90bf0bb
:108570009dfd0024104ba6421c7018bf01222b4603
:1085800008bf4ff0ff3200214ff48070cde9014465
:108590002c750094fef756f92046fbf779f923462f
:1085a000024600214ff48010cde901440094fef70b
:1085b00049f904b070bd00bf5fcc001070b511f078
:1085c00008020546047d01f0040301f0010626d1ee
:1085d0008cb3e3b984691cb1fff732ff041e10dbd2
:1085e0007eb9002021f0e8ff0446e1432846c90f88
:1085f000fff7b2ff002c10db4620fbf731f8002418
:108600000be02846fff756ff002ceedbe9e742219e
:10861000012021f09fff00eae074204670bd002c8d
:10862000fbd0002bebd10eb1fff744ff0021284611
:10863000fff792ffe3e76ff0d104eee72de9f04397
:108640001f46037d0446894616468db0002b57d041
:108650004ff000082c4bc3f8008021f047ff434641
:10866000c1193246484621f063ff0546c8b12023b0
:10867000264e04aacde904382549434601900096c8
:108680003220f9f7e5fc29463046f9f741fa414630
:108690002046fff761ff6ff0da0528460db0bde810
:1086a000f083a369bbb1149b3246009349463b4615
:1086b0002046fff70dfe70b12023cde90435154ba0
:1086c0000190009332202b46114904aaf9f7c0fc0f
:1086d0002046fff7effe637d13b9e720f8f7ecfdc6
:1086e000236902223b44636000234ff48070cde98c
:1086f00001330093002123462681fef7a3f8cce73f
:108700006ff0d105c9e700bf64cc001050400d02e6
:10871000e13f0d022c400d022de9f04fa5b0019074
:108720008846b02066491646b3f04cf9044698b125
:1087300000256449f9f798ff48222946c4e91155f4
:10874000c4e91355c4e9155504f15c00b3f0e5fe26
:10875000c4e92955c4f8ac500394002c00f0ad8056
:1087600004f14400fff760fd041ec0f296800398f8
:108770005030fff759fd041ec0f28f80039d482240
:1087800005f15c0739462846faf78af84828044676
:1087900040f08a80d5f89c30434552d1d5f8a030be
:1087a00043454ed8202231463846b3f07ffe8246fc
:1087b000002846d103984430fff74ffd041e6cdbc0
:1087c00051467c2205a8cdf810a0b3f0a6fe21f0fa
:1087d0008dfe8346d5f8a03000eb030ad34517d2af
:1087e000aaeb0b09b9f1800f28bf4ff0800958465a
:1087f0004a4604a921f0acfe041e4edb03984a460b
:1088000004a94430fff732fd041e46dbcb44e5e704
:10881000039800f1440150305ff002fe002838d187
:10882000039804a950305ff097fe18b131f082ff31
:10883000041e32db202204a905f17c00b3f036fed1
:10884000d8b10398f9f7c4ff06f1200356f8042bba
:108850009e4247f8042bf9d12022002105f17c002b
:10886000b3f05bfe00230398c5f89c80c5f8a030e8
:108870004430fff7f2fc041e0fdb00240399d5f807
:10888000a0300198c1f8ac3018300394fff7d0fd48
:1088900003e031f04fff041ec2da03a8fff7b7fd73
:1088a000204625b0bde8f08f0028cada10f1aa0fe3
:1088b000c7d010f58c7ff0d1c3e7034cede700bfc4
:1088c0000d700f021b400d02fcfeffff2de9f0476b
:1088d0008cb0149d04460f461e46904605f00409d0
:1088e00005f0010abab1b3b1c5f34005227da2b1ca
:1088f000002320216a4ccde904133220694904aadf
:108900000094f9f7a5fb2046f9f702f96ff0d100c2
:108910000cb0bde8f0870125e8e7012004a98df837
:108920001020faf703fe9df8102012b16fb95e48cf
:10893000eee7092004a98df81020faf7f7fd9df85d
:108940001030002bf2d15948e2e721f0d5fdb842b2
:10895000edd3baf1000f1bd1d5b9424639462046b6
:10896000fff7dafe002874da20220023cde9042381
:108970004f4a0190009232204a4904aaf9f768fb55
:10898000b9f1000f40f084802046fff793fd07e027
:10899000b9f1000f77d12046fff78cfd002ddcd018
:1089a00021f0a4fd3946002221f0b0fd0146002847
:1089b0005bd04ff00008002211461046faf79efdea
:1089c000f8f710fd0546607558b901200bf06efbf5
:1089d00029460b20fdf7a4fc00284dd000690bf0c0
:1089e00088fb01230025334a237513701423a44602
:1089f000cde90455cde907550695adf810300df1d8
:108a0000100ebee80f00ace80f00ccf80050e76095
:108a100021f06cfd206121f075fd236920816360e8
:108a20002a462346a57200214ff48070cde90155f6
:108a30000095fdf707ff2846faf72aff2b46024666
:108a400000214ff48010cde901550095fdf7fafea5
:108a500020e0a369d3f8a080b9f1000f0fd0002166
:108a600004f11800fff7e4fc14e004f11800fff72c
:108a7000dffc6ff0da004be74ff0ff10afe7b8f123
:108a8000000f98d18ce71db9baf1000f3ff465af24
:108a90004ff000080eb1c6f80080002038e700bf94
:108aa00071400d02e13f0d02b9faffff9cfaffff92
:108ab00098400d025fcc001048b10138222896bfc3
:108ac00005230723b0fbf3f34ff47a709840704707
:108ad00008b578b103881b2b0cd94ff0ff33037115
:108ae00000234371837105231422c37102490830a6
:108af000b5f05cfb1c2008bd83370d0210b50446a1
:108b0000007c10b1d4e902309847207410bd03688e
:108b100002224068184770470eb4f0b5002692b0a4
:108b200017ad55f8047b3c223146044603a8029653
:108b3000b3f0f3fc3a462b46402102a80195b5f06c
:108b400025ff3f28024605dd267412b0bde8f0403f
:108b500003b07047204602a9fff7d0fff5e710b534
:108b6000044614211df008f8204610bd13b5044634
:108b700008460191f8f726f902462046019902b00d
:108b8000bde810400af074bc37b56fea41416feaa6
:108b90005141adf8041001a904461546fff7b7ff8f
:108ba00030b104222368606801950deb02019847fb
:108bb00003b030bd7fb50e461546044608b10369c3
:108bc00023b90a20094a0a49f8f70afa0c23cde921
:108bd00001362b68012103932046236901aa984797
:108be00008b9039b2b6004b070bd00bf5769020237
:108bf000cb400d0237b5c3880446012b0d4604d087
:108c00000a20074a0749f8f7ebf9042329462046ca
:108c10000deb03020193fff7cdff03b030bd00bfa2
:108c200057690202f1400d0237b5c3880446022b92
:108c30000d4604d00a20074a0749f8f7d1f9042362
:108c4000294620460deb03020193fff7b3ff03b063
:108c500030bd00bf576902021d410d0273b5cb88bc
:108c60000546012b0c4605d0022b17d06ff077007c
:108c700002b070bd0023694620460093fff7baff9b
:108c80000246f0b9a388286801a9009eadf8043017
:108c9000fff73dff48b96ff0bd00e9e700236946e3
:108ca00020460093fff7c0ffeae704222b680196f5
:108cb0001c6858680deb0201a0470028ebd000208b
:108cc000d6e7a1882868fff75ffff6e70b46014665
:108cd0001846fff7c3bf13b5044608460191f8f7dd
:108ce00071f802462046019902b0bde810400af032
:108cf000afbb000038b5044615460068fff7ebff30
:108d000020680af0f3fa06492068fff7e4ff2946d5
:108d10000af0f8fa20680af0c7fa2368187c38bd10
:108d2000ff460d0273b5054688680c4630b1cb8806
:108d3000012b05d0022b19d06ff0770002b070bd67
:108d40000023204601a90193fff754ff0246f0b922
:108d5000019ea1682868fff7beff31460af0f6fac7
:108d60002b681b7ccbb96ff0bd00e7e700232046e2
:108d700001a90193fff758ff024640b9019ea1687f
:108d80002868fff7a8ff31460af0f2fae8e728461c
:108d9000a168fff7afff0028e5d00020cee70b4623
:108da00001461846fff7bebf2de9f04f9a4b99b028
:108db0001546039300240123cde90501974903a833
:108dc0008df81c308df81040fff785ff69880af098
:108dd00099fa24272b8aa3420dd907fb04f6eb68e6
:108de00003a89959fff777ffe9680134314404314a
:108df000fff7bcfeeee78a4903a8fff76cff03a864
:108e00000af068fa4ff00008dff848922b894345d2
:108e100040f2f980782606fb08f6d5f804b00beb93
:108e2000060494f82230052b00f2d280002b00f0cb
:108e3000d380a37b012b04d1b4f870309b0740f1a1
:108e4000cb8004f114073846f8f73ef8824603a8b1
:108e50000af04cfa734903a8fff73dff5bf80610d0
:108e60000af086fa704903a8fff735ffa37b032bae
:108e700096bf6e4a6e4952f82310fff777fe6d4990
:108e800003a8fff728ffb4f86e100af03bfa6a490e
:108e900003a8fff720ffb4f870100af033fabaf114
:108ea000050f2ed100213c2209a80891b3f035fb13
:108eb000624903a8fff70fff04f16c0604f14c03ad
:108ec00008aa13f8011b0232090901f1300cbcf1a8
:108ed000390f88bf01f1370c02f802cc13f8011cde
:108ee00001f00f0101f1300cbcf1390f88bf01f125
:108ef000370c9e4202f801cce3d1402208a90af0c7
:108f0000b7fa4f4903a8fff7e6fe06463846f7f7db
:108f1000dbff082898bf59f8201030464ff00006b4
:108f200088bf4349fff722fe38460896f7f7cfff80
:108f3000444a0346042108a8b4f026fb424903a88a
:108f4000fff7c9fe08a9fff711fe404903a8fff784
:108f5000c2fe82463846f7f7bfff014650460af088
:108f6000d1f93b4903a8fff7b6fe03a80af0b2f90e
:108f7000dff8ccb094f8247094f82530b4f826a02b
:108f8000052f34d8002f35d003a801930af0aef98d
:108f9000594603a8fff79ffe59f82710fff7e6fd93
:108fa000019b284a042108a8b4f0eefa264903a838
:108fb000fff791fe08a9fff7d9fd244903a8fff7a1
:108fc0008afe51460af09ef903a80af06df911e0f5
:108fd000073b012b7ff62daf08f1010816e70126ac
:108fe00094f8287094f82930b4f82aa0c8e7f91f3b
:108ff0000129c9d9002ef2d003a80af04cf903a820
:109000000af052f9e8e703a80af045f99df81c00b8
:1090100019b0bde8f08f00bfac410d0245770f02db
:10902000592d0d02d4450d02368f0d0294410d02cb
:10903000fbc40d02f1dc0d024a410d0275650d0203
:1090400044750f0274650d0258780f02a3d50d0206
:1090500083440d0270410d0218b10022012121f05c
:1090600054b90148704700bff2feffff18b100225b
:10907000114621f04ab90148704700bff2feffffd8
:1090800030b587b004460d461222002101a8b3f086
:1090900044fa14230022adf804300123114601a83c
:1090a000adf81630fff7d8ff294601aa2046fff792
:1090b0007bfe0446002101a8fff7d8ff204607b039
:1090c00030bd000003681f221b680149184700bf1c
:1090d0004d410d02f0b512f0010489b00e4605466f
:1090e0000e9933d0cde9033103ab0193022302a9da
:1090f00003a8adf80830fff70afd10b96ff0bd0006
:1091000022e00423019802a9adf80830fff7fffc24
:109110000028f3d095b100242746a64233d0002280
:1091200035f8140002a90297f9f772fa60b90299aa
:1091300001a8fff793fd38b90134eee72b46294625
:109140001f4801aaf9f740fa09b0f0bdcde9053191
:109150001c4b8df81040039301238df81c3003ab9a
:10916000184601930af0c2f8019b1b7c002bc5d066
:10917000e5b12746a64208d101980af095f8019b6f
:109180001b7c002bbad00020dee7002235f814004b
:1091900002a90297f9f73cfa0028d5d1029901a853
:1091a000fff7c0fd0028cfd10134e3e72b46294665
:1091b000054801aaf9f708fa0028ddd0c4e700bf86
:1091c0004d8c0002ac410d021f8d000213b500242e
:1091d0000346cde9001420462146fff77bffb0fa95
:1091e00080f0400902b010bd70b5264b88b0002455
:1091f00003930123cde90501234903a88df81c3011
:109200008df81040fff767fd0af064f801f024fcc8
:1092100026460546ac420ed0204602a9029601f031
:1092200021fc10b1002008b070bd029903a8fff71f
:109230009dfc0134eee703a80af02df8134903a8ba
:10924000fff749fd0af052f8002401f0e5fb26463d
:109250000546ac4211d0204602aa01a9cde901661b
:1092600001f0e0fb0028ddd1019903a8fff733fdf1
:1092700002990af047f80134ebe703a80af014f862
:109280000120d0e7ac410d0244750f02a3d50d02b9
:1092900040f6287384b0adf80c3040f6277341f2e5
:1092a000d832984288bf0df10603adf8060098bf8a
:1092b00003ab1988adf80e2091424ff0500288bfe1
:1092c0000df10e031b88a3f628739bb2adf80a308c
:1092d000bdf80a309bb2b3fbf2f3adf80a30bdf82b
:1092e0000a309bb203eb83031b019bb2adf80a303b
:1092f000bdf80a3003f628739bb2adf80a30bdf80a
:109300000a0080b204b0704770b5002501260446fb
:1093100020222946c0e90055c0e90555c0e9075596
:10932000c0e909550672c560067485853030b3f012
:10933000f4f804212b463246601826f06bfa636875
:1093400023b90a20024a0349f7f74afe204670bdb6
:1093500057690202bc410d0210b5084cd4e88f3f9a
:10936000db0709d420461ef013fd28b10448fff79f
:10937000cbff20461ef046fd014810bd1cd2001058
:1093800020d200101fb500234ff480620393cde973
:1093900000320849084b092203a826f0d1f9039ba3
:1093a00023b90a20054a0649f7f71afe05b05df809
:1093b00004fb00bfdf410d02019d0002576902025c
:1093c000e3410d0207b50122054b01a91a700023e4
:1093d00040681a46019326f028fa03b05df804fbb2
:1093e0007051001008b5fff7b7ffbde80840fff760
:1093f000e9bf0846fff7e6bf07b5036843b102239c
:109400004ff0ff3201934068002301a926f00dfac6
:1094100003b05df804fbcb0744bf002380f829307c
:109420008a0741bf002380f82b3080f82d30c361bc
:109430004b0744bf002380f82830002311f0080fa9
:109440001cbf036280f82c3080f82a30704737b593
:1094500004460d4601a801210bf0fdf9236b01a87c
:109460005b0500d4bdb10bf0b2fa78b1ff21204604
:10947000fff7d1ff01a80bf013fc01a80bf0eefce5
:1094800020f057fa60624ff47a73a36101a80bf0e1
:1094900001fa03b030bd0bf09afa0028f6d1ff2193
:1094a0002046fff7b8ff01a80bf0dffb01a80bf087
:1094b000ecfce8e707b50021084621f0c0fb88b9bd
:1094c0000146019021f0a8fc019a1346114610466e
:1094d00021f06afd019a1146104603b05df804ebd5
:1094e00021f004be03b05df804fb0000002320223d
:1094f00010b504468ab0cde90223104a1049009203
:10950000282002aaf8f7a4fd236bd9050ad401216b
:1095100002a80bf0a0f9012102a80bf083fc02a81d
:109520000bf0b8f91b200af0abf90023054a936150
:10953000054a936123600ab010bd00bf0c420d02c2
:1095400002420d0220cc00103ccc001037b504467e
:10955000084600212ff0d0fc2368054643b10123c3
:109560004ff0ff3201936068002301a926f05df9f6
:10957000284603b030bd000070b50c464e79204639
:1095800000212ff0a5fc054638b92379ff2b04d024
:109590006379013bdbb2fd2b07d9202e32462046f2
:1095a00028bf20221b49b2f091ff4ff6fd72e388dd
:1095b0002846013b9bb2934288bf40f628734ff682
:1095c000fd7288bfe3802389013b9bb2934288bf31
:1095d0004ff461734ff6fd7288bf23816389013bad
:1095e0009bb2934288bf4ff460734ff6fd7288bf01
:1095f0006381a389013b9bb2934284bf41f2100374
:10960000a381a37b013bdbb2fd2b84bf1223a37399
:1096100070bd00bf48420d0201462023303180f862
:109620003530fff7a9bf0000f0b587b00446002130
:1096300001a80bf010f901a80bf06ef902ad074676
:109640002a46184bb4f838c003f1100e2e4618689d
:109650005968083303c673453546f7d1082064239b
:10966000194632f8023b9c4502d30138f8d119461d
:109670008f4202d001a80bf09cfa01a80bf07ef9f2
:109680000546e08efff704fe854206d0e08efff728
:10969000fffd014601a80bf003fa01a80bf0faf850
:1096a00007b0f0bd2c240d0213b50c4601a8002113
:1096b0000bf0d1f801a80bf061f940f6287188424f
:1096c00002d001a80bf0ecf914b101a80bf0f5fbe6
:1096d00001a80bf0dff802b010bd8009431e022b79
:1096e00094bf013001207047f7b504460e4601a82b
:1096f00001210bf0b0f801a80bf0b5f801a80bf0b0
:109700007cfba18f01a80bf015fb642101a80bf0d5
:10971000b0f9618f01a80bf0dbfa4ff4807101a85a
:109720000bf03afb2b4b197e11b18a1f514251416c
:109730002046fff78cfe01a80bf05ef910b901a8d6
:109740000bf0d1fb01a80bf00df9054601a80bf0b9
:109750002cf928b901a80bf073fa002d18bf2e467a
:1097600001a80bf005f9074601a80bf0d5f864280d
:109770001fd93846fff7b1ff012806d0226b12f43b
:10978000007318d0831e58425841ceb105b9b8b9fc
:1097900020f0cff8054601a80bf0e4f868b120f0fe
:1097a000c8f8401bb0f57a7f07d232201df011f9be
:1097b000f1e70020e9e71846e7e701a80bf07dfb99
:1097c000ff212046fff727fe01a80bf063f803b046
:1097d000f0bd00bf20cc001037b5036804460d462d
:1097e000abb10d4b1b7e062b02d10021fff77cff96
:1097f0007db1237c6bb1002168460af0c5f968464b
:109800000af0f9fa0023684623740af0cdf903b090
:1098100030bd01232374fae720cc0010f0b587b0e7
:10982000044615460f4620f084f842f210730026d5
:10983000a361ab1f594260615941204684f82d60f5
:10984000e661a662fff703febd422dd1032d12d1c2
:1098500020f06ff8236ac01a41f2873398421dd86e
:1098600020f067f894f82c3020620133dbb2012b32
:1098700003d884f82c3007b0f0bd314684f82c6052
:1098800004a80af0e8ff802104a80bf085fa4ff441
:109890007a7304a8a3610af0fdffece720f049f811
:1098a00084f82c602062e6e7062f0dd1314604a82b
:1098b0000af06af904a80af095fa20460121fff798
:1098c00013ff04a80af070f9022d0ed0032d0fd05b
:1098d000104b2a469d6100234ff480300021cde9d2
:1098e00001330093fcf7aeffc5e701232372efe7d6
:1098f00020f01ff80021206284f82c1004a80af040
:10990000aaff4ff4807104a80bf046fa04a80af0ed
:10991000c1ffdde720cc0010012937b5054614460c
:109920001ad10b21fff777fd2f4b1a7e012a39d070
:109930001cb190f828400134e4b24ff47a72012c43
:1099400085f82840aa612dd901222846197e03b046
:10995000bde83040fff762bf022914d10e21fff7a6
:109960005afd214b1a7e022a1cd01cb190f82940c6
:109970000134e4b24ff47a72012c85f82940aa61cf
:1099800010d90222e1e703290cd10023038580f8d6
:109990002a304ff47a7383611ff0cbffe8611cb962
:1099a00085f82b4003b030bd95f82b300133dbb286
:1099b000032b85f82b30f5d995f82d3013b10622fd
:1099c000094bc2e7012185f82b3085f82d1001a83d
:1099d0000af041ff4ff4967101a80bf04af801a874
:1099e0000af058ffdee700bf20cc001030b52deda7
:1099f000028b002185b00446fff729fd012102a852
:109a00000af0c2f802a80af013f9264db0ee408a17
:109a1000297e91b9f7ee007ab4eee70af1ee10fa7a
:109a20004cbf062201222046fff7f8fe02a80af0ea
:109a3000bbf805b0bdec028b30bd062912d1f7eea4
:109a4000007ab4eee70af1ee10fa1ddd94f82a3040
:109a500013b94ff47a72a2610133dbb2012b84f89f
:109a60002a30e3d9012101a80af0f5fe01a80af085
:109a70007fff43070ad40422297e2046fff7cefe4b
:109a800001a80af007ffd1e70a46cce7f7ee007a13
:109a9000b4eee78af1ee10fa297e4cbf06220122cd
:109aa000ebe700bf20cc00107fb52d4d044601210f
:109ab00001a80af0d0fe2e7e062e28d101a80af0b9
:109ac00086ff20bb1ff035ff636ac01ab0f5fa5f4e
:109ad00015d3012102a80af057f802a80af0a8f845
:109ae000f7ee007ab4eee70af1ee10fa0cd5204654
:109af0003246297efff792fe02a80af055f801a827
:109b00000af0c8fe04b070bd02a80af04df80021aa
:109b10002046fff79cfc01a80af02affc0f30111c0
:109b2000032907d12b7e032b15d001222046fff7f6
:109b3000f3fee4e70139012902d801220221f5e709
:109b4000430705d404222046297efff767fed6e7a7
:109b500001221146eae742f21073a361cfe700bf8a
:109b600020cc001073b5294d04462b7e042b04d164
:109b700042f2107382699a4240d0e36993b91ff0b0
:109b8000d8fe6369c01aa369984237d31ff0d1fe8b
:109b9000236b60615b05204632d502b0bde87040a2
:109ba000fff724bf1ff0c5fee369c01ab0f57a7f46
:109bb000e5d3012101a80af04efe236b5a0510d40b
:109bc00001a80af004ff60b194f82d60032220463a
:109bd000297efff723fe76b1642101a80af049ff30
:109be00009e0ff212046fff716fc42f21073002126
:109bf000a361fff72cfc01a80af04cfe02b070bd77
:109c000002b0bde87040fff74fbf00bf20cc00108e
:109c10002de9f043574b04461a7889b0002a7cd0ce
:109c20000022012105a81a700af015fe012106a8dc
:109c300009f0aaff05a80af09efe8df8170005a8f6
:109c40000af099fe9df8173018430206c7b21dd5d9
:109c500001212046fff748fd05a80af089fe10f013
:109c6000300f0546c0f38006c0f3011814d005a8d4
:109c70000af0adfed0b1b8f1030f07bf0122414693
:109c8000002202212046fff747fe0fe005a80af058
:109c90008cfe0028dcd0dfe73b07c7f3c0023fd5ce
:109ca0000522354b2046197efff7b8fd0020d4f879
:109cb000309024f0c8fc314f8046002e35d12e4b19
:109cc0001b7e042b0cbf052500253b7eab420ad032
:109cd0000023bd612a464ff400300021cde9013355
:109ce0000093fcf7affd06a809f0f1ff78b106a8d4
:109cf0000af05bf8237a53b100234ff400401a4670
:109d00000021cde9013323720093fcf79bfd06a8e7
:109d100009f04aff05a80af0bdfd09b0bde8f083cf
:109d20000eb90422bde70121ace705a80af01afe2e
:109d300001460028c3d12846fff7cffc032805467b
:109d400014d0042812d0022805d119f4007f02d1c2
:109d5000b8f1030f04d82046fff766fc3546b4e798
:109d6000bb6913f0fd0f14bf012100212046fff74e
:109d70009bfcaae77051001020cc00103ccc0010d6
:109d8000f0b58db0fff7e8fa0446002025f0edfcb1
:109d900020602046fff740fc256b15f4807514d039
:109da00000252023cde90435494b4a49009304aaf4
:109db0002b462820f8f74cf92046fff797fb28465a
:109dc0000db0bde8f04025f0ecbc2046fff772fb7b
:109dd000022115201df044fc4ff0ff3302223e49c2
:109de0001520009509f022fd02211b201df038fcf2
:109df0004ff0ff33022238491b20009509f016fd71
:109e0000012103a80af027fd03a80af02cfd012177
:109e10002046fff769fc03a80af0adfd03a80af08d
:109e2000aafd012104a809f0affe04a80af007f872
:109e3000236b5b0503d4142104a809f091ff04a847
:109e400009f0b3ff00222146244824f0fefb42f231
:109e5000107304a8a36109f0a7fe03a80af01afd75
:109e60001f4f00234ff47a72606803a925f0fefcaf
:109e7000054650b9039e012e0dd12046fff7ccfbbd
:109e800029462046fff730fc3e703b78dbb9204680
:109e9000fff768fee5e7022ef7d101212046fff724
:109ea00023fc237c7bb9012104a809f06dfe04a8e2
:109eb00009f0c5ff01234ff4fa7023741cf089fdeb
:109ec00004a809f071fe2046fff7a2fedde700bfff
:109ed0002b420d0202420d026593000273930002b1
:109ee0007051001070470368c1f8d030d1f8e030ed
:109ef00043f00403c1f8e03070470368c1f8dc3078
:109f0000d1f8e03043f00803c1f8e030704703684f
:109f1000a1f8e830d1f8e03043f01003c1f8e030a8
:109f200070470368a1f8ea30d1f8e03043f020032d
:109f3000c1f8e03070470368c1f8e430d1f8e03090
:109f400043f04003c1f8e03070470368a1f8ec30fb
:109f5000d1f8e03043f08003c1f8e03070470023cf
:109f600081f8e03081f8e13081f8e23081f8e330c7
:109f700070470000f0b404460f46bab90388b3f541
:109f8000837f0cd10b4e051d06f12002334603cb17
:109f90009342286069601e4605f10805f6d100234a
:109fa0003a462146f0bc184612f00cb94ff0ff308b
:109fb000f0bc704774cd00101fb500240a46009411
:109fc000014603ab2046039412f00cf900b1039450
:109fd000039804b010bd10b5002488b02146cde927
:109fe000040404a8cde906441ff0f0fd2346012235
:109ff0004ff480400021cde901440094fcf722fc9d
:10a0000008b010bdf7b50d4616461f460446fef7cc
:10a0100043f933462a4621460097fef70ffb03b06b
:10a02000f0bd07b50190fef737f9019903b05df86f
:10a0300004ebfef7c3baf7b50d4616461f460446b5
:10a04000fef72af933462a4621460097fef73efce2
:10a0500003b0f0bd1830036800200b607047183063
:10a06000036800200b60704700b50b4a8bb0137873
:10a0700073b10121094b1e20197000231370202297
:10a08000cde90223064a0749009202aaf7f7e0ff4a
:10a090000bb05df804fb00bf5dcc00105ccc001081
:10a0a00068420d02f4370d0208b510b103685b6811
:10a0b0009847bde80840fcf726bc13b5044601915b
:10a0c000f6f780fe0199a0f1180204f11800b4f02f
:10a0d00059f8b0fa80f0400902b010bdf0b5efb009
:10a0e00005460c46f6f76efe172842d91822284678
:10a0f0006e49b4f047f8074600283ad12046f6f7f3
:10a1000061fe6b4902462046b4f03cf86949b0fa5a
:10a1100080f62846fff7d1ff7609044638b13a4663
:10a12000314609206fb0bde8f040f9f7e7b928469d
:10a130006149fff7c2ffd0b12046f9f7a9fb012220
:10a140005e4b05461a70314622462046f9f7d6f98d
:10a150002046f9f79dfb8542024608d023464ff47e
:10a1600080100021cde901440094fcf76bfb6fb037
:10a17000f0bd132228465249b4f004f8064680b9cf
:10a180002023cde924304f4b4f49009324aa0346a6
:10a190000120f7f75dff30466fb0bde8f04020f0da
:10a1a00081bb28464949f6f703fe002846d1002c1a
:10a1b000ddd02378002bdad021464548f6f7f8fdac
:10a1c00020b96fb0bde8f0400af0bbba2146414863
:10a1d000f6f7eefd20b96fb0bde8f0400af096ba90
:10a1e00021463d48f6f7e4fd20b96fb0bde8f040e8
:10a1f0000af0a4ba21463948f6f7dafd04460028e9
:10a20000b5d12023cde92430354b2f49009324aa22
:10a2100003462820f7f71cff32490c20b1f0d2fb8f
:10a2200001460028a3d0304b846003602f4b43606d
:10a230002f486fb0bde8f040fdf740bb182228461c
:10a240002c49b3f09fff002891d12023cde9243081
:10a25000294b1d4924aa009303461e20f7f7f8fe58
:10a26000032011f091fe04464ff49372ff2124a8bd
:10a27000b2f053f98022ff2104a8b2f04ef95cb18c
:10a280001e4b1f491a6824a8b2f020f91d4b1e4925
:10a290001a6804a8b2f01af9214624a820f055fb48
:10a2a000214604a820f05cfb61e700bf33480d02a3
:10a2b00088360d0213480d024c480d0260cc001088
:10a2c000ff470d0293420d02f4370d02ec470d02d9
:10a2d000c9420d02d3420d02d7420d02fe420d02c9
:10a2e000de420d020d700f02f03d0d0229a00002aa
:10a2f0003cd900101a480d0206430d02f82f0d023a
:10a300009c2f0d02982f0d027f2f0d02f7b50646e8
:10a31000184fd7e88f5f15f0010522d138461df0a0
:10a3200037fdf0b12a4614210f20fcf703f81e2256
:10a330000221114c0346cde9002120460f226ff087
:10a340007f410af021fa0d4b384623600c4b84f80c
:10a3500022506361642323841df054fd0948b1f049
:10a360008efe00223146084803b0bde8f040f7f702
:10a3700053bf00bf70d2001034d300105c480d02f0
:10a38000ee82ee0035a5000238d30010012a38b560
:10a39000044602d10b68236003e0022a03d0032a9b
:10a3a0000dd0002038bd0c200d681bf0ddfb0346ee
:10a3b0000028f0d095e8070083e80700ebe7006885
:10a3c0000028eed00c211bf0d7fbeae7012af8b5f4
:10a3d000064603d10b6803600020f8bd022a08d0ae
:10a3e000032af9d100680028f6d018211bf0c4fb1d
:10a3f000f2e718200c681bf0b7fb074630b10546a2
:10a400000fcc0fc594e8030085e803003760e3e74d
:10a41000012a08bf016000207047012a02d10160b3
:10a4200000207047022a04bf0b680360f8e7012a86
:10a4300002d1016000207047022a04bf0b6803604c
:10a44000f8e7012a02d1016000207047022a04bf08
:10a450000b680360f8e7012a02d101600020704711
:10a46000022a04bf0b680360f8e7012a02d10160e9
:10a4700000207047022a04bf0b680360f8e7012a36
:10a4800002d1016000207047022a04bf0b680360fc
:10a49000f8e7012a08bf016000207047012a08bfc1
:10a4a000016000207047012a70b5054603d10b6892
:10a4b0000360002070bd022a11d0032af9d104687c
:10a4c000002cf6d004f1180009f0e6ff04f10800b2
:10a4d00009f0e2ff2c2120461bf04efbe9e72c207f
:10a4e0000e681bf041fb044688b1338806f1080171
:10a4f00003807368083040f8043c0af063f806f102
:10a50000180104f118000af05df8b36aa3622c6028
:10a51000cfe7002307b5009342f001033c22fbf78d
:10a5200059fd03b05df804fb10b58ab002f0a0fb42
:10a53000042813d100242023cde90234084b02aab9
:10a5400000931e2023460749f7f782fd224606495d
:10a5500006480ab0bde81040fff7dbbf0ab010bde7
:10a560003e430d02f4370d02af2c0e0256430d028e
:10a57000002210b50446044b114640f8043bf7f79f
:10a580004bfe204610bd00bf64470d0210b50446c7
:10a59000fff7eeff204620211bf0eefa204610bd0b
:10a5a00010b50446024b0360fff7e2ff204610bde2
:10a5b0005c480d020148fff7f3bf00bf34d3001021
:10a5c00010b50446fff7ecff204624211bf0d4fa17
:10a5d000204610bd038c8b4211d890f822300133f5
:10a5e000dbb2072b08bf002380f8223090f822202e
:10a5f000044b53f8223043616423038470475b1a91
:10a60000fbe700bfd0470d0207b50068036901935f
:10a6100002238df8033083680bb9b1f0d7f9c36812
:10a620000df1030201a9984703b05df804fb000097
:10a6300070b500242026144b8ab0144d1e201449f6
:10a64000009302aa2346cde90264f7f701fd2246f2
:10a65000022128680af0c1fd044620b10ab0bde815
:10a6600070400af037bd0b4bcde90260009302aa9f
:10a67000034607491e20f7f7ebfc286821460af03d
:10a68000ddfe20460ab070bd6c430d0260d30010a1
:10a69000f4370d0289430d0230b500248bb02346f8
:10a6a00022460f49cde900440e48fbf7d3fa234672
:10a6b00005462246cde9004409490b48fbf7cafa92
:10a6c00000b155b920220023cde90223074a3220e8
:10a6d0000092074902aaf7f7bbfc0bb030bd00bfe0
:10a6e0005da000029f430d02a8430d02ae430d0280
:10a6f000f4370d022de9f041adf58a6d08238e4d3a
:10a7000002af00222868391dbb800af0a4fe02f0c7
:10a71000affa042800f0ec80f988002022f087ffcf
:10a720000120398922f083ff032011f02dfc382409
:10a7300080462246002107f14400b1f0eefeb8f158
:10a74000000f14bf02230123a7f8444087f84630c6
:10a7500000f0ec80794bbb64794bfb64794bfb6672
:10a76000794b3b67794b7b67794b1c223b65794b77
:10a7700000217b65784b07f18000bb65774b07f1c3
:10a780007c04fb65764b07f1bc063b66754b7b662c
:10a79000754bbb66754bbb67b1f0bffe40232360b2
:10a7a000734b4ff49372e360724bff21a363724bc0
:10a7b00030462362714b6362714ba362714be3635a
:10a7c000714b6363714be362714b2363b1f0a5fe80
:10a7d00007f5f27318464ff41972ff21b1f09dfe90
:10a7e0001022ba820822fa60012207f10c013a74a1
:10a7f000c7e9060620f010f830461ff0f6ff97f87c
:10a80000bc30ff2b19d120220023c7e90923614a5c
:10a8100028200092604907f12402f7f719fcb8f1eb
:10a82000000f05d05d4b30461a685d49b1f04efe11
:10a830005c4a136843f001031360002108461af0d4
:10a840003bfe0026c1b2cb1d03f4fc73adeb030d40
:10a850000df1080840461af02ffe4146286807f11e
:10a86000440307f11402cde900460af099fc33468f
:10a8700032460221286800960af0f5fd25f074f9a9
:10a88000b0f57a7f06d3334601220321286800966b
:10a890000af0e9fd002441f28a32234604212868a7
:10a8a00000940af0e0fd2e681ff026fe23460246c3
:10a8b0000521304600940af0d6fd2e681ff022fed6
:10a8c000234602460621304600940af0ccfd0823b8
:10a8d000bb84354b07f124011b682868bb620af072
:10a8e00059fcfff7d9fe07f58967bd46bde8f08141
:10a8f000002022f09ffef880012022f09bfe4ff600
:10a90000ff73f9883881994204d0002328681a46d9
:10a910000af09dfd4ff6ff73398999423ff404af69
:10a92000002328681a460af094fdfde61f4bbb641d
:10a930001f4bfb6418e700bf60d30010d94b000227
:10a94000294c000274cd0010f59e0002399f0002d0
:10a95000b79f0002a39f0002859f0002c1bd0102b4
:10a960008da20002b3980202579f0002e99f0002e5
:10a97000e9b90002f1b7000263a7020267a7020269
:10a9800001900002699100024d91000269b5000238
:10a990008dae0002ca430d02f4370d02f82f0d02ee
:10a9a0009c2f0d0258d300105cd300108d4b000279
:10a9b000dd4b000210b500232024144accb01e2029
:10a9c000134900920aaacde90a43f7f741fb002395
:10a9d0004ff4837219460aa8b1f09ffd00234ff48b
:10a9e00083711a460aa8fff7c5fa00284ff0000342
:10a9f00009da084a019000923220054902aacde9fd
:10aa00000243f7f725fb4cb010bd00bff2430d0227
:10aa1000f4370d0208440d02014b5868704700bf1f
:10aa20001cd3001010b50a4b5c6884420bd950242b
:10aa30001b6804fb003009b1431d0b602ab1037988
:10aa40000020136010bd0348fce71046fae700bf82
:10aa50001cd30010defeffff014b5868704700bf9b
:10aa600028d30010074b5a68824208d929b14c22da
:10aa70001b6802fb00300830086000207047024865
:10aa8000704700bf28d30010defeffff10b5044c56
:10aa9000236813b90af020ff2060206810bd00bfb2
:10aaa00060d30010f8b50b4b0546d3e900465023a0
:10aab00003fb0646b442274609d0601d40222946c2
:10aac000b3f060fb50340028f4d13846f8bd0027bd
:10aad000fbe700bf1cd300102de9f0410f461646de
:10aae0001c46beb005464c22002103a8b1f015fd5e
:10aaf00002978df80c6034b16368149323880b2b94
:10ab000084bfa36815932846f6f75cf940280246ef
:10ab1000294628bf40220df10d00b1f0d7fc284690
:10ab2000fff7c0ff044638b1502202a9b1f0cefcb5
:10ab300020463eb0bde8f081254d6e68632e41d8b9
:10ab4000502402a9224616a8b1f0c0fc224616a93c
:10ab50002aa8b1f0bbfcab689e4215db06fb0441a2
:10ab60002868b2f05bfc771c044658b92023cde975
:10ab70002a30184b00933220234617492aaaf7f7a8
:10ab800067fad5e72860af604ff050086a6808fba5
:10ab900006f608fb02f22f68921b3744394607eb92
:10aba0000800b1f0a0fc424638462aa9b1f08efc5c
:10abb0006c6801346c6008fb04f4a4f150002c684c
:10abc0000444b5e72023cde92a30044bd2e700bf87
:10abd0001cd30010b72c0d02f4370d0220440d02d7
:10abe000f8b50b4b0546d3e900464c2303fb06465c
:10abf000b44227460ad004f1080040222946b3f0a7
:10ac0000c1fa4c340028f3d13846f8bd0027fbe7e1
:10ac100028d300102de9f0410d460446bcb0442273
:10ac2000002105a8b1f079fcab6820460493eb68dd
:10ac30000393f6f7c7f840280246214628bf402272
:10ac400005a8b1f043fc2046fff7caff044638b11f
:10ac50004c2203a9b1f03afc20463cb0bde8f0819b
:10ac6000254d6e68632e41d84c2403a9224616a8b0
:10ac7000b1f02cfc224616a929a8b1f027fcab683c
:10ac80009e4215db06fb04412868b2f0c7fb771c27
:10ac9000044658b92023cde92930184b00933220bf
:10aca0002346174929aaf7f7d3f9d5e72860af60fb
:10acb0004ff04c086a6808fb06f608fb02f22f68a2
:10acc000921b3744394607eb0800b1f00cfc4246b2
:10acd000384629a9b1f0fafb6c6801346c6008fbb6
:10ace00004f4a4f14c002c680444b5e72023cde91a
:10acf0002930044bd2e700bf28d30010b72c0d0237
:10ad0000f4370d0239440d0210b588b00446684688
:10ad100009f00dfc694604a809f054fc04a8a047fa
:10ad2000044604a809f0b8fb684609f0b5fb2046c4
:10ad300008b010bd10b50446f6f744f801462046a9
:10ad4000bde8104011f07cb870b5094b0025d3e97f
:10ad500000464c2303fb0646a64206d004f1080039
:10ad6000fff7e8ff4c340544f6e7284670bd00bf06
:10ad700028d30010f8b50b4b0026d3e90047502329
:10ad800003fb0747a7420bd0601dfff7d3ff01214c
:10ad90000546201d11f054f8284406445034f1e7cc
:10ada0003046f8bd1cd3001007b5fff7e3ff009055
:10adb000fff7caff08210190684611f041f803b07f
:10adc0005df804fb10b50c46fff7eeffd4f8e03059
:10add000c4f8d40043f00203c4f8e03010bd70b5ed
:10ade000142486b02246002101a8b1f096fb7826f3
:10adf000adf8044000240022012101a81ff085facb
:10ae0000bdf80650bdf80c30a34209dd02982021a0
:10ae100006fb04004c3011f013f801340544f1e74f
:10ae2000002201a811461ff070fa284606b070bd36
:10ae300010b50c46fff7d3ffd4f8e030c4f8d800c3
:10ae400043f00103c4f8e03010bd38b5846805460e
:10ae50005cb144684cb12046f5f7b4ff402808d8ef
:10ae600020462946fff7d6fe0446201e18bf0120c3
:10ae700038bd0024f9e710b410461a46d1e9103461
:10ae800024b1014620465df8044b184711465df891
:10ae9000044b18471b681268fff7edbf07b5016840
:10aea0000a468b6a32f8080b009301f118034968cf
:10aeb000fff7f0ff03b05df804fb30b5c3b04ff40b
:10aec0008372002104466846b1f027fb00234ff44b
:10aed00083711a466846fff76ff8b0f5837f12d189
:10aee000bdf80050b5f5837f0dd1a3680bb9b0f064
:10aef0006dfd69462046e3689847002329461a46b7
:10af00006846fff737f843b030bd000003291fb58e
:10af100015d128b101280ed0002005b05df804fb42
:10af20002d4b03932d4b68460293fff7c6ff6846ef
:10af3000f7f796fff0e72a4b03932a4bf3e7022932
:10af400032d102380628e7d801a353f820f000bf19
:10af5000edae0002f7ae000299ae000201af0002b2
:10af60000baf000215af00021faf00021e4b009294
:10af700003931e4bd7e71e4b009203931d4bd2e762
:10af80001d4b009203931d4bcde71d4b0092039385
:10af90001c4bc8e71c4b009203931c4bc3e71c4b94
:10afa000009203931b4bbee701290cd130b101285d
:10afb000b2d105b05df804ebfff711bf05b05df845
:10afc00004ebfff7f1be0429a6d10428a4d1124b4b
:10afd0000393124ba7e700bf45ad00021da400027a
:10afe000b1ad000213a40002679e0002ffa300029d
:10aff0007b9e0002eba300028f9e0002d7a30002fb
:10b00000a39e0002c3a30002b79e0002afa30002ea
:10b01000cb9e00029ba30002df9e000291a30002d0
:10b020002de9f04302291646984691b03dd10a46d3
:10b0300001461f48b1f03afa0446002835d11c25d4
:10b0400001a8faf72bfc2a46214609a8039fb1f074
:10b0500064fa214609a8adf82450fdf739fd9df8a2
:10b060002b20144905a809f0ddfaddf81c9007eb48
:10b070000905a84513d93a4601993046b1f026fa98
:10b080004a460599f019b1f021fa05a809f004fa29
:10b0900001a809f001fa284611b0bde8f08305a81f
:10b0a00009f0faf901a809f0f7f90025f3e700bf64
:10b0b000bd490d0252440d020138c0b208289abfa2
:10b0c000014b185c02207047c4470d02042906d0ca
:10b0d000092907d0012914bf04200120704718b1a5
:10b0e000f5f770be082070477047000010b5184b88
:10b0f0008cb01b7803f0ff001bb1164b1c7814b109
:10b1000001200cb010bd1ef014fc134b1b78002b5b
:10b11000f6d043f69821114a1368c31a8b42efd92f
:10b120002023cde9043413680d49cde901030d4b0b
:10b130002820009304aa2346f6f78aff20462346d8
:10b1400022462146009403f093ff2046d9e700bf32
:10b150005ecc001074d900105bcc001074d20010cb
:10b16000f4370d0257440d0208b5fff78ffc054b6d
:10b1700018680af029f818b9bde80840fff7baba0c
:10b1800008bd00bf60d3001008b50120f8f7eef944
:10b190000920f8f7ebf9002008bd00002de9f04385
:10b1a00000244ff02008b14bb1b01c70b04bb14e31
:10b1b00020ad2a46b04901900093074623461e2041
:10b1c000cde92084f6f744ff2146306809f0efff0f
:10b1d0000d28034657d12346032240200021cde904
:10b1e00001440094fbf72efba44ba3492a461e20e2
:10b1f00000932346cde92084f6f72afffff794f960
:10b20000fff7c2ff20461ef0c7fc014628b9faf737
:10b21000b1fa0146002800f0e58001f029fd01287f
:10b2200040f00081964b1b78002b40f0fb80954b43
:10b230001868b0b101230a22294609f02cfa00242b
:10b240002023cde91034904b1e208b49009310aa87
:10b2500023460195f6f7fcfe224629468b48fff768
:10b2600058f900220823306810a9cde91022adf862
:10b2700040300af072f90446002800f0dd8009f041
:10b2800029ff0446d4e020b131b0bde8f04309f015
:10b2900021bf02220021cde9010000900df14009fb
:10b2a0004020fbf7cffa402148461ff028fb044618
:10b2b000b0b99df84030013bdbb2fd2b10d8744b88
:10b2c0002a46cde920806c490093cdf804900346ce
:10b2d0001e20f6f7bdfe224649466e48fff719f9d3
:10b2e000002340224946184600931af00bf9044601
:10b2f00090b99df840307bb12023cde92030664bda
:10b300002a465d49009303461e20f6f7a1fe224619
:10b3100049466248fff7fdf8fff706f900220620cc
:10b320000df117018df81720f8f700f904460028f1
:10b3300052d19df81730002b4ed002460146062010
:10b34000f8f7dcf8224607a906a8cde9064410f074
:10b350006bfd002840d1ddf81880b8f1000f3bd01c
:10b360005ffa88f3502b079c7bd047d8282b7bd0e3
:10b370003cd8142b00f0b2801e2b00f0b1800a2bb9
:10b3800000f0b0804346464a40212846b2f0fcf81f
:10b39000b8f1820f01460ed1631edbb20c2b28449c
:10b3a000c1f140013bd83f4a52f82330002b36d040
:10b3b0003d4ab2f0e9f800242023cde908343b4ba4
:10b3c0001e202d49009308aa2346f6f741fe224687
:10b3d00029463748fff79df8fff7d6fe0fb1f9f77a
:10b3e0006efc002130680af001f816e73c2b7bd098
:10b3f000462b7bd0322bc5d12e4b33e0782b77d028
:10b4000007d8642b76d06e2b76d05a2bbad12a4b24
:10b4100028e0822b72d08c2bb4d1284b22e023461b
:10b42000274ac6e7fff704f9044600283ff4ffaeb9
:10b43000204631b0bde8f083119b012013f0010fcd
:10b440000cd0204b2a4618702023cde920341e4b07
:10b45000094900932346f6f7fbfde9e71b4b1870fb
:10b46000e6e71b4b1b4a8fe71b4bfbe770cd001039
:10b4700005450d0260d30010f4370d022e450d0274
:10b480000cd5001058d3001011460d0236460d029f
:10b4900055450d0284450d029c450d02bc450d022b
:10b4a00082440d0290470d02d1450d02d6450d0292
:10b4b000f9450d02a2440d02f1440d0200450d02b2
:10b4c00080440d025dcc00104d460d025ccc001096
:10b4d000e4440d02d3450d02d9440d02084bc1e7e7
:10b4e000084bbfe7084bbde7084bbbe7084bb9e784
:10b4f000084bb7e7084bb5e7084bb3e7084bb1e794
:10b5000085440d02bf440d0208930d02d0440d0284
:10b51000be610d0299440d02b1440d028f440d022b
:10b52000b4290d02024b0021186809f042be00bf89
:10b5300060d3001010b5104b8ab01b78bbb1fff779
:10b54000f1ff044698b92023cde902300b4b0c499a
:10b55000009302aa03462820f6f77afd23462246e6
:10b5600001212046009403f083fd0ab010bd1ef0b7
:10b57000e0f9044b1860f8e75ecc001096460d0227
:10b58000f4370d0274d20010f8b50c461646114976
:10b59000054608f0ccff2644a64219d0274623785a
:10b5a00028461b0903f13001392988bf03f15701ef
:10b5b00009f02af83b78284603f00f0303f1300125
:10b5c000392988bf03f15701013409f01df8e3e779
:10b5d0002846f8bdaf2c0e020048704778d2001004
:10b5e0000048704704d30010f0b50c461d46096ca6
:10b5f0003d4ba5b0994206462a9f08d12b462146cd
:10b6000030462a9725b0bde8f040fff734bc002053
:10b61000019201f039fb019a0028efd0114602a8ef
:10b6200008f085ff294606a808f081ff2f4b93f804
:10b630002c203ab906a808f02fff02a808f02cff2a
:10b6400025b0f0bd586a24f092f805460028f1d1e3
:10b6500002a910a80f94adf8386008f0b3ff06a94e
:10b6600014a808f0afffbdf8383010a9adf8643069
:10b670000f9b1ba81a93189708f0a4ff14a91fa8e2
:10b6800008f0a0ff189b2c2023930c951af06cfa5d
:10b69000044680b1bdf864301ba903801a9b0830b2
:10b6a00040f8043c08f074ff1fa904f1180008f0ea
:10b6b0006fff239ba3620e4b1fa80d930d4b0a94a3
:10b6c0000c9308f0e9fe1ba808f0e6fe0aa907485b
:10b6d000f8f766fe0aa8f7f7c3fb14a808f0dcfe2b
:10b6e00010a808f0d9fea5e75da000028cd40010d8
:10b6f0001dae000227a400022de9f0431f46194b9e
:10b70000164693f82c2085b00446dde90c890d46d9
:10b71000eab1586a24f02bf8c8b9029018201af040
:10b7200023fa28b1c0e90045c0e90267c0e90489ed
:10b730000d4b694603930d4b00900a480293f8f7ae
:10b740002ffe6846f7f78cfb05b0bde8f0833b465b
:10b75000324629462046c446cdf8309005b0bde8b3
:10b76000f04360479ccd0010f1b600024da30002eb
:10b7700007b500684369019303690093d0e9022388
:10b78000d0e90001fff7b8ff03b05df804fb00004b
:10b790002de9f041304b174693f82c2004460e4615
:10b7a00088b0d2b1586a23f0e2ffb0b906900c20fd
:10b7b0001af0daf910b1c0e900468760274b04900f
:10b7c0000793274b244804a90693f8f7e9fd04a83a
:10b7d000f7f746fb08b0bde8f0810023cde903335d
:10b7e000e36c25688bb1284603aa04a99847002872
:10b7f00025da00231e201a461946cde90067fff717
:10b800007bff0498b0f03cfee4e7d4f84880b8f140
:10b81000000f04d02a462179601dc04705462846fe
:10b820002179fff753fc8046039040b1b0f020fe31
:10b8300004900028ddd042462946b0f047fe20792a
:10b84000fff73afcdde903320146cde9006700204d
:10b85000fff752ffbee700bf8cd40010e5b700022f
:10b860000da3000203681868d3e90112fff790bf27
:10b8700037b50c461546fff715f9034630b12a4691
:10b88000214603b0bde83040fff782bf02460146c3
:10b8900000951d20a04703b030bd38b5002383605c
:10b8a0008b6804460d462bb102229847eb68e36093
:10b8b000ab68a360204638bd012a70b5054603d1a8
:10b8c0000b680360002070bd022a0dd0032af9d155
:10b8d0000468002cf6d004f10800f7f7c1fa18212b
:10b8e00020461af049f9ede718200e681af03cf9e5
:10b8f000044648b1336806f10801036073680830f4
:10b9000040f8043cfff7c9ff2c60dbe7012a70b563
:10b91000044603d10b680360002070bd022a0cd0de
:10b92000032af9d10468002cf6d02046f7f798fadc
:10b93000142120461af020f9eee714200e681af0c0
:10b9400013f9054620b13146fff7a7ff33692b6194
:10b950002560e1e713b56c460b460246d0e90001cd
:10b9600084e8030093e8030082e8030094e80300fe
:10b9700083e8030002b010bdf0b517461c46002254
:10b9800043688fb000680d469847064627b11db141
:10b99000012128461af0f0f8264b93f82c20002ab3
:10b9a00039d0586a23f0e3fe0546002833d12146fa
:10b9b00004a8fff772ff04a909a80896fff76dff16
:10b9c000089b14200d9302951af0cef8044670b12e
:10b9d0000146856009a8fff7bdff0b9ba268a36025
:10b9e0000c9b0b92e268e3600d9b0c922361124b5f
:10b9f00009a80393114b00940293f7f731fa6946b3
:10ba00000c48f8f7cdfc6846f7f72afa04a8f7f7d0
:10ba100027fa0fb0f0bd02238df81030a368099605
:10ba20000bb9aff0d3ff2046e36804aa09a99847f1
:10ba3000efe700bf9ccd001089a500028db8000281
:10ba400030b5016885b0d1e9004568460831fff797
:10ba500024ff6b46012229462046fff78dff6846ea
:10ba6000f7f7fef905b030bdf0b591b00d461746b9
:10ba7000fff7b6f80446002855d02846b1f02cfe52
:10ba80002a4b064693f82c20002a40d0586a23f00f
:10ba90006efe054600283ad1394606a8cde904468f
:10baa000fff7fbfe049b06a90a93059b0ca80b93ca
:10bab000fff7f3fe182002951af056f8044688b1f5
:10bac0000a9b056103600b9b00f1080143600ca811
:10bad000fff740ff0e9b226923610e920f9b626964
:10bae00063610f92124b0ca80393124b00940293c4
:10baf000f7f7b6f969460d48f8f752fc6846f7f7cc
:10bb0000aff906a8f7f7acf9002011b0f0bd39463f
:10bb10000aa8fff7c2fe2046012231460aabfff712
:10bb20002bff0aa8eee74ff0ff30eee78cd40010b1
:10bb3000c1b9000239b800022de9f84300254ff0e1
:10bb400014082c4b2c4cc3e900559d602b4b0a214b
:10bb5000c3e900552a4a9d602046f7f711f8294ba2
:10bb6000294a1e2104f11c002360a561f7f708f89b
:10bb7000264bdff8c090e361254b264fc4e90f83c5
:10bb8000254b2946636404f13c0004f13803a364a7
:10bb90006563c4f83890e764f6f7d8fc1f4b204e75
:10bba000e365204b2946236604f1580004f1540351
:10bbb000c4e91937c4e91459a663c4f85880f6f7e4
:10bbc000c5fc194a0d2104f170006665e566f6f7bb
:10bbd000d7ff47f23052154bc4f888502367144bf7
:10bbe000c3e903551d705a601d725d729d82bde8e8
:10bbf000f88300bf1cd3001078d2001028d30010a7
:10bc0000c5460d0278470d02d0460d0288470d0249
:10bc10000e000200512a0002df460d021d00020044
:10bc2000e43c0d02eb460d02f9460d02f43c0d0218
:10bc300004d3001008360d0209490c2008b5aff0f6
:10bc4000c1fe014650b1074b036000238360064be1
:10bc50004360bde808400548fbf730be08bd00bfa3
:10bc60000d700f02f03d0d02f1bb00023cd9001037
:10bc700010b510b103685b689847f9f7e9fd40b16a
:10bc8000fef704ffbde81040002304211a4609f026
:10bc90004abc10bdc0e8af1f7047002108b503467d
:10bca000c0e9001101620a460830c0e8af1f03f185
:10bcb0000c00fff7efff03f11000fff7ebff03f1bc
:10bcc0001401c1e8af2f03f11801c1e8af2f012122
:10bcd00003f11c02c2e8af1f184608bd10b50a4c9c
:10bce000d4e88f3fdb070cd420461cf051f840b15c
:10bcf0000648fff7d2ff20461cf084f80448b0f055
:10bd0000bef9024810bd00bf64d3001068d3001014
:10bd1000b5bc000210b50446006818b12af0b4faa8
:10bd200000232360606818b128f0d4f80023636012
:10bd300010bd00000148fff7edbf00bf68d3001041
:10bd40000c30d0e8af0f831e584258417047103076
:10bd5000d0e8af0f831e5842584170471fb51c30c2
:10bd6000d0e8af3f022b0fd193681b78022b0bd189
:10bd700000230522cde90133009320200021faf7aa
:10bd800061fd05b05df804fbd0e8af3f002bf8d1b2
:10bd900092681278012af4d10322cde9013300938d
:10bda000ebe773b50024054601a8019427f074ff62
:10bdb000a04219db0198264603465bb15a682ab1b6
:10bdc0005278022a04d00a2a08bf01241b68f4e72b
:10bdd0000126fbe727f058ff05f11403c3e8af6f16
:10bde00005f11803c3e8af4f02b070bd002307b5db
:10bdf000084669460093adf8043029f0a8fd0222f8
:10be000068460649b2f0bef930b910f0d5fd17f01a
:10be1000b3fb03b05df804fb0120fae768480d02ac
:10be2000f7b506460c4611bb6846009129f05afb4f
:10be3000002819db2746009d9db1686878b101a9eb
:10be4000019729f086fc002809db019b1b0706d41b
:10be500030466968fff7caff002818bf04462d68fe
:10be6000eae7009829f06afb204603b0f0bd03b072
:10be7000bde8f040fff7babf2de9f0470e4688b0a5
:10be80000021fff7cdff0027002851d004a8049718
:10be900029f028fbb84204da264c204608b0bde859
:10bea000f087049d234cdff89080dff8909085b3f5
:10beb000686808b305a9059729f04bfc00281bdb2f
:10bec000059b13f0080317d1d5f804a006a9504626
:10bed0000693adf81c3029f03afd0eb156450bd152
:10bee0000222414606a8b2f04df9824630b910f060
:10bef00063fd544617f032fb2d68d8e7022249460d
:10bf000006a8b2f03ff90028f6d112f0bff80446b7
:10bf1000f2e7049829f012fb002cbed1234602223e
:10bf200010200021cde901440094faf78bfcb4e71e
:10bf30000446b2e7f2feffff68480d02f5540d0219
:10bf4000006a20b183688b4201d00068f9e770472e
:10bf5000f0b5002585b016460c468df8075031bb6c
:10bf600002a8029129f0befaa8421ddb2746029dd5
:10bf7000bdb1686898b103a9039729f0eafb0028ce
:10bf80000ddb039b1a070ad468680df107012af03c
:10bf900044fa20b99df80730b34208bf01242d6848
:10bfa000e6e7029829f0cafa204605b0f0bd20461f
:10bfb0000df107012af031fa28b99df80740a31bbb
:10bfc0005c425c41f0e72c46eee77fb500250c466d
:10bfd000019539bb02a8029129f084faa8421edb20
:10bfe0002646029dc5b16868a0b103a9039629f051
:10bff000b0fb00280edb039b13f008030ad168682e
:10c0000001a9019329f014fb20b9019b13f4801faf
:10c0100018bf01242d68e5e7029829f08ffa204621
:10c0200004b070bd204601a929f002fb18b9019c9b
:10c03000c4f30054f3e72c46f1e738b50222044676
:10c040000d46fff785ff28b129462046bde8384058
:10c05000fff7bbbf38bd38b5012204460d46fff7d8
:10c0600077ff30b129462046fff7afff80f001008f
:10c07000c0b238bd08b5fff763ff00b1007908bd55
:10c080002de9f043002485b0064602a80f4602942d
:10c0900029f028faa04224dba146029df5b1686888
:10c0a000d0b103a9cdf80c9029f053fb002813db85
:10c0b000ddf80c8018f0080f0ed169683046019148
:10c0c000fff794fe40b130460199fff7d3ff18b156
:10c0d00037ea080308bf01342d68dfe7029829f02a
:10c0e0002dfa204605b0bde8f08370b50546002660
:10c0f000046a4cb123792bb12846a168fff776fe7c
:10c1000000b101362468f4e7304670bd08b5fff78a
:10c1100017ff10b10c30d0e8af0f08bd08b5fff71e
:10c120000fff10b11030d0e8af0f08bd0a4608b5b8
:10c13000036a73b112b19968914208d103f10c00fe
:10c140000021fff7a7fd03f11000fff7a3fd1b6817
:10c15000efe708bdd0e8af0f704708b50830fff72c
:10c16000f9ff013818bf012008bd08b50830fff7f6
:10c17000f1ff043802288cbf0020012008bd08b55b
:10c180000830fff7e7ffc31f5842584108bd2de9ab
:10c19000f3410546fff7e9ff58b14ff00008684644
:10c1a000cdf8008029f09ef9002808da02b0bde839
:10c1b000f0812846fff7e3ff0028eed1f6e7009c68
:10c1c0007cb3606820b301a9cdf8048029f0c1fade
:10c1d00000281ddb019f3b071ad4666828463146bc
:10c1e000fff704fea0b131462846fff7a9fe78b15b
:10c1f000037907f001076bb157b90121304629f0e7
:10c2000001fb002804db4ff48031304629f053fb5a
:10c210002468d5e7002ffbd00121304629f01ffb11
:10c22000f6e7009829f08af92046bfe708b50830fc
:10c23000fff790ff08bd0000f0b500f108050446c7
:10c240008db028460e46fff785ff072813d1072e2d
:10c2500000f0e580002104f10c00fff71bfd04f164
:10c260001000fff717fd04f11402c2e8af1f04f13c
:10c270001802c2e8af1f731e062b1ed8dfe803f0ba
:10c280000439698793c8cf00002704f11c03c3e871
:10c29000af7f2a213b463a463846f9f78dff3b46a9
:10c2a000022200212020cde901770097faf7cafa8f
:10c2b000faf7a6fc00f118031f6020230027284688
:10c2c000cde90437fff746ff634b644953f8262056
:10c2d00053f8203002920193614b1e20009304aa70
:10c2e0003b46f5f7b5fe04f10803c3e8af6f0db0a8
:10c2f000f0bd00232a211a460120f9f75dfffaf765
:10c300007ffc022200f118031a602846fff722ff83
:10c3100003280ed1072204f11c03c3e8af2f00232a
:10c320000b22cde90133009320200021faf78afa8d
:10c33000c3e72846fff70eff0128bed1022204f111
:10c340001c03c3e8af2f00230422cde9013300937f
:10c35000eae7062204f11c03c3e8af2f2846fff7e3
:10c36000f9fe072803d1faf74bfc0023c36600232c
:10c370000a22cde90133009320200021faf762fa66
:10c38000faf73efc052200f118031a6095e7002336
:10c390002a211a460220f9f70ffffaf731fc03228f
:10c3a00000f11803f1e7042204f11c03c3e8af2fe6
:10c3b0002846fff7cffe07280fd1faf721fc01220c
:10c3c00000f134031a60faf71bfc07460ff042fb3a
:10c3d0003b6d01333b650ff041fb00232a211a46d8
:10c3e0000220f9f7e9fe00230622cde9013300938c
:10c3f00000212020faf726fafaf702fc032200f1c6
:10c4000018031a60faf7fcfbc36e0133c36654e7e6
:10c4100000232a211a460320f9f7cefe4de7052214
:10c4200004f11c03c3e8af2f00232a211a4604207d
:10c43000f9f7c2fefaf7e4fb042200f118031a60d0
:10c440002846fff787fe07283ff437af002307226f
:10c45000cde90133009367e78c490d026b480d026b
:10c4600075480d0210b50368044623b90146084813
:10c4700029f0fafe2060636823b92146054827f0b9
:10c4800013fd60602046bde810400121fff7d4bed7
:10c4900075c9000269c7000210b504460830fff7ed
:10c4a00059fe012803d102212046fff7c5fe6ff097
:10c4b000d10010bd10b504460830fff74bfe01282f
:10c4c00008d0022803d101212046fff7b5fe6ff006
:10c4d000d10000e0002010bd2de9f74307460830e9
:10c4e000fff738fe02284bd1002504213846fff71c
:10c4f000a3fe6846009528f0f5ff041e37db2c46a6
:10c50000a946ddf80080b8f1000f2bd0d8f8040060
:10c5100028b301a9cdf8049029f01bf900281edbef
:10c52000019e32071bd4d8f8045038462946fff73d
:10c530005dfca0b129463846fff79cfd78b1f307b2
:10c540000dd40121284629f05df9002807db4ff4be
:10c550008031284629f0aff90028a8bf0134d8f867
:10c560000080d0e7009828f0e9ff24b14446204637
:10c5700003b0bde8f08305213846fff75dfef6e71e
:10c580006ff0d104f3e7f7b5054608300c46fff726
:10c59000e1fd0138012846d92846fff7f0fd88b1b2
:10c5a000faf72efb06466cb100f134031c60012c37
:10c5b00001d0062c06d10ff04dfa336d01333365ef
:10c5c0000ff04cfa002703212846fff735fe684696
:10c5d000009728f087ff041e1ddb3c46009eaeb18d
:10c5e000706888b101a9019729f0b3f800280bdb26
:10c5f000019b1a0708d4db0706d50121706829f0d2
:10c600002ef90028a8bf01343668e8e7009828f022
:10c6100095ff1cb13446204603b0f0bd02212846e8
:10c62000fff70afef7e76ff0d104f4e710b593685f
:10c6300004461b78083093b1fff78cfd04281ad10b
:10c6400005212046fff7f8fd40212046fff718fda1
:10c6500088b106212046bde81040fff7edbdfff789
:10c6600079fd032807d101212046fff709fd0128a4
:10c6700001d80221eee710bd2de9f3470027002184
:10c680000646fff753fd6846009729f08bfdb84238
:10c69000c0f28580b846ddf80090b9f1000f56d0a1
:10c6a000d9f8083013f0080434d103f04103412bca
:10c6b00030d1d9f80c306bb3196859b34d78022dcd
:10c6c0002bd11a7c002a3fd09b68002b3ad0a8457a
:10c6d000b8bfa84699f81000a74201a9b8bf2746dd
:10c6e00028f072ffb0b930460199fff729fc0346e4
:10c6f00080b10c30d0e8af2f954202dd2946fff71c
:10c70000c9fa03f11000d0e8af3f9c4202dd214698
:10c71000fff7c0fad9f80090bfe70a2d15d1da6803
:10c720001c7c8b6943b984b172b1147814f0020493
:10c730000bd002240025cae73cb12ab11478c4f317
:10c740004004f7e71c46f5e700242546bfe70098bc
:10c7500029f03bfb06f10c0adae8af9f06f1100462
:10c76000d4e8af5f3046fff71cfb41465046fff769
:10c7700091fa39462046fff78dfab8f1020f11d031
:10c78000022f16d0002406f1080a5046fff7e2fcfb
:10c79000072816d1acb906213046fff74dfd02b08f
:10c7a000bde8f08706f11403d3e8af4f012ce7d1c1
:10c7b000e9e706f11803d3e8af4f631e5c425c4122
:10c7c000e1e75046fff7c6fc062800d154b95046b1
:10c7d000fff7c0fc0728e2d1002ce0d0c84501d10a
:10c7e000af42dcd00721d7e7fff746bf38b59368e3
:10c7f00004461b7800f10805d3b12846fff7aafcd0
:10c80000052807d106212046fff716fd2046fff731
:10c8100033ff09e02846fff79dfc0728f6d028469d
:10c82000fff798fc0628f1d0bde83840fff704babe
:10c83000fff77cfc2846fff78dfc07280ad1412131
:10c840002046fff71dfc0028e0d105212046fff718
:10c85000f3fce9e72846fff77dfc0628e4d1eee784
:10c8600038b500f1080504462846fff773fc072891
:10c8700006d12046fff700ffbde83840fff7dcb9de
:10c880002846fff767fc0628f6d1f2e7d0e88f0fbd
:10c89000c0b2704770b58cb0fff752fb0e4604462d
:10c8a00070b92023cde90430254b2649009304aa12
:10c8b00003463220f5f7ccfb6ff0a9000cb070bd39
:10c8c00000f114051ab3022328468df80c30fff747
:10c8d000ddff022807d02846fff7d8ff042802d042
:10c8e0000422c5e88f2f20210023cde90413164a26
:10c8f0000092012004aa1349f5f7aafb0023009334
:10c9000001233046194603aa29f0f0fcd6e701239b
:10c9100028468df80c30fff7b9ff012809d02846ca
:10c92000fff7b4ff032804d0032204f11403c3e883
:10c930008f2f20220023cde90423044ad8e700bf2b
:10c940008d480d026b480d02a8480d02ca480d0221
:10c95000f0b58fb00d461646fff7f2fa60b9202306
:10c96000cde90630164b1749009306aa034632203c
:10c97000f5f76efb0fb0f0bd00f114073846fff776
:10c9800085ffb3681b789842f4d0c7e88f3f0df15c
:10c990001701284628f0bffe202200239df817101b
:10c9a000cde90623d7e88f2fd2b2cde90112064a8e
:10c9b00001200092034906aaf5f74afbdae700bf17
:10c9c0008d480d026b480d02ed480d021368033bc4
:10c9d000052b0ed8dfe803f00305070d090bfff761
:10c9e00025befff703bffff73bbffff7b1bffff760
:10c9f000b5b97047fff7eabf00232de9f04f93b0b8
:10ca0000054608a80591089328f06cfd00285fdb17
:10ca1000089cdff8c8a0dff8c8b0002c55d06068cb
:10ca2000002850d0002309a9099328f092fe00287d
:10ca300049db099b13f0080845d166682846314652
:10ca4000fff77efa074680b959461820aef0baffc4
:10ca50000746002837d02b6ac0e9038880f8048095
:10ca600080f81480866003602862059b30463b7125
:10ca700000230df11e018df81e3029f0cefc8146f9
:10ca800008bb07f114084046fff700ff9df81e1091
:10ca9000884218d0c8e88f1f0df11f01304628f0da
:10caa0003afe20229df81f10cde90a29d8e88f2fe1
:10cab000094bd2b2cde90112009351464b460120f9
:10cac0000aaaf5f7c5fa2468a7e7089828f036fd02
:10cad00013b0bde8f08f00bf12490d026b480d0284
:10cae0000d700f0210b521b90121fff785ff00205d
:10caf00010bdfff725fa10b101230371f7e76ff0be
:10cb0000a900f5e770b505460c461646faf778f821
:10cb100000f134031e60214628461cb9fff76cff64
:10cb2000204670bdfff70cfa10b100240471f7e73e
:10cb30006ff0a900f5e7f7b5174613f001020546b7
:10cb40000e461c4605d10b4601200521009202f03d
:10cb50008ffa032d0ad0042d0cd0022d0dd1c4f371
:10cb600040000ff007f9002003b0f0bd00200ff0e7
:10cb7000e9f8f8e70ff0d4f8f5e700223946304637
:10cb80000ff0c0f8efe700680179d0e902230078e0
:10cb9000fff7d1bf012a70b5054603d10b680360ca
:10cba000002070bd022a08d0032af9d100680028ad
:10cbb000f6d0102118f0e0fff2e710200e6818f010
:10cbc000d3ff044618b196e80f0084e80f002c60ec
:10cbd000e6e7000010b5012400220d4b1c700d4b40
:10cbe0001a70fef7fdfcd0e8cf3fc0e8424f002aa4
:10cbf000f9d1dbb2002bf6d1c2680361c3600375c3
:10cc00004375c0e88f3fd30758bf037a10bd00bffc
:10cc10007151001012d100100022014b1a707047a0
:10cc200071510010024b1878003818bf012070476e
:10cc3000715100100b4b28b91a788ab901221a7069
:10cc4000fff7c8bf0328187008d80128f8d00022c1
:10cc5000054b1a700122054b1a7001e00428efd031
:10cc6000704700bf8dd300107151001012d1001019
:10cc7000014b1878704700bf8dd30010014b18701e
:10cc8000704700bf8cd30010014b1878704700bf6d
:10cc90008cd30010f0b51c46431e032b06460d46f0
:10cca000174685b04fd8294ad35c002908bf1d46d6
:10ccb000274b5b68c3f308035bb144f00104e9b29e
:10ccc00023463a46f0b2fff736ff0025284605b066
:10ccd000f0bdf8f7bdfd0028efd0fef781fc037a28
:10cce000002bead0e307ead41a4b93f82c20002a51
:10ccf000e5d0586a22f03bfd0028e0d102901020d8
:10cd000018f032ff18b1c0e90065c0e90274124b97
:10cd100000900393114b69460e480293f6f7a4f96d
:10cd2000044670b100224ff0ff31406922f038fe16
:10cd3000236820469b68a56998476846f6f790f8ef
:10cd4000c4e70546f9e7064dc0e700bfac490d0250
:10cd500000ed00e09ccd001007cb000215cb0002d7
:10cd6000f2feffff10b503681446db689847031b0b
:10cd70005842584110bd08b54068fff7f3ff08bda1
:10cd800070b5037a04460d4616462bb9d0e9031256
:10cd9000fff7f1ff01232372324629462046fff7b1
:10cda000eaff70bd704770470139012908b505d801
:10cdb00000210830f6f712fc012008bd0020fce736
:10cdc000002201211046faf7d9bb10b50446fff73f
:10cdd000e9ff20461c2118f0cffe204610bd08b503
:10cde0000021022002f0e0fbbde8084022f0a8bdcf
:10cdf000002108b5022002f0d7fb22f0a8fdb0fa0e
:10ce000080f0400908bd08b50021022002f0ccfbeb
:10ce1000bde8084022f0a3bd38b500f1080504467e
:10ce20002846fff7e5ffe8b1284606f05efdb0b101
:10ce3000284606f04bfd011e11db236820465b6986
:10ce4000c9b2984758b9284606f04ffd38b1284670
:10ce500006f034fd2368c1b21b6920469847284676
:10ce6000fff7d1ff38bd000010b50446d0e9051228
:10ce7000024b0360fff784ff204610bd404b0d02bc
:10ce800038b50c46054601462046aff01ffb284644
:10ce90001349f3f78dff28b912492046b0f003fc7f
:10cea000002038bd28461049f3f782ff08b90f4922
:10ceb000f3e728460e49f3f77bff08b90d49ece785
:10cec00028460d49f3f774ff08b90c49e5e72846f1
:10ced0000b49f3f76dff0028e2d10a49dde700bff7
:10cee000b0490d02b5490d02ba490d02c0490d0203
:10cef000dc460d02c6490d02d4490d02d7490d0288
:10cf0000e5490d02ec490d0238b504460b4b0546c8
:10cf100044f8083b204606f02ffdfff760ff20464f
:10cf2000fff771ff204606f01bfd20b94ff41651a4
:10cf3000204606f011fd284638bd00bf4c4b0d02bf
:10cf400070b50d46002400f108062846f3f73affb5
:10cf5000a04205d9295d304606f0cefc0134f4e745
:10cf600070bd000038b5044600f1080528460023ce
:10cf700007f0e6f820460649fff7e2ff284606f0ec
:10cf8000b4fc002803dd284606f098fcf6e738bd1f
:10cf90002b6c0e022de9f04369290446a5b070d12f
:10cfa000142500212a4607a8aff0b7fa0022012174
:10cfb00007a8adf81c500ff0fbfb00252023cde99e
:10cfc0000c35bdf82c30012001938f4b8f49009315
:10cfd0000caa2b46f5f73cf8bdf82c30002b3fd0bf
:10cfe0008b492046fff7acff03a8f8f757fc204613
:10cff0000399fff7a5ff20468649fff7a1ff2427e5
:10d00000dff85482dff80c92bdf82c30ab421cdd07
:10d0100007fb05f60a9b142298590ca9fff730ff6d
:10d0200088b920460ca9fff78bff41462046fff741
:10d0300087ff0a99204631440431fff781ff4946b2
:10d040002046fff77dff0135dee703a807f024fa4d
:10d05000002207a811460ff0abfb25b0bde8f08316
:10d060006d492046fff76cff0ca8f8f717fc204627
:10d070000c99fff765ff20466649fff761ff0ca892
:10d08000e4e76d293ed16549fff75aff5d22002193
:10d090000ca8aff042fa002205201146f9f7c2ffb2
:10d0a000014638b102882ab15d2a28bf5d220ca84a
:10d0b000aff00cfa01220df1870107a8fef764fa20
:10d0c00020460799fff73cff07a807f0e5f905257b
:10d0d000534f0df18d0639462046fff731ff0122ef
:10d0e000711b07a8fef750fa20460799fff728ffa3
:10d0f00007a807f0d1f9013dedd120464549fff7da
:10d100001fffaae766290bd108342046454907f0de
:10d110008bf80021204625b0bde8f043f6f75eba53
:10d12000782905d10368db6825b0bde8f0431847ce
:10d13000732916d13c4b00220c933c4b08340f93bf
:10d14000012310933a4b0ca91193032339480d94f2
:10d150008df838201293fbf793ff0ca8fff784fe9d
:10d160007be7762908d1344b0c9300f108030ca817
:10d170000d93fbf7a7ffc0e74c290ad1002201213c
:10d180000420f6f7bbf9002025b0bde8f04307f016
:10d19000d8ba632910d100201df0c3fb05462749ea
:10d1a0002046fff7cdfe2649264b002d08bf194625
:10d1b0002046fff7c5fea0e7432917d12249fff714
:10d1c000bffe3f2220460ca9fff7ccfe0ca8f3f7c8
:10d1d000f9fd3f2808d10ca81df064fb1b4920462f
:10d1e000fff7aefe0ca9e3e71949e1e764297ff4f4
:10d1f00034af002200f10803009311461046154b8e
:10d200000192fbf767ff78e7064a0d02f4370d023b
:10d21000264a0d022b6c0e02324a0d02454a0d02bf
:10d2200032370d02624a0d02404b0d02b0650d020d
:10d23000a24a0d0239400002344b0d02a64a0d02eb
:10d24000ff490d02034a0d02b74a0d02d34a0d02ef
:10d25000e74a0d02e5cc00022f4a0d024ff0ff30e5
:10d260007047d0e88f0fc0b2003818bf0120704758
:10d270000048704790d3001008b5fff7f2ff08bdd3
:10d280007fb50546fff7edffe0b1686810b10368b0
:10d290009b6898471cf04dfbeb68c01ab0f57a7f8d
:10d2a0000ed31cf046fb00240646aa682346821ac9
:10d2b00000210420cde901440094f9f7c3faee609f
:10d2c000002001e06ff0d10004b070bd38b514202b
:10d2d0000d460021144602f03ff9014640b1054bce
:10d2e0000573046143600448faf7e8fa002038bd8a
:10d2f0000248fce7a5d400023cd90010fcfeffff69
:10d3000030b58bb0fff7adff002857d000242023a5
:10d31000cde902342b4b1e202b49009302aa234651
:10d32000f4f796fe21460920f8f7faff08b30469de
:10d33000002214210120f8f7fdff282202210346d4
:10d34000cde9002102a82146012207f01dfa0022a2
:10d35000012103a8f4f760ff1a24013c0bd09df8cb
:10d360001a30322083f002038df81a3019f031fba5
:10d37000f3e7ff24dce7fef7b1fc2146fef77cfd76
:10d380000446a8b14ff47f031a2507939df81a307d
:10d3900003f0fd038df81a30013d09d09df81a30d5
:10d3a000322083f002038df81a3019f012fbf3e7f4
:10d3b00002a8fdf7ddf820460bb030bd6ff0d104b8
:10d3c000f9e700bf764b0d02684b0d020368016060
:10d3d0001bb11a68184652681047704730b58db0b7
:10d3e0000546fff745fc042807d12846fff739ff1b
:10d3f000044650b16ff0d10045e009200ef0c4fda5
:10d400000028f2d06ff081003de00123c5e88f3f96
:10d410002023cde904301d4b1d49009304aa034687
:10d420001e20f4f715fe2346224604210120009415
:10d4300001f01efefef752fc0721fff7a4f8234679
:10d440002246a2210920f8f7b7fe234622460021f2
:10d450000220cde901440094f9f7f4f91cf069facf
:10d46000c5e9020000f0bef800f0befc1c2018f078
:10d470007bfb044610b104a9fff746fd281d214699
:10d48000fff7a4ff00200db030bd00bf904b0d0290
:10d49000684b0d0230b58db00546fff7e2fe48b38c
:10d4a00000242023cde90434144b04aa00931e2049
:10d4b00023461349f4f7ccfd224621460920f8f70c
:10d4c0008dfe2146281dfff781ffc5e88f4f1cf018
:10d4d00030faaa682346821a00210820cde90144c7
:10d4e0000094f9f7aff900f07df800f013f9204649
:10d4f0000db030bd6ff0d100fae700bfa84b0d02b0
:10d50000684b0d02022906d0032906d0012906d155
:10d510000021fff763bffff7bdbffff7f1be6ff05c
:10d520007700704713b5047b02690021019202f075
:10d5300025f82146019a034802b0bde81040fff7e4
:10d54000e1bf00bf90d300100022024b1a705a6056
:10d55000704700bf90d3001010b50378044613b194
:10d56000002024f0dff9204610bd00004ff0fa73d0
:10d57000194a10b5c0e90023184b00f10d02836071
:10d5800000230373164b03f1100153f8044b8b4235
:10d5900042f8044bf9d102220023426540f2626254
:10d5a000c0e90833c0e90a33c0e90c33c0e90e33df
:10d5b000c0e91733c0e91933c0e91b33036480f8ad
:10d5c0004430c0f84630c0f84a30c0f84e30a0f8b9
:10d5d0005230a0f8582010bd180028002000640028
:10d5e0003c240d0210b50a4cd4e88f3fdb070cd465
:10d5f00020461af0cdfb40b10648fff7b7ff2046a2
:10d600001af000fc0448aef03afd024810bd00bf1d
:10d61000a0d30010a4d3001099d9000290f85700ad
:10d62000704780f857107047a0f8581000207047d6
:10d6300073b5374b05461e78002e65d130468df800
:10d64000046024f041f9d5e90801012332468df840
:10d65000043024f0f4fa041e2bdbd5e90b0132462a
:10d6600024f021fb041e24db314605f1460024f0a2
:10d6700072fa041e1ddb314605f1380024f0affac2
:10d68000041e16db314695f9440024f092fa041e7c
:10d690000fdb314695f8540024f050fb041e08dbe4
:10d6a00095f8521059b13146304624f010fc90b133
:10d6b000002401a8fff750ff204602b070bd95f886
:10d6c00053306bb1084624f002fc0028f0d195f8e5
:10d6d0005430022b14d124f01afb00eae074e8e77e
:10d6e0001946184624f0f3fb50b195f85430022b3c
:10d6f000ded10120002185f8540024f01ffbece767
:10d70000002024f031fbe8e76ff0d104d4e700bf3c
:10d710007251001070b51b4e044635788cb06dbb4d
:10d7200028468df80c5024f0cff8012328468df8b8
:10d730000c3024f01bf994f8563083b1204684f85d
:10d740005650fff775ff50b12023cde904350e4b3d
:10d75000322000930d492b4604aaf4f779fc0022ed
:10d7600021460b4824f04cf901233370002303a811
:10d77000636223632366e366fff7eefe00200cb0ce
:10d7800070bd00bf72510010d14b0d02bf4b0d0296
:10d7900001d90002f0b52d4b06461d7889b0002d49
:10d7a00050d128468df8045024f08ef801232846e5
:10d7b0008df8043024f0daf8041e38db0c273388a7
:10d7c0002946adf80c30738802a8adf80e30f38806
:10d7d000adf80850adf81230b388adf80a70adf866
:10d7e000103024f0b8f9041e21db33892946adf846
:10d7f0001830738905a805950795adf81670adf832
:10d800001a3024f0ecf9041e11db2946022024f022
:10d8100095fa041e0bdb294696f90c0024f0c9f991
:10d82000041e04db284624f09ff8041e08da304664
:10d83000fff770ff01a8fff78ffe204609b0f0bd8b
:10d840002c46f7e76ff0d104f7e700bf72510010e4
:10d85000037a2bb903681b7813b94068fff75abfe6
:10d8600070470000f0b52a4b05461b7885b0002ba9
:10d870003fd190f8523013b990f85330cbb395f8ac
:10d8800055607ebb012730468df8006024f01cf8ff
:10d890000df103033046cde901358df800708df8a8
:10d8a00003608df80c6024f061f8041e24dbd5e9d8
:10d8b0000801324624f0c3f9041e1ddbd5e90b0133
:10d8c000324624f0f0f9041e16db304624f04cf802
:10d8d000041e11db01a88df80370fff7b9ff68463d
:10d8e000fff73afe95f8553083f0010385f855307f
:10d8f0005bb96ff0d10405e001a8fff7a9ff684606
:10d90000fff72afe204605b0f0bd0024fae700bf6d
:10d910007251001073b5194b06461d7855bb284649
:10d920008df8045023f0d0ff012328468df80430f1
:10d9300024f01cf8041e12dbd6e917012a4624f055
:10d940007ef9041e0bdbd6e91a012a4624f0abf956
:10d95000041e04db284624f007f8041e08da3046cb
:10d96000fff7d8fe01a8fff7f7fd204602b070bd13
:10d970002c46f7e76ff0d104f7e700bf72510010b3
:10d9800030b5144b0c461d788bb0adb90368012b34
:10d9900012d10846fff766ff80b12046fff7baffb5
:10d9a00060b12023cde902350b4b00932b4632208a
:10d9b0000a4902aaf4f74cfb0bb030bd002024f05a
:10d9c000a6f90028f8d020220023cde90223044a3a
:10d9d0000092ece772510010f74b0d02bf4b0d02a5
:10d9e0002d4c0d0210b504460068aef049fd2046ee
:10d9f00010bd10b504466830fff7f4ff04f15c0079
:10da0000fff7f0ff04f12c00fff7ecff04f120001a
:10da1000fff7e8ff204610bd0148fff7eabf00bf4f
:10da2000a4d3001003680a6802600b6043684a6868
:10da300042604b6083688a6882608b607047002315
:10da400010b50446c0e900338360fff7ebff2046c2
:10da500010bd38b50d1e0446006803ddaff0defcd6
:10da600018b938bdaef00cfd00202060a560012083
:10da7000f7e770b500260d1e0446c0e90066866013
:10da80000bddfff7e6ff40b123685a199a4203d035
:10da900003b11e700133f9e76560204670bdf8b52b
:10daa000d0e901539d4204460e460cda27686268ad
:10dab0007919521b481caef016fd01207e55636893
:10dac00001336360f8bd691cfff7c3ff0028edd187
:10dad000f8e72de9f041476883688846b91899420c
:10dae0000446154612dc266862683e443146d21b65
:10daf0007019aef0f8fc2a4641463046aef0e6fc1e
:10db0000012062682a446260bde8f081fff7a1ff4e
:10db10000028e8d1f8e7000070b5674b06461c788e
:10db200098b0002c40f0c580022104a8cde904443f
:10db3000cde90644cde90844fff7b1ff48b95f4d90
:10db400007a8fff74fff04a8fff74cff284618b0bf
:10db500070bd012104a8fff7a2ff0028efd0062125
:10db600004a8fff79cff0028e9d01122214613a842
:10db70001294aef0d2fc2246152112a823f0adff7c
:10db8000051edddb12a8f3f71df90130c1b204a8b0
:10db9000fff785ff0028d2d0092104a8fff77ffff7
:10dba0000028ccd012a8f3f70df912a9024604a858
:10dbb000fff78fff0028c2d01c23adf80430b6f861
:10dbc0005830062102a8adf806300294adf80c409a
:10dbd0001ff07afc051eb3db0b2104a8fff75fffe3
:10dbe0000028acd0ff2104a8fff759ff0028a6d0d9
:10dbf00002220df1060104a8fff76bff00289ed05a
:10dc0000022201a904a8fff764ff002897d006228a
:10dc100002a904a8fff75dff002890d0f6f722fbc9
:10dc200000f118010da802f06bfc9df84430012ba7
:10dc30002fd1112107a8fff732ff00283ff47faf53
:10dc4000072107a8fff72bff00283ff478af102229
:10dc50000da907a8fff73dff00283ff470af04a906
:10dc60000aa8fff7ecfe0aa906f15c00fff7dafe4e
:10dc70000aa8fff7b7fe07a90aa8fff7e0fe0aa95e
:10dc800006f16800fff7cefe0aa8fff7abfe0025fd
:10dc900056e7032107a8fff702ff00283ff44faf24
:10dca000032107a8fff7fbfe00283ff448af02223c
:10dcb000cee76ff0d10549e772510010fcfeffff7f
:10dcc00038b5436805468b420c4612da83689942a0
:10dcd0000adcd5e900230021134422449a420ad0e9
:10dce00003b119700133f9e7fff7b3fe0028f0d153
:10dcf00038bd0029fcdb6c60fae7000070b5394bd9
:10dd000005461e788ab0002e68d11f2101a8fff7b2
:10dd1000b0fe1f2104a8fff7acfe32461f21019878
:10dd200023f0a7ff041e50db214601a8fff7c8ff20
:10dd300032461f21049823f0d0ff041e45db214604
:10dd400004a8fff7bdff0c2331466b8705f13800af
:10dd500023f05dff041e38db314605f1440023f05b
:10dd600033ff041e31db314605f1460023f0fefe91
:10dd7000041e2adb314605f1540023f0eaff041e9d
:10dd800023db304624f007f8314685f85200304650
:10dd900024f09df801a985f8530007a8fff74ffe6e
:10dda00007a905f12000fff73dfe07a8fff71afebf
:10ddb00004a907a8fff743fe07a905f12c00fff708
:10ddc00031fe07a8fff70efe344604a8fff70afe4f
:10ddd00001a8fff707fe20460ab070bd6ff0d1041e
:10dde000f9e700bf7251001037b50024264b0546f5
:10ddf00020461c708df8044023f066fd0123204668
:10de00008df8043023f0b4fd20b10a201f4a2049c8
:10de1000f3f7e6f8002023f0a7fd041e2fdb2846c9
:10de2000fff77afe041e2adb2846fff767ff041e71
:10de300025db0123284685f85630fff76bfd041ecd
:10de40001ddb2846fff7a6fc041e18db002229462e
:10de5000104823f0bafd041e11db95f8523033b19f
:10de6000002401a8fff778fb204603b030bd95f8e9
:10de700053000028f4d123f04aff041ef0da2846ac
:10de8000fff748fcede700bf72510010576902022e
:10de9000504c0d0201d90002c0687047c26840684a
:10dea000101a704710b500200c461bf035fd4ff4da
:10deb0007a720023f2f7d8fd2060002010bd70b503
:10dec000202488b0224606460d4668460021aef062
:10ded00024fb00216846adf800400ef02df9044601
:10dee00030b96846b36998472860204608b070bdcd
:10def0006ff06300fae70000012208b5094b1a70c1
:10df0000fef7b6fe01280cd1f7f7a2fc28b9064ba4
:10df10001b7813b9054b1b781bb1bde80840fcf713
:10df200087bb08bd0cd500105dcc00105ccc001088
:10df3000fff7e2bf438c8b422cd890f82030012ba6
:10df400016d0022b11d03bbb90f82430013bdbb242
:10df500080f82430c3b1012380f820304ff4af7330
:10df600043844ff420634361704790f824203ab112
:10df7000002380f82030322343844ff47f43f2e7bc
:10df800011460430f4f748b9022380f8203040f2fb
:10df9000ee23e5e75b1a43847047012a08bf01605e
:10dfa0000020704710b50446024b0360fcf7e0fa0e
:10dfb000204610bd0c4d0d020148fff7f3bf00bf16
:10dfc000c0d4001010b50446fff7ecff204628210e
:10dfd00017f0d2fd204610bd10b50446024b036079
:10dfe000fcf7c6fa204610bd204d0d020148fff790
:10dff000f3bf00bfecd4001010b50446fff7ecfff0
:10e000002046202117f0b8fd204610bd028c0023c9
:10e010000421303021f0febb024610b508b10020cb
:10e0200010bd0146f9f7f5f80028f8d1054c238812
:10e030009bb2002bf3d01bf07cfc2388c01a80b26b
:10e04000eee700bf20d4001070b58cb02a4904a8b8
:10e0500005f0a8fb04a805f0bdffb5eec00af1ee7f
:10e0600010fa47db04a805f0b5ffb3ee047ac0ee62
:10e07000077af8fe677afdeee77a17ee905a1f4ea0
:10e08000d6e88f2f12f001021d4c1cd130460392ae
:10e0900019f07efe039ab0b114210f20f8f74af967
:10e0a0001e2202210346cde9002120460f226ff0f7
:10e0b0007f4106f069fb134b3046236019f0a2fe46
:10e0c0001148adf0dcff002210481146f4f7a4f827
:10e0d000022384f8203040f2ee2363844ff420635f
:10e0e00000220121094884f824506361f4f794f870
:10e0f0000cb070bd0025c2e794d9001018d40010f0
:10e10000c0d400100c4d0d0239df0002c4d4001041
:10e1100008b50023a2211a460c20f8f74df8012279
:10e12000024b1a70bde8084001f00aba0dd5001084
:10e1300010b5094c2378012bdab204d0022a07d09b
:10e140000023237010bd0028fcd1fff77dfff7e707
:10e15000fff7defff4e700bf28d400101fb500234f
:10e1600010490a780b70104902f0ff040b60bab135
:10e1700001220093cde901324ff4005022460021e4
:10e18000f8f760fb094b1c70094b5868c0f3080096
:10e19000003818bf012004b0bde81040fff7c8bf29
:10e1a00004b010bd30d4001034d4001028d40010b6
:10e1b00000ed00e030b51d2885b025d9b0f5fa7f17
:10e1c00004d305b0bde83040fff7c8bf104c23783a
:10e1d0000133dbb223702378042b17d81bf0a9fb83
:10e1e0004ff47a7200250b4b18600b4b1a6000231a
:10e1f00001214ff48050cde90131227800210093b4
:10e20000f8f720fb002ddcd105b030bd0125eee78d
:10e2100030d400102cd4001034d400107fb5064642
:10e220002a4de0b1002211461046f8f7f2ff284cc3
:10e2300020701bf07efb80b22880227802f0ff0362
:10e2400042b901228020cde9013200211a46009313
:10e25000f8f7f8fa00221f4b1a7004b070bd2b8833
:10e260009bb2002bf9d01bf064fb2c883246041bb8
:10e2700031463046a4b2f8f7ccff60b901230090d4
:10e28000cde901032246034600218020f8f7dafa9f
:10e290002046fff78fff41f286330022a4f6b934ff
:10e2a000a4b29c422a80d8d8094b1b78002bd4d02a
:10e2b00011461046f8f7adff00220028cdd001210d
:10e2c000104604b0bde87040f9f758b920d40010ea
:10e2d00038d4001039d40010012802d80846fff7be
:10e2e0009dbf704710b5394c2288013a92b2228006
:10e2f0002ab911461920f3f7fbff19232380344c68
:10e300002388013b9bb223801bbbfcf7effe4ff43d
:10e310007a7323802f4b1a68b2f57a7f51d300228b
:10e320001a600df0a1fb4ff6ff7017f0fdf92a4cb3
:10e3300018f0fcff2368002b47d01bf0fafa274b9c
:10e340001a682368801a98423fd9bde81040fff749
:10e3500005bf002211461046f8f75bff80b142f27c
:10e3600010700df0bcfc58b11d4b197801f0ff0284
:10e3700031b90121104619700321f8f751ffc9e79f
:10e38000002211461046f8f744ff0028c2d140f69b
:10e39000b8300df0a4fc0028bcd0124b1b7803f061
:10e3a000ff04002bb6d101f0cbf82046fff736ff73
:10e3b000204622462146f9f7e1f80120fff72eff1b
:10e3c000a8e71a6801321a60b1e710bd7451001055
:10e3d0007651001024d4001034d400102cd4001036
:10e3e00039d4001038d4001013b501200df0d8fe38
:10e3f000ff281ed0c3071cd50420fef71bfc0021fc
:10e4000000240846fef73afc224604200df10701dd
:10e410008df80740f5f78af89df807304bb1224692
:10e4200021460420f5f76af8224621462046f9f7ee
:10e43000a5f802b010bd000010b50446fef718fca8
:10e44000022801d0002010bd002cfbd1fef7eafb12
:10e450000028f7d0f7f7fcf90028f3d1024b187821
:10e46000b0fa80f04009eee712d1001030b50d4d42
:10e4700002462c7885b034b108200b4a0b49f2f7dc
:10e48000affdadf0f5fd01234ff48020cde9014350
:10e490002b70002123460094f8f7d4f92c7005b0b6
:10e4a00030bd00bfe8d4001057690202924c0d0243
:10e4b00001287fb50c463fd00a2843d1224dd5e82c
:10e4c0008f2f12f001021cd12846039219f060fc34
:10e4d000039ab0b114210220f7f72cff02221e216b
:10e4e0001a4e0346cde9001230466ff07f4106f028
:10e4f0004bf9174b2846336019f084fc1548adf0f2
:10e50000befd14f0010212d000210846f7f708ff03
:10e5100050b10369002201210c484361043004b06a
:10e52000bde87040f3f778be6ff07f43f2e7a307d2
:10e5300008d511460848f2e7084604b0bde8704027
:10e54000fff794bf04b070bd1cd40010ecd40010d1
:10e55000204d0d026ddf0002f0d4001070b50446ae
:10e5600086b0062017f0e0f8002c65d1204600f0b8
:10e5700053ff3e4b1b78002b5ad1fef753fb00286c
:10e5800056d0f7f765f9002852d1394b1b78002b8c
:10e590004ed1fef76dfb01284ad106b070bdfef7e3
:10e5a00067fefef769fe0028f7d14ce0072017f060
:10e5b000bbf8fef75dfb042801d0f2f7d9fc01237c
:10e5c0002c4e2b7096f82c303bb9fff795fc20466b
:10e5d000fff732ff0028e0d139e0706a21f0c7f878
:10e5e00005460028f1d1244b14200593234b0493b6
:10e5f00017f0bafa044690b1214b02a940f8043b47
:10e60000f6f756fe1f4b3046236001a90194f6f73a
:10e61000d8fd40b1706a10b1294621f0d5f802a8a2
:10e62000f4f71efcb9e7236820469b689847f6e795
:10e63000154b1b78002bb0d12046fff7fdfe0028bc
:10e64000abd1002cabd00a4d2b78012baed10820da
:10e6500017f06af8fef70cfb04289ed0f2f794fc42
:10e66000092006b0bde8704017f05eb812d1001066
:10e67000e9d400109ccd0010b1de00021bdf0002c7
:10e68000c8370d02dc370d025fcc00100120fff708
:10e6900065bf000030b593b026f000fff2f75cfcd8
:10e6a0000df0a2fa002000f025fa052017f03cf842
:10e6b00000232a211a461846f7f77efd2bf098fd15
:10e6c000474bda88012a04d100229a71da712bf0c3
:10e6d000abfdf4f77bfa002200242025114602202e
:10e6e000f3f7b6ff06a8f7f7d9f8069b3d49019363
:10e6f0003d4b0aaa1e2000932346cde90a54f3f7a6
:10e70000a7fc204624f00efd24f010fd2246012037
:10e710003449f3f75bfdb0b1224605a904a8cde961
:10e7200004440df081fb70b9049b63b1059acde9f7
:10e730000a50cde901322d4b2a4900930aaa03461b
:10e740000120f3f785fc17f0bffbf5f78bfdf5f71c
:10e7500073fdfff749fe1ff0bffd25481ff070ff56
:10e760000020fef791fa60b3fef782fa041f18bf8b
:10e770000124002108461bf0cfff012807d86420a0
:10e7800018f027f90022462011460df0bbfa20466a
:10e7900000f0eef9174db4b11748fff737fc1648f3
:10e7a000f9f73ef82846fff731fc002020f0ddffa6
:10e7b00068622846f9f769f806a805f06dfe13b0ff
:10e7c00030bd0446d5e7204620f0cfff0a4b586203
:10e7d000204620f0caff68620020fff7bffefbe77b
:10e7e000b8000c00f4370d029e4c0d02b04c0d0227
:10e7f000993500028cd400109ccd00102de9f04317
:10e800003d4b8db000933d4b694603933c4b04a8b0
:10e8100000250293f6f74cfd4ff44063cde908352f
:10e8200041f28833374c0a930223204614268df890
:10e830002e30354b04a940f8043badf82c60f6f7b8
:10e8400037fd089b65626361099b04f12800a361a1
:10e850000a9bdff8f480e361bdf82c302b4f238452
:10e860009df82e30dff8e49084f8223021f033f860
:10e87000274b84f82c502360256304a8f4f7f0faa2
:10e880006846f4f7edfa294622481bf057f8224c67
:10e89000224b2946a360224bc4e90086c4e9033415
:10e8a0006761201df3f752fe1e4b294623601e4c64
:10e8b0001e4bc4e90086a3601d4b6761c4e90334a5
:10e8c000201df3f743fe1b4bc4f80090a3611a4cc4
:10e8d0001a4b2946a3601a4bc4e90086c4e90334e5
:10e8e0006761201df3f732fe164bc4f80090a36158
:10e8f0000db0bde8f08300bf0de60002c351000279
:10e90000af5100028cd40010343b0d02512a00029a
:10e91000fc4c0d0231e400023cd400100600020061
:10e92000d54c0d02344d0d0270d4001019000100b9
:10e93000e04c0d0219de000254d400101a00010050
:10e94000e94c0d021dde000208360d02444d0d0299
:10e95000f0b50246406890b10831d46821f0030355
:10e960009168201a091a043399424ff0000107d325
:10e97000c4e90013d1680b4401f10800d360f0bd75
:10e980000d460846146974b166689e4205d338b1d5
:10e990004768be423cbf0d46204621462468f2e748
:10e9a0000d462046f9e70028e9d003684db12b60f9
:10e9b0002b465169814208bf5361002340f8083b50
:10e9c000dde71361f5e7704710b50446182117f02d
:10e9d000d3f8204610bd0000014b586a20f0c7be96
:10e9e0008cd40010012a38b5044602d10b6823608c
:10e9f00003e0022a03d0032a0dd0002038bd0c20ea
:10ea00000d6817f0b1f803460028f0d095e807002c
:10ea100083e80700ebe700680028eed00c2117f030
:10ea2000abf8eae730b5002939d051f8044cc26898
:10ea3000a1f108031d19aa4214d1121bc2600024bf
:10ea4000426962b35168c3685518ab4227d15b1a5b
:10ea5000c360036913b119688a421cd14361e3b9e9
:10ea60000361ede7056900222c4624b19c4238bfc2
:10ea700022462468f9e72ab905b9436141f8085ce0
:10ea80000361dce7146841f8084c13604169914266
:10ea9000d5d14361d3e70b46dce71c60d0e730bd3e
:10eaa000438c8b4223d890f8203013b1012b0ad02d
:10eab0007047012380f82030fa234384837c43f09d
:10eac00002038374704790f82420013ad2b280f890
:10ead000242042b1002380f82030fa234384837c31
:10eae00003f0fd03ede711460430f3f795bb5b1a25
:10eaf0004384704738b50c4cd4e88f3f13f0010fb6
:10eb00000a4d09d1204619f043f928b120f080fec2
:10eb10002860204619f076f920f07afe2b681b1a3f
:10eb20005842584138bd00bf14d500106cd90010b0
:10eb300010b50446024b0360fbf71afd204610bdda
:10eb4000f04e0d020148fff7f3bf00bf44d900109b
:10eb500010b50446fff7ecff2046282117f00cf80b
:10eb6000204610bd014b586a20f001be9ccd00101c
:10eb7000002210b5044611461046f8f745fa6cb16c
:10eb8000fef776f8042805d100231a4619461846e0
:10eb9000f8f77efdbde81040fcf7e6bafef768f82e
:10eba0000128edd1f0e7000008b5064b1b78032bd8
:10ebb00006d104f0fbfebde808400021f4f70ebdcd
:10ebc00008bd00bf5fcc001070b52d4a8cb0137823
:10ebd000002b52d00023157813702022cde9042396
:10ebe000284aedb2009228202749019504aaf3f79c
:10ebf0002ffa264cd4e88f2f12f001021dd12046a7
:10ec0000039219f0c5f8039ab8b114210f20f7f751
:10ec100091fb1e2202211e4e0346cde90021304603
:10ec20000f226ff07f4105f0affd1a4b2046336095
:10ec300019f0e8f81848adf022fa012d1bd8e5b11b
:10ec40004ff47f060022124c1146201df3f7e4fa20
:10ec5000fa230022012166616384a37c201d03f056
:10ec6000fd0384f8245084f82020a3740cb0bde880
:10ec70007040f3f7d1ba094ee4e70cb070bd00bfa5
:10ec80000ed500104c4d0d02f4370d0210d50010ba
:10ec900044d90010f04e0d02c5ea00020060ff00ea
:10eca000002270b5314d8cb007200df10f018df8a9
:10ecb0000f20f4f73bfc2b685a1c2a601bb91af092
:10ecc00038fe2b4b18609df80f301bb31af031fe45
:10ecd000274e3368c01a274b98421bd900242023a3
:10ece000cde9043405230193234b04aa0093282083
:10ecf00023462249f3f7acf90122214b34601a7004
:10ed0000204b2c601c709df80f300bb91e4a13600d
:10ed10000cb070bdf5f7caff1c4cc8b110f1aa0fba
:10ed200014d01b4a1b4b10f1a00f08bf1a4600233a
:10ed300020210192184acde90413009228200f499e
:10ed400004aaf3f785f902232370dce7134aeee700
:10ed50002023cde90430124b0849009304aa03464e
:10ed60002820f3f775f90323eee700bf70d90010f0
:10ed70001cd50010df930400694d0d02f4370d021d
:10ed800011d1001020d50010f8d100100ed50010c0
:10ed9000fe420d02f12a0d02b74d0d02654d0d0226
:10eda000d04d0d0208b5074a1378ff2b1cbf013365
:10edb00013701af0befd044b1860bde80840fff761
:10edc0006fbf00bf20d5001018d5001000222de91c
:10edd000f04111468cb01046f8f75ef900287ed05d
:10ede000404b1b78002b7ad13f4f3b7803f0ff0458
:10edf000002b74d12346224652210520f7f7dcf977
:10ee00001af097fd394b1d68394b451b1878f9f7f7
:10ee100053fe854263d34ff02008364b04aa36498f
:10ee200000931e202346cde90484f3f711f9fcf783
:10ee3000d3fb0122054600f118031a604020234647
:10ee40000021cde901440094f7f7fcfceb6e01339f
:10ee5000eb66f5f725fe061e10db01233b70274b02
:10ee60001e2000932449234604aacde90484f3f725
:10ee7000eff80cb0bde8f041fff7a6be204b0196bd
:10ee80000093282023461c4904aacde90484f3f703
:10ee9000dff8e63609d1224621460620f7f79ef92b
:10eea000224621460520f7f799f9002305f11802bb
:10eeb0003b70136040201a46cde9013300930021d6
:10eec000f7f7c0fc0f4b1b7803f0ff023bb911466c
:10eed0001046f8f79ef910b9fff764ffc9e70cb0c8
:10eee000bde8f08112d100105ecc001018d50010e2
:10eef00020d50010f84d0d02f4370d020a4e0d0218
:10ef0000214e0d0211d1001008b503200df03cf880
:10ef1000034b1870bde8084080f00100fcf73eb9d3
:10ef200074d9001008b5fef7a3f9fef7a5f948b1aa
:10ef300009200df029f828b1fef79af9bde808403c
:10ef4000fef7a8ba08bd08b5002000f055fe40b194
:10ef500009200df019f8014618b9bde8084000f085
:10ef6000b7be08bd2de9f74f0d460446002855d021
:10ef7000dff8b8804ff47a79d8f80030dff8b0b015
:10ef80000344c8f800301af0d4fc06461af0cdfc51
:10ef90000746002017f01dfd0cf066fd1af0c9fcb5
:10efa000a0eb060a544533d3621e924510d34ff4aa
:10efb0007a7000fb04741b4d1af0b7fc201aa842ab
:10efc0002cd84008012828bf012017f004fdf3e7e2
:10efd000012017f0fefc144b1a78002adcd1002d1a
:10efe000dad1ca4504d2d8f80020b2f57a7fd3d35b
:10eff0000020fdf749fe0af57a790190f6f738fc12
:10f0000001980028c8d19bf80030002bf5d1c3e748
:10f0100025b903b0bde8f04ff6f72abc03b0bde850
:10f02000f08f00bfa086010012d1001078d9001027
:10f030005fcc001013b50c4b0446586a019120f0c8
:10f0400096fb58b1094b01995b68c3f308032bb9d0
:10f05000204602b0bde81040fff784bf204602b052
:10f06000bde8104017f0b5bc8cd4001000ed00e0f6
:10f070002de9f04fdff8b0b193b005939bf8003065
:10f0800080460e469246604f1bb93b78002b00f03d
:10f09000ad8020230024cde90a345c4b1e205c495e
:10f0a00000930aaa2346f2f7d3fffcf795fa3b78c0
:10f0b0000546b3b1c4663eb100f134031e60012eb3
:10f0c00002bf036d01330365032205f118031a60c3
:10f0d0000023092240200021cde901330093f7f7f6
:10f0e000b1fbfcf77dfa4ff00102d0e8cf3fc0e85a
:10f0f000412f0029f9d1dbb2002bf6d1c26801699a
:10f10000047d90f81590c360036103754375c0e8f2
:10f110008f3fd3075cbf047ae4b2930758bf4168be
:10f1200053073b7858bf90f8099018f0010f08bfbb
:10f13000002413b3002c5fd01023adf81830059bca
:10f14000adf81a60adf81e301c9badf81ca0cde9df
:10f15000083106f0c1fb0022022106ab06f0e3f9fc
:10f1600058b120220023cde90a232a4a01900092b7
:10f17000282027490aaaf2f76bffb9f1000f01d046
:10f18000fbf718fc18f0020f02d12046f5f730fd0e
:10f190000024214b3c701c70204b22462146072046
:10f1a0001c708bf80040f7f719f82246214606201c
:10f1b000f7f714f8224621460520f7f70ff8202329
:10f1c000cde90a34164b0aaa00931e2023461049a3
:10f1d000f2f73eff224605f118031c60402023464b
:10f1e0000021cde901440094f7f72cfb00220d4be0
:10f1f0001a7013b0bde8f08f06f06efb234622466e
:10f20000032106f090f9b8e75bcc0010444e0d02e4
:10f21000f4370d02594e0d025dcc00105ccc00108d
:10f220008b4e0d020ed500105ecc0010f0b5634b76
:10f2300005461b788db0002b00f0bd80604f3b78f9
:10f24000002b40f0a1805f4b1b7803f0ff04002be4
:10f2500040f09a805c4e327802f0ff03002a3dd0e5
:10f26000fcf760f9002800f097802023cde90434f2
:10f27000564b04aa564900931e202346f2f7e8fe97
:10f2800001233b70534b34701c70fcf7a5f902222c
:10f2900000f118031a600822234600214020cde91e
:10f2a00001440094f7f7cefafdf7e2fc0428234668
:10f2b00022464ff052010cbf08200720f6f77cffd2
:10f2c000002205201146f6f789ff0022062011468c
:10f2d000f6f784ff0022404b1a6055e01a4652218f
:10f2e0000620f6f769fffff70ffe04460028f1d06d
:10f2f0003a4b1b7803f0ff02002b3ad1114610461f
:10f30000f7f787ffa8bbfff74dfd062c46d0082c6a
:10f3100014bf4ff47f074ff0ff1700262023cde9dd
:10f3200004362f4b28202a49009304aa334601941f
:10f33000f2f78efe324614210120f6f7fbff1e2263
:10f3400002210346cde9002104a80122394605f037
:10f350001bfa3246012105a8f2f75eff1af0e9fa1e
:10f3600006461af0e6fa831bf92bfad904a8fbf734
:10f37000fff8fcf731f90023c0f888401a4607214e
:10f3800018460093fff774fe164b1b7843b10db07f
:10f39000bde8f040fcf7ceb80a24a9e7124fbce75d
:10f3a000002df4d1fdf764fc0328f0d12846fdf7c9
:10f3b0006bfc0128ebd00db0f0bd00bf5ecc00109f
:10f3c0005bcc00105dcc00105ccc00109f4e0d0299
:10f3d000f4370d0220d5001070d9001011d10010a3
:10f3e000af4e0d025fcc00100060ff0013b5044665
:10f3f000fdf718fc034638b90246009002210120af
:10f40000fff736fe02b010bdfff7e0fc204602b069
:10f41000bde81040fff70abf10b504460cf024fb0e
:10f420000022194b19481a60f8f762fa184b1b783a
:10f4300003f0ff0023bbfef77bfefff7b5fbf8f7f9
:10f4400095f9f7f746fff7f74bff2046fff7ceff9a
:10f45000f8f722fff9f74af8fdf70afc042801d073
:10f46000fff760fdf4f7fefef4f7f9fefdf700fc90
:10f47000042801d0fff767fdbde81040f4f74cb950
:10f480008c20f4f7edf8ede778d900103cd90010a6
:10f490000dd50010f0b5224e044696f82c300d46de
:10f4a000174687b0002b38d0706a20f060f900282a
:10f4b00033d104900c2016f057fb10b1c0e9004581
:10f4c0008760184b02900593174b1420049316f095
:10f4d0004bfb0446d8b1154b03600023c360049b6b
:10f4e0003bb1022202a904309847059b2361049b8b
:10f4f000e3600f4bf2692360306b002301a9019494
:10f5000020f093f918b1236820469b68984702a819
:10f51000f3f7a6fc002007b0f0bd2846a047f9e7a6
:10f520008cd40010b5f4000265e90002c8370d0262
:10f53000dc370d0203681868d3e90112fff7aabf90
:10f5400008b5002301211a461846f7f712febde858
:10f550000840f5f755bb000037b501900cf07afa7a
:10f56000019905460448fff7f3f9044628460cf0d4
:10f5700075fa204603b030bd24d9001013b50190b0
:10f580000cf068fa044601990448fff74bfa20464c
:10f5900002b0bde810400cf061ba00bf24d90010e1
:10f5a0006ff0770070470000032809d8dfe800f00b
:10f5b0000a02040604487047f5f74cbef8f71cbe73
:10f5c00000207047014870479ccd00108cd400107b
:10f5d00013b500240b4a23460b490c480094f1f75d
:10f5e000cbff0b4b0b4a1c605c600b4bc2e9044425
:10f5f0005360d3604ff480639360084b136002b094
:10f6000010bd00bf59e90002e5ea000275ea0002f8
:10f610003cd9001024d9001024d50010d84e0d027a
:10f62000002270b511468cb00546f7f784fd0246fe
:10f6300090b1002228461146f7f77dfd28b100233e
:10f6400001211a462846f7f794fd00220521284695
:10f65000f7f748fe012606e001462846f7f71cfdad
:10f660000028e6d1064600212846f7f79dfd04460e
:10f6700038bb284604a925f0a7ff68b9fcf72efb84
:10f6800002220499fcf764fcc8b9fcf727fb0422aa
:10f690000499fcf75dfc044600230322202000218e
:10f6a000cde901330093f7f7cdf80123002063f390
:10f6b000070064f30f2066f317400cb070bd0124ff
:10f6c000eae700242023cde90434054b0120009310
:10f6d00004492346019504aaf2f7bafce5e700bf06
:10f6e000094f0d02fc4e0d02012a38b5044602d125
:10f6f0000b68236003e0022a03d0032a0dd0002008
:10f7000038bd0c200d6816f02ffa03460028f0d003
:10f7100095e8070083e80700ebe700680028eed0d3
:10f720000c2116f029faeae770b50446154649b1ee
:10f730000021f7f739fd28b1002320461a46194663
:10f74000f7f732fe3db100232046bde870401a466f
:10f750001946f7f79dbf70bd21b18b88834201d058
:10f760008968f9e7084670470b46c1681846fff7f5
:10f77000f3bf0a4608b50e21fff7f6ff58b1037b29
:10f78000934202d1c389db0704d581680e20fff7bd
:10f79000e3fff3e7012008bd08b500680a46438887
:10f7a000022b02d84ff0000008bd0e21fff7dcff4e
:10f7b0000028f9d0037b934201d1c089f4e7816826
:10f7c0000e20fff7c9fff3e74ff00102d0e8cf3f6b
:10f7d000c0e8412f0029f9d1dbb2002bf6d17047e8
:10f7e0002de9f04fbb4b144693f82c208fb0064602
:10f7f0000491e2b1586a1ff0baffc0b90c900c2016
:10f8000016f0b2f918b1049b0660c0e90134b24b9e
:10f810000a900d93b14baf480aa90c93f3f724fc5f
:10f82000044670b907460aa8f3f71afb05e0002161
:10f83000304615f0b3fd071e0fda38460fb0bde8ad
:10f84000f08f00224ff0ff31406920f0a9f82368c3
:10f8500020469b68a7699847e5e7f8f71dfd082152
:10f86000f8f7acfe042130460a96fff782ff002825
:10f8700068d105213046fff77cff002862d10321c3
:10f880003046fff776ff804600285bd104213046e2
:10f89000fff76aff002853d04ff47a73c568b5fbb1
:10f8a000f3f5b368da072bd5f5f7d2ff40b3fbf7d2
:10f8b00097fe0446fff788ff0023e268d4f8109013
:10f8c000677de360236123756375c4e88f3fd307c9
:10f8d00058bf237a900758bfd4f80490510758bff7
:10f8e000677afbf77dfe0446fff76eff0723e360b0
:10f8f0000123c4f81090237567750023c4e88f3f77
:10f90000002306211a4601200095fff7b1fbfdf701
:10f9100089f98346fdf780f90a9f04213846fff7ed
:10f9200028ff0446002850d104210aa8fff734ff1d
:10f93000c2070dd520460ef0c7fca246254618e0aa
:10f940004546aee7f5f784ff4ff0000b8046e3e74e
:10f950000420fff765fec0f3072ac0f307448df8c3
:10f960001da08df81e408df81c00c5b25ffa8afa02
:10f97000e4b205213846fff7fcfe60b34ff0000902
:10f98000cde902990320fff74bfe0021c0f30723c6
:10f990008df82530c0f307438df824008df826300c
:10f9a000c3b208460593f2f77bfce720f1f76cfc45
:10f9b00001213846fff7d8fe38b383891b2b7cd052
:10f9c00081680120fff7c8fef6e7002108460ef027
:10f9d00081fc0024b1e704210aa8fff7ddfec3077c
:10f9e000ccd40520fff71cfec0f30723c0f3074962
:10f9f0008df82130c2b2dbb28df822908df8200054
:10fa0000029203935ffa89f9bce70120f3f7e5f866
:10fa100000220499304615f007fd0746f3f7e7f892
:10fa200001200021f2f73cfce720f1f709fc002d52
:10fa300045d0224651460420fff776fe029b23b1b3
:10fa40004a4605200399fff76ffe059b33b103205b
:10fa50009df826209df82510fff766febbf1000fec
:10fa60003ed0fdf7b7f8fdf703f904460020fdf797
:10fa70000bf9054600287ff4e0ae013ce4b2012c0e
:10fa80003ff6dbaefdf7cef800283ff4d6ae2846b1
:10fa900019f042ff4ef660250446002019f03cffa5
:10faa000001b61f10001a84271f100030fd2f5f7cc
:10fab000cffe60b9f5f7dcfeefe70020a6e72846a9
:10fac0000ef005fc294601200ef004fcb6e7f5f720
:10fad000bffeb2e69ccd001079fa000269f6000282
:10fae000b8f1000f3ff4a9aefaf7d0ff5b465a46d3
:10faf000042105f018fda0e603681868d3e9011297
:10fb0000fff76ebe70b500231646202204460d4650
:10fb10008ab0cde90223074a01200092064902aad1
:10fb2000f2f796fa3246294620460ab0bde8704000
:10fb3000fff756be254f0d02fc4e0d02012a03466b
:10fb400002d1016000207047022a04bfd1e9000100
:10fb5000c3e90001f6e7012a034602d10160002053
:10fb60007047022a04bfd1e90001c3e90001f6e7aa
:10fb7000012a034602d1016000207047022a04bf17
:10fb8000d1e90001c3e90001f6e7012a034602d1e9
:10fb9000016000207047022a04bfd1e90001c3e9d7
:10fba0000001f6e7012a034602d1016000207047f8
:10fbb000022a04bfd1e90001c3e90001f6e7012ae6
:10fbc00002d1016000207047022a04bf0b68036065
:10fbd000f8e7012a034602d1016000207047022a9b
:10fbe00004bfd1e90001c3e90001f6e700224ff0ac
:10fbf000ff311ff0d5be000070b52d4e044696f8bb
:10fc00002c3086b0002b4bd03046f5f79bfd0546d7
:10fc1000002845d1274b1c200593274b02940493c1
:10fc200015f0a2ff0446002831d0244bc5600360c4
:10fc3000049b3bb1022202a904309847059b236133
:10fc4000049be360002520461d4b2a4623600121ca
:10fc500040f8145f1ff094fe1a4b01a92360f2696b
:10fc60002b46306b01941ff0e0fd014650b9706add
:10fc700008b11ff0a9fd00224ff0ff3160691ff0ad
:10fc80008ffe257e236820469b68984700e0054646
:10fc900005f0010502a8f3f7e3f8284606b070bda9
:10fca000fdf7a0fc06b0bde87040fdf7b7bc00bf93
:10fcb0009ccd001049fc00023ffb0002543b0d02aa
:10fcc000683b0d027c3b0d020068fff795bf00000a
:10fcd00070b5534d044695f82c300e468ab0bbb132
:10fce0002846f5f72ffd98b94e4b284605934e4b05
:10fcf00002a98df8084003960493f3f7b5f9054679
:10fd0000c0b9044602a8f3f7abf820460ab070bdac
:10fd100009200cf039f9b0b92023cde90230434b6a
:10fd20004349009302aa03463220f2f791f96ff09b
:10fd30008104eae74069fff759ff2b6828469b6872
:10fd4000ac699847dee7002c4cd0fdf74bfcfdf783
:10fd500065fc044608b10024d7e7fdf789fafdf7f2
:10fd60008bfa90b109200cf00ff970b12023cde986
:10fd70000234304b2e4902aa012000932346f2f7a9
:10fd800067f9fdf775fafdf785fb002520262a4b5c
:10fd900002aa2749012000932b46cde90265f2f71c
:10fda00057f9fdf71ffc0121fdf73bfcf4f75afa68
:10fdb000183000f0a5fcfdf715fcfef715f8044619
:10fdc0000028a2d01d4b1a49009302aa2b460120fd
:10fdd000cde90265f2f73cf9fdf704fc2946fdf791
:10fde00020fc92e7fdf7fefbfdf718fc0028b2d0df
:10fdf0002023cde90234124b02aa0d4900930120c1
:10fe00002346f2f725f9fdf7edfb2146fdf709fc46
:10fe1000fdf7e8fb0ab0bde87040fdf77bbc00bf12
:10fe20009ccd0010c5fd000253fb0002414f0d02a6
:10fe3000f4370d02764f0d02c44f0d02d94f0d025b
:10fe4000f74f0d0241680078fff742bf7fb51c4da8
:10fe5000044695f82c300e46b3b12846f5f772fcef
:10fe600090b9184b69460393174b2846cde90046d5
:10fe70000293f3f7f9f8044648b905466846f2f7e5
:10fe8000efff284604b070bd54b9104df9e7406942
:10fe9000fff7acfe236820469b68a5699847ede70d
:10fea00009200cf071f840b1f4f7dcf92146183064
:10feb00004b0bde8704000f0c3ba6ff08105e0e720
:10fec0009ccd001051fe000225fb0002f2feffff58
:10fed000d0e90001fff7babf7fb51c4d044695f885
:10fee0002c300e46b3b12846f5f72cfc90b9184bd0
:10fef00069460393174b2846cde900460293f3f772
:10ff0000b3f8044648b905466846f2f7a9ff284603
:10ff100004b070bd54b9104df9e74069fff766feb3
:10ff2000236820469b68a5699847ede709200cf0f7
:10ff30002bf840b1f4f796f92146183004b0bde82b
:10ff4000704000f095ba6ff08105e0e79ccd00109d
:10ff5000ddfe00020bfb0002f2feffffd0e9000114
:10ff6000fff7babf7fb51c4d044695f82c300e46fe
:10ff7000b3b12846f5f7e6fb90b9184b69460393f1
:10ff8000174b2846cde900460293f3f76df8044677
:10ff900048b905466846f2f763ff284604b070bdcd
:10ffa00054b9104df9e74069fff720fe2368204659
:10ffb0009b68a5699847ede709200bf0e5ff40b184
:10ffc000f4f750f92146183004b0bde8704000f055
:10ffd00067ba6ff08105e0e79ccd001069ff000271
:10ffe000f1fa0002f2feffffd0e90001fff7babf0d
:10fff0007fb51c4d044695f82c300e46b3b128460b
:020000040807eb
:10000000f5f7a0fb90b9184b69460393174b2846a8
:10001000cde900460293f3f727f8044648b90546b0
:100020006846f2f71dff284604b070bd54b9104d64
:10003000f9e74069fff7dafd236820469b68a56968
:100040009847ede709200bf09fff40b1f4f70af95c
:100050002146183004b0bde8704000f039ba6ff0a6
:100060008105e0e79ccd0010f5ff0002d7fa000201
:10007000f2feffffd0e90001fff7babf7fb5174dd1
:10008000044695f82c300e4603b32846f5f75afb84
:10009000e0b9134b69460393124b2846adf8004074
:1000a00001960293f2f7e0ff044668b14069fff75a
:1000b0009dfd236820469b68a56998476846f2f72e
:1000c000cffe284604b070bd0546f7e7fdf78afa73
:1000d000214604b0bde87040fdf7a6ba9ccd0010e3
:1000e00069000102bdfa000241680088fff7c6bf3f
:1000f000f8b5044605462f4615f8016b3046acf0be
:1001000091f80028f7d15f2ef5d0381bf8bd2de906
:10011000f8430c461746994678b119b38e18a64293
:1001200005d9054615f8013b4bb904f8013b0023fe
:10013000781e341b06f8013c001bbde8f883242b15
:100140000dd12846fff7d4ff804630b12246014644
:10015000331b2846c847454404442846dfe704f8d3
:10016000013bfae70846e8e77047704737b50446b1
:1001700001910bf06ffc019905462046fef7e8fb64
:10018000044628460bf06afc204603b030bd10b58b
:100190000446042115f0f0fc204610bdc86910b5d6
:1001a0000c4608b115f0e6fc0023c4e90133e36115
:1001b00010bd000010b5044b04460360406808b150
:1001c00015f0d8fc204610bd20520d0210b5044693
:1001d000fff7f0ff2046182115f0cefc204610bd99
:1001e00008461146adf01ab90846acf049b90846c0
:1001f000acf03eb92de9f0410c461e4617460546c7
:100200000368ddf818805b689847c4e90968e7620d
:10021000a8691ff06ffbeb6843b19c610023a361e9
:10022000a869ec60bde8f0411ff073bbac60f5e776
:1002300037b5054601910bf00dfc0446019928469f
:10024000fef7f0fb204603b0bde830400bf006bce3
:1002500010b5084cd4e88f3fdb0709d4204617f0cf
:1002600097fd28b1204617f0cdfd0348abf007fffe
:10027000024810bd7cd90010e9000102785100103d
:1002800008b558f069f918b1bde808402af052ba2b
:1002900008bd38b50446062058f084f8054668b114
:1002a000204658f08bf801222946204658f0def807
:1002b000034628b1bde838402af03cba6ff0770316
:1002c000184638bd08b558f0e5f918b1bde8084042
:1002d0002af030ba08bd13b5044608460191f0f77c
:1002e00071fd019902462046fff7ecff02b010bdf8
:1002f00010b5c368044623b90a200e4a0e49f0f728
:100300006ffee3685a681989023a5a60e268936896
:1003100002339360e3685b681980d4e90223916a31
:1003200029b10b60002119609362e16010bd536236
:10033000f8e700bf576902020d500d0270b50025a5
:100340000446394bc0e902550360c0e904554160d9
:1003500040f8185f1ff0bffa344be56163654ff654
:10036000ff732562a4f86c30a4f86e30c4e9095517
:100370002f4bc4e90b55c4e90d55c4e90f55c4e929
:100380001155c4e91355c4e91955c4e91755c4e911
:100390001c55e567a56584f88050a56784f88150f1
:1003a00084f8825004f1840203f11006154618689f
:1003b0005968083303c5b3422a46f7d118681d4b64
:1003c000286004f1980203f1100615461868596870
:1003d000083303c5b3422a46f7d11868164b286084
:1003e00004f1ac0203f11006154618685968083389
:1003f00003c5b3422a46f7d11868104b286004f1b0
:10040000c00203f11006154618685968083303c581
:10041000b3422a46f7d11868002328602046a4f882
:10042000d430a4f8d83070bdb4520d0220520d0261
:1004300084520d0298520d026c520d0258520d0258
:1004400030b581b10b4600f1840201f1100514466c
:1004500018685968083303c4ab422246f7d11868bc
:100460002060002030bd0148fce700bff2feffff26
:1004700030b581b10b4600f1ac0201f11005144614
:1004800018685968083303c4ab422246f7d118688c
:100490002060002030bd0148fce700bff2fefffff6
:1004a00030b581b10b4600f1c00201f110051446d0
:1004b00018685968083303c4ab422246f7d118685c
:1004c0002060002030bd0148fce700bff2feffffc6
:1004d00030b581b10b4600f1980201f110051446c8
:1004e00018685968083303c4ab422246f7d118682c
:1004f0002060002030bd0148fce700bff2feffff96
:1005000070b50246054601f1840601f194033446b4
:1005100003cc9c4210605160264602f10802f6d1dd
:1005200020681060284670bd8b890022a0f86e30cc
:100530001423c36780f8802090f88030dbb280f805
:10054000813000f17803c3e8af2f00f1740353e862
:10055000001f0131c3e8e01f0028f8d110467047a2
:10056000b0f86e308a899bb29a4202bf4b68033b57
:10057000c36700207047b0f86e308a889bb29a42f9
:1005800012d1ca88b0f8d6309a420dd1002380f833
:1005900080308a689a42c8bf012380f8803090f882
:1005a0008030dbb280f88130002070472de9f041c7
:1005b000044690b0002021f0dbf920b10a204a4a1d
:1005c0004a49f0f70dfd94f88250002d40f08980e3
:1005d0002b4601200df1020204f1840122f02efbd2
:1005e00000287bdb424f2822294606a8059708ae43
:1005f000abf093ff04f1980cbce80f000fc6dcf8d9
:1006000000302a46336002238df81830bdf80230de
:1006100001a905a8adf8343022f042f900285ddbcd
:100620002b4601223349bdf80a0021f01ffd0028a6
:1006300054db2022294606a8059708aeabf06dffd3
:1006400004f1ac0cbce80f000fc6dcf80030dff89a
:10065000ac80336010238df81830bdf802302a4684
:1006600001a905a8cde90e84adf8343022f018f9bf
:10067000002833dbbdf80a302022a4f8d430bdf8be
:100680000e302946a4f8d630059706a808ae04f126
:10069000c007abf042ff0fcf0fc63b682a4633605e
:1006a0000c238df81830bdf8023001a905a8cde95a
:1006b0000e84adf8343022f0f3f800280edbbdf8dc
:1006c0000a302a4621460c48a4f8d83022f024f9f2
:1006d000002803db0123284684f8823010b0bde8ef
:1006e000f0816ff0d100f9e757690202504c0d021a
:1006f00003002c0080520d02650f0102e109010286
:10070000002238b504461146104614f0a4ff2046d6
:10071000fff74cff054660b94ff480600749abf026
:1007200053f940b14ff48063c4e91955a0652066c0
:10073000e365284638bd024dfbe700bf0d700f0290
:10074000fcfefffff8b506460d4638201049174657
:10075000abf038f90446c0b138220021abf0ddfe21
:100760000b4905f11000abf02ff9e06148b10db174
:10077000083060600020336fa560236366613c60d1
:10078000f8bd3821204615f0f7f90248f8e700bf18
:100790000d700f02fcfeffff70b50d461668144683
:1007a000fff756fd036831461b6905f10c029847b7
:1007b00046b948b1066000f10c03c0e9013520607c
:1007c000002070bd0028f6d10048fae7fcfeffffcc
:1007d00070b5c36804460d46164623b10a200c4a7c
:1007e0000c49f0f7fdfba06804f10c02b11cfff707
:1007f000d3ff00280adb0020e2685368023353600d
:10080000e2689368023b9360e3682b6070bd00bfb1
:100810005769020223500d0230b5002585b04ff410
:10082000007202a904460295fff7d2ff00280edbf2
:10083000114b02990093019503ab04f12800d1e913
:100840000112039552f0ccfc18b129f073ff05b0ea
:1008500030bddde9023204f11c0059689a60f7f7f7
:1008600005fd0028f3db2046fff742fd03230120ae
:10087000c4f8c831ebe700bf7da60302f0b500263f
:1008800085b02022694605460096fff7a1ff041ea9
:1008900023db009b05f11c0738465968fff7f0fc85
:1008a000041e1adb384657f08efd01a8cde901661b
:1008b0000396fff7eefc041e0cdb202205f5d47135
:1008c00001a857f087fe58b91b4901a8fff703fd9f
:1008d000041e0ada01a857f076fd204605b0f0bde7
:1008e00029f028ff041ef5dbeee7144901a8fff705
:1008f000f2fc041eeedb124901a8fff7ecfc041e1b
:10090000e8db009b01a8d3e90112fff7dbfc041e22
:10091000e0db009b01a8596857f0ccfe38b92846a7
:10092000fff7e6fc07230024c5f8c831d2e729f019
:1009300001ff041ecedbf2e73a500d0241500d02da
:10094000c9a60d0230b5002585b04ff4007202a98a
:1009500004460295fff73cff00280edb114b02997d
:100960000093019503ab04f12800d1e9011203952e
:1009700052f090fb18b129f0ddfe05b030bddde985
:10098000023204f11c0059689a60f7f76ffc0028e6
:10099000f3db2046fff7acfc04230120c4f8c83188
:1009a000ebe700bf7da6030238b515460c4601f102
:1009b000200205f11001fff7effe002806db35b13c
:1009c000236a5b6808330020c4e9033538bd2b4631
:1009d000f9e7000038b554300c460c311546fff7e6
:1009e000c5fb40b10246002342f80c3bc0e901249c
:1009f0002860184638bd0148fce700bffcfeffff39
:100a000073b5b0f86e308a889bb29a4205460c46a0
:100a10001fd1b0f8d830ca889a424ff000031dd1d8
:100a2000c96801aa0193fff7d5ff002812dbd4e9ba
:100a30000321019b5868abf049fd019e0bf00af8b9
:100a40002b6a4bb12b6a1e60002434602e620bf0bf
:100a500005f8002002b070bdee61f5e71846f9e731
:100a600070b503680546092b0c468cb003d00b2be0
:100a700026d00cb070bd01462046fff7c1ff00280c
:100a8000f7d020230026cde904362b68029001938d
:100a90000e4b04aa0093322033460d49f1f7d8fae1
:100aa0004ff6ff72b4f86e309bb29342e1d03146fc
:100ab000b4f86e0080b20cb0bde8704021f024baea
:100ac00001462046fff757fdd9e700bf58500d02f9
:100ad00048500d0210b50446006808b115f04af8f8
:100ae000204610bd03681bb19a69026002b94260da
:100af0001846704710b50379044613b90120aaf0cf
:100b0000fcff036823b118681ef003ff0023237164
:100b100010bd03681bb11a68026002b94260184632
:100b2000704738b5056804464db10af093ff256853
:100b30002b682360236803b963600af08fff28469f
:100b400038bd0b46014618b11a681846d2681047de
:100b5000704710b50c4629b1fff77afb01462046d5
:100b6000fff7efff10bd70b50c46a1b1d1e90956f2
:100b7000096afff7eeffe06908b114f0fbff3821c6
:100b8000204614f0f9ff35b131462b46bde87040e0
:100b90006ff06300184770bd2de9f04390f8813085
:100ba00004468bb023b9002528460bb0bde8f0837e
:100bb000436c23b90a20304a3049f0f711fad4f8cf
:100bc0007c8004f12409a66cb0451fd9656aedb19b
:100bd000aa68a8eb0607974228bf1746606c3a46fa
:100be00069683044abf072fc6b683b446b60ab6887
:100bf000db1bab6033b94846fff78bff2946204625
:100c0000fff7a7ffa36c3b44a364dce7beb904f184
:100c10007803d3e8af3f002bc5d104f11007384665
:100c2000fff760ff05460028bdd0d0e9093100205c
:100c30009847294620466e62fff795ffefe70023ad
:100c40003246616cb4f8d40021f02cfaa36c05464e
:100c500083424ff000030bd02022cde90223084a43
:100c6000019000923220074902aaf1f7f1f99be7bf
:100c70001d46a36498e700bf5769020284500d0225
:100c8000a0500d0248500d0208b50346084619b1a0
:100c900003f15401fff755ff08bd00002de9f84f9f
:100ca000044689461746002500f11c06636bbb42cb
:100cb00028d34ff00008dff888a0dff888b0474558
:100cc00039d9e66a26b9524659460a20f0f788f91a
:100cd000b268a7eb0805954228bf154671682a46f9
:100ce00009eb0800abf0f2fbb3685b1bb360f3b930
:100cf00004f12c00fff70dff31462046fff7c4ff3b
:100d0000a844dce73046fff70cff58b1236b3bb13a
:100d1000186005602063636b826813446363c5e7f2
:100d2000e062f6e7636bbb42c3d2bde8f88f73683d
:100d30002b447360e4e7626b0120d21b6263f4e72b
:100d400057690202dd500d02f7b50446154600262c
:100d500000f11c07636bab4211d238460191fff7db
:100d6000e0fe019958b1236b3bb118600660206327
:100d7000636b826813446363ece7e062f6e7626bdf
:100d8000954228bf15464db12a462046fff786fffb
:100d900020b90a20034a0449f0f722f9284603b093
:100da000f0bd00bf57690202f2500d02f7b51546bb
:100db000d0e905329a4204460e4610d1002702229d
:100dc000806801a9adf80470fff768fff8b1bdf8bd
:100dd00004306361013bb3f5007f14d2a761616801
:100de000d4e90523a068d21a1944fff7adffa3691f
:100df00018446369a061984209d363680020336096
:100e000063692b6001e06ff0bd0003b0f0bd01200d
:100e1000fbe7002313b5694601aa0446cde9003378
:100e2000fff7c4ff40b9dde9001204f1280052f0d9
:100e3000f5f818b129f07efc02b010bd04f11c00d9
:100e4000dde90012f7f712fa0028a2bf0223012001
:100e5000c4f8c831f0e7002313b5694601aa044677
:100e6000cde90033fff7a2ff40b9dde9001204f13c
:100e7000280052f057f918b129f05cfc02b010bdff
:100e800004f11c00dde90012f7f7f0f90028a2bf19
:100e900005230120c4f8c831f0e70000f0b5836bea
:100ea00004468fb0d3b9022206a9adf81830fff777
:100eb000f5fe00286ad0bdf818502046294604f1f6
:100ec0003802fff73ffc002860dba36bbdf8182059
:100ed000db6910351a800223e5632364a36bd4e930
:100ee0000f21dd69521a20462944fff72dff236c9c
:100ef0001844e36b2064984247d3e36c23b90a207b
:100f0000234a2449f0f76cf8e66ca36baa1c9f688f
:100f1000736d013373650693706cb16c07ab03c3db
:100f200008230593fb182b44cde9032302230292e7
:100f3000cde9005330460c2306aab91d57f026fa16
:100f400018b129f0f7fb002820db6988a36baa8879
:100f50009986a36b00255a802023cde90635a36b23
:100f600001209a8e0c4902925b8806aa01930b4bd2
:100f700000932b46f1f76cf8606822460368a16b7a
:100f80001b689847c4e90e55256400200fb0f0bdda
:100f90005769020206510d0248500d021f510d0201
:100fa00038b5b0f86e308a899bb29a42044617d1a0
:100fb00000f11c052846fff7b4fd014618b1204694
:100fc000fff762fef6e74ff6ff73743424f8063c31
:100fd000607354e8003f0133c4e8e23f002af8d1cf
:100fe000002038bd70b503680546042b0c468cb054
:100ff00027d0062b2ad0032b2dd101462046fff700
:1010000093fa40b320230026cde904362b680290e2
:101010000193124b04aa0093322033461049f1f792
:1010200017f84ff6ff72b4f86e309bb2934212d0ad
:101030003146b4f86e0080b20cb0bde8704020f0cc
:1010400063bf01462046fff7abffdae701462046c3
:10105000fff786fad5e70cb070bd00bf58500d02ff
:1010600048500d020368016013b1184614f082bda8
:10107000704710b5044600210430fff7f3ffd4e9b0
:101080000201fff766fd0023c4e90533e36010bdec
:1010900000232de9f04194b004aa03a90646cde946
:1010a0000333fff783fe0446a0b9049a202a40f0d8
:1010b000b9805f4b06f1280806f5c47505900190cc
:1010c00000932946404605ab52f020f930b129f093
:1010d00031fb0446204614b0bde8f081059f202f67
:1010e00040f0a280404651f03cff06a8cde90644fe
:1010f0000894f7f799f8041e36db06a8f7f7adf861
:10110000041e31db3a46294606a8f7f7aff8041e5d
:101110002adb0822474906a8f7f7a8f8041e23dbb4
:1011200006f5d478414606a8fff7aaf8041e1bdb93
:1011300006a857f048f906a8f7f776f8041e13db5f
:1011400006f11c07394606a857f06af980b9002550
:101150001c2229460da80c95abf0dff90ca906a8b6
:10116000fff78ef8041e08da06a857f02cf9b1e74d
:1011700029f0e0fa041ef7dbe9e706a857f023f9a7
:1011800009a8cde909550b95fff783f8041e0bdb81
:101190002022414609a857f01dfa48b9264909a856
:1011a000fff799f8041e08da09a857f00cf9dbe7f5
:1011b00029f0c0fa041ef7dbf0e7204909a8fff781
:1011c0008af8041ef0db1e4909a8fff784f8041e04
:1011d000eadb20220ca909a8fff774f8041ee3db60
:1011e0000ca909a857f066faa8b9039c202220464a
:1011f0000ca9abf05bf998b921463846049af7f789
:1012000035f8041ed0db3046fff733ff06230124f8
:10121000c6f8c831c8e729f08dfa041ec4dbe4e73c
:10122000084cc1e7074c55e76ff0f90452e700bfdf
:101230007da603024c510d023a500d02c9a60d02c3
:1012400041500d02e8feffff10b5d0f8c83104464a
:10125000013b062b05d8dfe803f0070f1215181b1a
:101260001e006ff0d10010bdfff7d3fd0028fadaa1
:101270000823c4f8c831f6e7fff764fbf6e7fff789
:10128000eafdf3e7fff7c8faf0e7fff701ffede744
:10129000fff7f4faeae70020e5e7000010b504469e
:1012a0000f4b40f8283b51f05cfe2022002104f552
:1012b000c470abf032f92022002104f5d470abf0f9
:1012c0002cf904f11c0057f07ef8064b20462360f1
:1012d000fff7cffe201dfff7fdfb204610bd00bf2e
:1012e0004c520d0238520d0210b50446fff7d6ffde
:1012f00020464ff4e67114f03ffc204610bd036811
:1013000001601bb11a681846526810477047000008
:10131000f0b5002689b004ad074632460f212846b5
:101320000696cde90466cdf81b6014f094f9002808
:1013300052db0e2858dd4ff4e6702e49aaf042fb2e
:10134000044690b12c4bc0e90167c0e90366c0e9cf
:101350000566c0e90766036046624ff4b072314625
:101360002830abf0daf8c4f8c861214607f1500024
:10137000fff7c5ff3c6d002c39d01e494ff40070bb
:10138000aaf022fb0146201dfff76cfe63684bb3f9
:1013900018f0cffa04f11c0620613046f6f744ff3e
:1013a000031e17db3046f6f758ff031e12db04f16d
:1013b0002800039051f0aafd0f230622cde9005327
:1013c00001210323039851f0f7fd034630b129f0c2
:1013d000b1f9034603eae37009b0f0bd0122c4f895
:1013e000c821f7e7054bf5e76ff0f900f4e703488c
:1013f000f2e700bf0d700f024c520d02fcfeffff22
:1014000010b50a490446f420aaf0defa014604f1b8
:101410004400fff727fe636c2bb12046fff778ffef
:1014200000eae07010bd0248fce700bf0d700f023b
:10143000fcfeffff034607b50068196048b1019044
:1014400056f048ff5c21019803b05df804eb14f0fe
:1014500093bb03b05df804fb70b5036d054623b97b
:101460000a20214a2149eff7bbfd2c6dd4f8c83181
:10147000072b26d104f5c4745c201d49aaf0a2fafa
:10148000064630b144220021abf047f80023c6e9fc
:10149000153305f14c003146fff7ccffed6c05b379
:1014a000284656f0f0fe802322460221284656f0b8
:1014b000eefe034660b129f03df9034603eae3700e
:1014c00070bd0a20084a0b49eff78afd0024d3e7d4
:1014d00022696a646269aa64a269ea64e2692a65a7
:1014e000ece70548ece700bf5769020255510d02d1
:1014f0000d700f026d510d02fcfeffff10b5036869
:10150000044613b90120aaf0f8fa02790ab12d2095
:10151000f9e718681ef0eef90123237110bd0000f1
:10152000f0b500f1180391b006930023064606a813
:101530008df81c30fff7e2ff012306f108058df856
:101540001c302846fff7cefa044640b1026b336fd9
:101550009a4204d001463046fff705fbf1e706a8a2
:10156000fff7c8fa002c6cd0236a002b58d0236aee
:101570005d6823692b80e36aa28e6b606a80f36cde
:1015800023b90a20304a3149eff72afdf76cd4f825
:1015900010c0bb6daa1c0133bb6543f00043089328
:1015a000f86c396d09ab03c30823059363442b44de
:1015b000cde9032302230292cde9005338460c23e0
:1015c00008aa0cf1060156f0a7fe18b129f0b2f8ee
:1015d000051e2ddbb36a226a002b2ed01a60002371
:1015e0001360b26220222362cde90823a28e01207b
:1015f0000192174a1749009208aaf0f729fd656a77
:10160000b5b17369dbb19c610025a56174619df87a
:101610001c3013b106a8fff76dfa284611b0f0bdd3
:101620001021304604f12002fff7b6f8051e9edabd
:1016300021463046fff797fae9e77262cfe7346157
:10164000e2e72546e3e700bf5769020206510d02b3
:1016500085510d0248500d0273b590f88230044652
:10166000002b58d000215030fff749fe002104f133
:101670004c00fff7dffe002104f14400fff7f2fc0d
:1016800004f118030093002368468df80430fff737
:1016900035ff012304f108058df804302846fff7d3
:1016a00021fa014618b12046fff75dfaf6e76846d1
:1016b000fff720fa04f110052846fff713fa014658
:1016c00090b904f124052846fff723fa014678b9ba
:1016d00004f12c063046fff71cfa054660b10146be
:1016e0002046fff7d1faf5e72046fff73cfae3e79b
:1016f0002046fff72efae6e72046a16bfff733fa04
:101700009df80430c4e90e5525646563a56413b1e2
:101710006846fff7eff902b070bd000070b50546ee
:101720008cb000f17403d3e8af3f026f9a4260d0ef
:10173000b0f86e20b0f86c400367a0f86c20fff79b
:101740008bff4ff6ff72b5f86c30934239d000240e
:101750002023cde90434574b01205749009304aab4
:101760002346f0f775fc234622464ff40020002163
:10177000cde901440094f5f765f82846fff740feef
:101780000446002835d02023002601944ff6ff742c
:10179000cde90436494b322000934749334604aa29
:1017a000f0f756fcb5f86c00a04204d0314620f0aa
:1017b000abfba5f86c4028460cb0bde87040fff7c5
:1017c0004bbf9c4266d000242023cde904343c4b1f
:1017d00001203949009304aa2346f0f739fc234637
:1017e00001224ff400200021cde901440094f5f7d7
:1017f00029f84ff6ff73b5f86c209a424ad0286d4d
:10180000002849d003689b689847041e16da002612
:101810002023cde904362b4b322000932649334652
:1018200004aaf0f715fc3346cde9016600960222c2
:101830004ff400200021f5f705f8a4e723d128464e
:10184000fff70afe044620b10023cde901330093df
:10185000ede7014605f15000fff751fd2023cde9ea
:101860000434194b01201449009304aa2346f0f7cd
:10187000effb234603224ff400200021cde9014471
:101880000094f4f7dfff2846fff786f904460028a6
:101890007ff479af0cb070bd2846fff741fe0446d7
:1018a00000287ff470af2846fff7f8fa04460028b6
:1018b000e9d068e7b2510d0248500d02e9510d021e
:1018c000bc510d02c9510d02da510d022de9f04350
:1018d00004460f461568dff8888087b0002d3dd09c
:1018e000d5f80c90d9f800305e78022e01d02d6822
:1018f000f4e7182200216846aaf00ffed9f800305c
:101900005a78022a18d101225b688df800201bba90
:10191000019399f8103039462046059329f0ecf8e8
:1019200030b16a464146204629f070fa0028ded1df
:10193000002007b0bde8f0830a2af9d103f10802bc
:101940008df800600df1040c18336646106851687c
:10195000083203c69a42b446f7d1dae70120e8e735
:10196000f2340d0238b51468054623685bb163682c
:101970004bb129f0c1f838b1d4e900122846bde8ce
:10198000384029f000ba012038bd00002de9f043ad
:1019900004460f461568dff88c8087b0002d3ed0d6
:1019a000d5f80c90d9f800305b780a2b01d02d685f
:1019b000f4e7182200216846aaf0affdd9f80030fc
:1019c0005a78022a18d101225b688df800201bbad0
:1019d000019399f8103039462046059329f08cf888
:1019e00030b16a464146204629f010fa0028ded17f
:1019f000002007b0bde8f0830a2af9d102220df1d8
:101a0000040c8df8002003f10802183366461068b4
:101a10005168083203c69a42b446f7d1d9e701208b
:101a2000e7e700bff2340d0270b50c460546eff74c
:101a3000c9f906462046eff7c5f98642024607d3a4
:101a400021462846acf09efbb0fa80f0400970bdfc
:101a50000020fce710b512490446fff7e5ffb8b9ce
:101a600020461049fff7e0ffa0b920460e49fff7d6
:101a7000dbff88b920460d49fff7d6ff70b9204635
:101a80000b49fff7d1ff002814bf1020002010bd24
:101a90000120fce70220fae70420f8e70820f6e737
:101aa000c0520d02617c0e0267c60d0268480d022d
:101ab000f5540d022de9f04f05460e460027146837
:101ac000dff88480dff884908db0002c3ad0606815
:101ad0000df10f018df80f7023f01dfe70bb049007
:101ae000adf814000df1100b5946606823f02fff7c
:101af000019018bb5846fff7adff8246f0b101993f
:101b0000102208a8aaf009fd5846eff75bf906abca
:101b1000cde909839df80f30cde906b0314628465e
:101b200008938df82ca028f0e7ff38b149462846e5
:101b300008aa29f06bf908b12468c6e700200db0a7
:101b4000bde8f08f0120fae7e518010210350d021b
:101b5000002330b585b0054601a8019323f0c2fcef
:101b6000041e0ddb019b28460393074b074902aa7d
:101b7000029300f073fa00eae074019823f0defcaf
:101b8000204605b030bd00bf351a0102b6340d0243
:101b9000f0b500269fb06a4647490546009600f01a
:101ba00097fa041ec0f282809df8000001a90196f8
:101bb00023f00afd041e79db019b23b90a203f4a6a
:101bc0003f49eff70dfa0026402200210ea8aaf0a7
:101bd000a4fc04af009b394601980d930496adf820
:101be000146023f0b4fe041e60db3846eff7eaf819
:101bf00006ab0f93334bcde9067038460e93fff7d3
